:020000040800F2
:1080000060CC0020A1810008A98100082DAA0008E9
:10801000AD810008AF810008B181000800000000B8
:10802000000000000000000000000000B381000814
:10803000B581000800000000B7810008B981000880
:10804000BB810008BB810008BB810008BB81000820
:10805000BB810008BB810008BB810008BB81000810
:10806000BB810008BB810008BB810008BB81000800
:10807000BB810008BB810008379900083F990008C0
:10808000BB81000847990008BB810008BB8100083C
:10809000BB810008BB810008BB810008BB810008D0
:1080A000BB810008BB810008BB810008BB810008C0
:1080B0007DAB0208BB810008BB810008BB810008C2
:1080C000BB810008BB810008BB810008BB810008A0
:1080D000BB81000857BB02085FBB020867BB0208F0
:1080E000AD9D0008BB810008BB810008BB81000872
:1080F000BB810008BB810008BB8100084F990008C4
:10810000BB810008BB810008BB810008BB8100085F
:1081100047BB02084FBB0208BB810008BB810008B7
:10812000BB810008BB810008BB810008BB8100083F
:10813000BB810008BB810008BB810008BB8100082F
:10814000BB810008BB810008BB810008BB8100081F
:10815000BB810008579900085F9900086FBB0208AF
:10816000BB810008BB810008BB810008BB810008FF
:10817000BB810008BB810008BB810008BB810008EF
:10818000BB810008BB810008DFF810D000F058FC6C
:108190000048004755D90208AFF3008060CC0020AA
:1081A0000648804706480047FEE7FEE7FEE7FEE791
:1081B000FEE7FEE7FEE7FEE7FEE7FEE715AB020897
:1081C000898100082DE9F0410024061B254671F144
:1081D000000605DA01240027D0EB070067EB010158
:1081E000161E73F1000605DA0027D2EB07020125FF
:1081F00067EB030300F0C1FA86460E4617469C461D
:10820000AC4204D00025D0EB050E65EB010624B18D
:108210000020D2EB000760EB030C704631463A4673
:108220006346BDE8F081202A06DBCB17203A41FAED
:1082300002F043EAE07306E041FA02F3D040C2F1F3
:108240002002914008431946704740EA01039B070A
:1082500003D009E008C9121F08C0042AFAD203E0BB
:1082600011F8013B00F8013B521EF9D27047421E43
:1082700012F8013F002BFBD111F8013B02F8013B42
:10828000002BF9D17047421C10F8011B0029FBD1CB
:10829000801A704730B505460020034600E05B1C9D
:1082A000934205D2EC5CC85C201A01D1002CF6D1B7
:1082B00030BD2DE9FE4F804681EA0300C00F0C4619
:1082C000009021F0004123F00045B8EB0200A941E5
:1082D00005D24046214690461C460B46024623F0F6
:1082E0000040104347D0270DC7F30A00C3F30A51DB
:1082F0000290401A019040286BDAC3F3130040F457
:10830000801B0098924620B10023D2EB030A63EB56
:108310000B0B01985946C0F14002504600F05EFA3E
:1083200006460D4650465946019AFFF77CFF10EB72
:1083300008006141002487EA115284EAE7731A4376
:1083400040D0009A62B3019A012A4FEA075215DC25
:10835000001B61EB02014FF0004202EA0752CDE937
:108360000042001C41F5801132462B4600F0EAFA2B
:1083700003B0BDE8F08F40462146F9E7001B61EBF2
:108380000201001C41F5801300185B412018A2F582
:10839000001747EB030140EAD570B6196D4111E0B3
:1083A0006D084FEA360645EAC0754FEA0752001BD2
:1083B00061EB0201001C41F5801149084FEA3000D1
:1083C0000019514132462B4603B0BDE8F04F00F092
:1083D000AABA0098012240000023D0EB020263EB0E
:1083E000E073009821464FEAE074B8EB000061EBBF
:1083F0000401E9E783F000435BE781F0004158E7BF
:108400002DE9FE4F81EA030404F0004421F000410D
:1084100000944FF0000B23F0004350EA01045ED0BB
:1084200052EA03045BD0C3F30A54C1F30A552C4447
:10843000A4F2F3340194A0FB0254C1F3130141F4FC
:108440008011C3F3130343F4801301FB024400FBC8
:10845000034E840A970A44EA815447EA8357A4FBEF
:10846000076802958D0A05FB07854FEA932C04FBEC
:108470000C542705029D4FEA065847EA1637B5EB1C
:1084800008056EEB070C870E920E47EA811742EA49
:108490008312A7FB0201B6EB0B0164EB00042B0D6A
:1084A00043EA0C335E1844EB1C50DA465146E7FBB6
:1084B0000201C5F313044FEA0B3343EA14534FEAA6
:1084C0000432019C43EA0603A4F10C040294009CCC
:1084D000CDE900B400F036FA03B0BDE8F08F00201B
:1084E0000146F9E72DE9F04D81EA030404F0004B61
:1084F00021F0004514464FF0000A23F0004150EAF5
:10850000050220D054EA01021DD0C5F30A570246E5
:10851000C5F31303C1F31300C1F30A5640F48015E9
:1085200043F48013A7EB0608101BD64608F2FD386B
:1085300073EB050002D308F1010801E092185B41DA
:10854000B8F1000F03DA00200146BDE8F08D0020ED
:108550004FF48011064684460EE0171B73EB0507A7
:1085600005D3121B63EB050306434CEA010C4908D3
:108570004FEA300092185B4150EA0107EDD152EA10
:10858000030012D082EA040083EA0501084305D003
:10859000101BAB4106D20122002306E000224FF05F
:1085A000004302E06FF0010253101AEB06004CEB9F
:1085B000085110EB0A0041EB0B01BDE8F04D00F053
:1085C000B2B9F0B4CA17CB0F50405140C61841F1B0
:1085D00000054FEAC372314628004FF0960303D0DE
:1085E000B623F0BC00F071B930460021F9E70EB5B2
:1085F000C10F80EAE0700844CA07002140F233430B
:108600008DE80E000A460B4600F09CF903B000BD51
:108610000EB540F2334102910021CDE900110A4626
:108620000B4600F08FF903B000BD3EB5CA17CB0F63
:10863000002450405140C0186141DA0740F23343F2
:108640000094CDE901232246234600F07BF903B0D4
:1086500030BD10B500F0004420F00040C20DC0F362
:10866000160040F400007F2A02DA0020014610BD07
:108670000021962A03DCC2F19602D04002E0963A2D
:1086800000F0ACF8002CF2D00023D0EB030063EB39
:10869000010110BD70B5C1F30A5201F0004500247C
:1086A000C1F3130140F2FF3341F480119A4201DA21
:1086B000002070BD40F233439A42A2F2334203DC01
:1086C000524200F09AF800E090402C43F1D0404232
:1086D00070BD70B5C1F30A5201F000450024C1F32A
:1086E000130140F2FF3341F480119A4202DA002074
:1086F000014670BD40F233439A42A2F2334203DC9A
:10870000524200F07AF801E000F068F82C43F0D013
:108710000023D0EB030063EB010170BD00F00042C9
:1087200030F000400AD0C10D01F56071C0F31600B1
:1087300042EA0151C2084007114370470020014638
:10874000704701F0004330B421F0004150EA0102CB
:1087500006D00A0DA2F56072C1F31301002A02DCF3
:1087600030BC00207047440F44EAC104C100E01847
:1087700030BC00EBC25000F09FB82DE9F05F054619
:10878000002092469B4688460646814640241BE0D0
:10879000284641464746224600F02FF853465A469F
:1087A000C01A914110D311461846224600F016F81F
:1087B0002D1A67EB01084F4622460120002100F0E8
:1087C0000DF817EB00094E41201EA4F10104DFDC77
:1087D000484631462A464346BDE8F09F202A04DB3E
:1087E000203A00FA02F1002070479140C2F12003C4
:1087F00020FA03F3194390407047202A04DB203A03
:1088000021FA02F00021704721FA02F3D040C2F1B0
:108810002002914008431946704700000FB400231E
:1088200000B589B00CA900910B996FF00042CB60A4
:108830001E4B06931E4B07930423CDE901321D4ABC
:10884000089202466B46002000F0A6F909B05DF8D8
:1088500014FB70B586B006464FF0FF300091CDE9AD
:108860000101002015460C4604903246694604A8D2
:10887000FFF7D4FF02460498211825B108B1084635
:1088800000E020462860049800280DD0002A02DD70
:108890000098884208D0081B0094CDE901043246B4
:1088A000694604A8FFF7BAFF06B070BDD18D000875
:1088B000EF8D0008658A00080029A8BF7047401C9A
:1088C000490008BF20F00100704710B4B0FA80FCE6
:1088D00000FA0CF050EA010404BF10BC704749B123
:1088E000CCF1200421FA04F411FA0CF118BF012193
:1088F00021430843A3EB0C01CB1D4FEA00614FEA73
:10890000102042BF002010BC704700EBC350104441
:108910000029A4BF10BC7047401C490008BF20F0CC
:10892000010010BC704710B5141E73F1000408DA82
:10893000401C41F1000192185B411A4301D120F023
:10894000010010BD2DE9F04D92469B4611B1B1FAE0
:1089500081F202E0B0FA80F220329046FFF73EFF4B
:1089600004460F4640EA0A0041EA0B0153465A46C4
:10897000084313D0114653EA010019D0C8F1400250
:108980005046FFF73AFF05460E46504659464246C6
:10899000FFF724FF084305D0012004E020463946B4
:1089A000BDE8F08D0020054346EAE0762C433743CE
:1089B0000A986305E40AA0EB08000022FD0A44EAD5
:1089C00047540A3002D500200146E9E70105101995
:1089D0006941DDE9084500196941BDE8F04DA2E7AC
:1089E00070B521F0004303430CD0C1F30A550024B5
:1089F000D5EB040564EB0403D617AD1AB34102DBD3
:108A00000020014670BD201841EB025170BD0000EE
:108A100030B5041E71F1000404DB4FF00044404205
:108A200064EB0101141E73F1000405DB1C464FF0DA
:108A30000043524263EB0403994208BF904230BDA9
:108A4000064C074D06E0E06840F0010394E807009B
:108A500098471034AC42F6D3FFF79AFB505C0308FA
:108A6000705C0308C0B24FF4F05100F03BBA000054
:108A70002DE9FF4F087883B09946FF2805D0491C9F
:108A80002D2804D00024002008E000200BE0012461
:108A9000F9E700EB800003EB4000491C0B78FF2B4B
:108AA000F7D104B1404200230293147819461D46C1
:108AB0002D2C01D02B2C04D1521C2D2C13D0002492
:108AC0000294AA461478FF2C0FD00A25A3FB057840
:108AD00001FB05814FF0000C03FB0C11521CE31944
:108AE0004AEB0101EEE70124EAE7814453EA010081
:108AF00002D019F5C87F06DA03980021C0E90011F9
:108B000007B0BDE8F08F0025AE4E2F46DFF8B882E3
:108B1000184600F0FBF9CDE90001B9F1000002DAD6
:108B2000C9F1000400E004460023A74A1AEB030B36
:108B300042EB045A12E0E00707D02A463346384693
:108B40004146FFF75DFC074688462A4633461046F5
:108B50001946FFF755FC05460E466410002CEAD175
:108B6000DDE90001B9F1000F5A46534606DAFFF776
:108B7000B9FC3A464346FFF7B5FC05E0FFF740FC79
:108B80003A464346FFF73CFC029A0AB181F00041A5
:108B9000039AC2E90001B3E72DE9FF4F1F468DB0EC
:108BA000D7E901464FF0FF382E2045464FF0000927
:108BB0000B90B9696D1C0E988847396A82468847C0
:108BC0000028F6D1BAF1FF3F0AD024F4D064002E79
:108BD00011DDBAF12B0F08D0BAF12D0F0BD102E045
:108BE000404611B08DE744F48064B9696D1C0E985D
:108BF00088478246761E6946600501D52D2000E033
:108C00002B208DF8000001F1010B0DF1200809E087
:108C1000B9696D1C0E98884782460F9844F4007419
:108C2000761E0560002E02DDBAF1300FF0D00B99F0
:108C30008A453ED144F0800406E00F99681CA9F1F2
:108C4000010944F400740860B9696D1C761E0E9821
:108C5000884782463028F0D02BE00B998A4505D111
:108C6000200603D444F08004761E18E0504624F019
:108C7000BDFA08B30DF11301761E44F400748B4560
:108C800008D2AAF130000BF8010B200607D5A9F194
:108C9000010003E0200602D409F101008146A0058D
:108CA00002D50F99681C0860B9696D1C0E98884739
:108CB0008246002ED1DC53E0002E51DDBAF1650F63
:108CC00002D0BAF1450F4BD1A00549D5B9696D1C49
:108CD00024F44074761E0E9888478246002E0CDDE0
:108CE0002B2804D0BAF12D0F07D144F48074B96950
:108CF0006D1C0E9888478246761EE00501D52D2111
:108D000000E02B2108F8011BCDF82C8021E00DF1AB
:108D10002901761E44F4007488450CD2AAF1300073
:108D200010F0FF0088F8000002D10B99884509D99E
:108D300008F1010806E0E00501D5244801E042F20F
:108D40000F708146B9696D1C0E98884782460F984E
:108D50000560002E04DD504624F048FA0028D6D1E4
:108D6000F9690E988847FF208BF8000088F800000A
:108D70000020069007904B466A4608A906A8FFF710
:108D800077FEA00502D46FF001002AE714F0240F4B
:108D90000AD0E00714D1DDE906123868031D3B60F4
:108DA0000068C0E900120BE0DDE90601FFF7C9FC2D
:108DB0000146E00704D13868021D3A60006801608E
:108DC00028460EE7000014400000F03FF1D8FFFFF6
:108DD000426842B1016811F8013B23B1521EC0E95B
:108DE0000012184670470121C160881E7047426812
:108DF0005AB1C368016843B983688B4205D0491EE4
:108E0000521CC0E90012002070474FF0FF3070473D
:108E10002DE9F04D00231A461B1A8A4103DB00207E
:108E20000146BDE8F08DC1F30A52C1F3130141F4CC
:108E300080154FF0000BD10702D100186D41521E72
:108E40000027044640F2FF11384601EB620A3E4615
:108E50008046024600204FF48011FFF7CEFCC21975
:108E60007141BB1846EB0100B4EB030C75EB000C31
:108E700004D3E41A65EB000517460E46241908F1E1
:108E800001006D4180463428E3DDF91946EB060008
:108E9000091BA84103D24FF0FF32134601E0002224
:108EA00013461BEB070046EB0A51BDE8F04DFFF7F8
:108EB0003ABD000030B5041E71F1000404DB4FF030
:108EC0000044404264EB0101141E73F1000405DB11
:108ED0001C464FF00043524263EB04038B4208BF31
:108EE000824230BD7F2801D9002208E0064A02EB09
:108EF0005002C007127800D1120902F00F020120BF
:108F00009040084070470000105C03080EB540F226
:108F1000334202920022CDE900221346FFF712FDF0
:108F200003B000BD70B58C1810F8015B15F0070395
:108F300001D110F8013B2A1106D110F8012B03E0F2
:108F400010F8016B01F8016B5B1EF9D12B0705D4FA
:108F50000023521E0DD401F8013BFAE710F8013B43
:108F6000CB1A921C03E013F8015B01F8015B521E5F
:108F7000F9D5A142D8D3002070BD10B502461078B3
:108F800003E012F8014B2318D8B20B1EA1F1010423
:108F9000A1B2F6D110BD000070B5ADF5287D044634
:108FA0000D460020A790A690002604EB44004549FA
:108FB00001EBC000408AA84203DC00200DF5287DAB
:108FC00070BD0020A69077E004EB44003D4B03EB1E
:108FD000C000028A04EB440003EBC00080892844EF
:108FE00081B2394800F010F90020A79011E004EB9D
:108FF0004400344901EBC0004068BDF89C12405C5D
:1090000001A9BDF89C228854BDF89C02401C80B286
:10901000A79004EB44002B4901EBC000008ABDF887
:109020009C128842E3DC04EB4400264A02EBC000B9
:10903000008A401E81B201A8FFF79FFF23490870F4
:1090400004EB44001F4901EBC000008A401E01A947
:10905000085C1E490978884226D10020A79016E0B6
:1090600004EB4400174901EBC0004068BDF89C12B6
:10907000405C04EB4401134A02EBC1018968BDF86E
:109080009C228854BDF89C02401C80B2A79004EB3F
:1090900044000C4901EBC000008A401EBDF89C1240
:1090A0008842DDDC012089E7642024F0D7FABDF88E
:1090B0009802401C80B2A690BDF89802062883DB77
:1090C00000207BE70C320308C8850020310A00200D
:1090D0002DE9F043ADF5257D04460E460025002719
:1090E000A846A94604EB4400324901EBC000408A7F
:1090F000B04204DC00200DF5257DBDE8F08300259D
:1091000018E004EB44002B4901EBC0008068405D8F
:1091100004EB4401274A02EBC1014968485504EBBE
:109120004400114601EBC0004068405D0DF80500A9
:10913000681C85B204EB44001E4901EBC000008AA4
:10914000401EA842DDDC04EB44000A4602EBC000EE
:10915000008A401E81B26846FFF70FFF04EB44010E
:10916000144A02EBC101098A491E0DF801000027CB
:109170001BE004EB44000F4B03EBC000028A04EB3E
:10918000440003EBC0008089304481B2684600F09F
:109190004FF931462046FFF7FFFE012800D1AAE72C
:1091A000642024F05BFA781C87B2062FE1DB0020F4
:1091B000A1E700000C32030808B5002000901EF063
:1091C00077FC0F49087000F09BF80D4800782428C0
:1091D00004D0272807D028280FD109E0002109480A
:1091E00080F8ED1109E00121064880F8ED1104E056
:1091F0000221044880F8ED1100BF00BF08BD000047
:109200002C0A0020BC2200202DE9F04106460D4624
:1092100017460024012023F0E0FF002028490880A1
:109220000DE01EF027FC00F0800000B10BE00120F3
:1092300024F014FA22480088401C21490880204864
:109240000088C828EDDB00BF1D480088C82832DA36
:1092500010211C4801F0DEFB08211A4801F0DCFB5C
:10926000E82000F031F8C5F3871000F02DF8A906CA
:10927000080E00F029F8002000F026F8002404E091
:10928000002000F021F8601C84B2042CF8DB0024DC
:1092900005E0FF2000F018F83055601C84B2BC4295
:1092A000F7DB1021074801F0B7FB002023F095FF02
:1092B0000120BDE8F081002023F08FFF0020F8E7B7
:1092C0002E0A00200000024010B5044600BF022113
:1092D0000A481EF0FDFC0028F9D0214607481EF080
:1092E00003FD00BF012105481EF0F2FC0028F9D063
:1092F00002481EF0F6FCC0B210BD00000030014074
:1093000010B5012023F069FF00201E4908800DE000
:109310001EF0B0FB00F0800000B10BE0012024F053
:109320009DF918480088401C164908801548008897
:10933000C828EDDB00BF13480088C8281CDA1021BC
:10934000114801F067FB08210F4801F065FB3D2043
:10935000FFF7BAFF2A20FFF7B7FF8020FFF7B4FF1F
:10936000A720FFF7B1FF1021074801F055FB0020AF
:1093700023F033FF012010BD002023F02EFF00203A
:10938000F9E700002E0A00200000024070B50546F3
:109390000E460024012023F020FF002022490880EF
:1093A0000DE01EF067FB00F0800000B10BE0012033
:1093B00024F054F91C480088401C1B4908801A48B6
:1093C0000088C828EDDB00BF17480088C82825DAC8
:1093D0001021164801F01EFB0821144801F01CFB67
:1093E0008420FFF771FF0020FFF76EFF0020FFF7DA
:1093F0006BFF0020FFF768FF002404E0285DFFF703
:1094000063FF601C84B2B442F8DB1021074801F00E
:1094100003FB002023F0E1FE012070BD002023F0BB
:10942000DCFE0020F9E700002E0A002000000240C8
:1094300070B506460C461546012023F0CEFE29469F
:109440003046FFF7A3FF08B9002070BD00201F4978
:1094500008800DE01EF00EFB00F0800000B10BE074
:10946000012024F0FBF819480088401C17490880A7
:1094700016480088C828EDDB00BF14480088C828BB
:109480001EDA1021124801F0C5FA0821104801F037
:10949000C3FA8320FFF718FFC4F38710FFF714FF08
:1094A000A106080EFFF710FF0020FFF70DFF1021A7
:1094B000074801F0B1FA002023F08FFE0120C4E735
:1094C000002023F08AFE0020BFE700002E0A0020C3
:1094D0000000024030B502460020002304E012F8EC
:1094E000014B60405C1CE3B28B42F8DB30BD0000F6
:1094F00010B50446392024F0C9FAE0B224F0E6FAA7
:10950000C4F3072024F0E2FAC4F3074024F0DEFAA3
:10951000200E24F0DBFA4FF48051034801F07CFA6E
:1095200022F068FC10BD0000000402402DE9F0416B
:1095300007460E4614463A2024F0A8FAF0B224F06A
:10954000C5FA301224F0C2FA4FF480510F4801F0EE
:1095500063FA19E022F04EFC05461D2D11D1384664
:1095600000F0ACF805463B2024F090FA4FF480510F
:10957000064801F051FA2F4434B120882844208055
:1095800002E02846BDE8F081E4E700000004024064
:109590002DE9F04107460E4614463C2024F076FAA9
:1095A000F0B224F093FA301224F090FA4FF4805184
:1095B000104801F031FA0CB10020208019E022F0AF
:1095C00019FC05461E2D11D1384600F02BF9054631
:1095D0003D2024F05BFA4FF48051064801F01CFA5C
:1095E0002F4434B120882844208002E02846BDE87A
:1095F000F081E4E70004024010B51EF033F908B131
:1096000000F02EF8302000F0A9F810BD10B5044687
:109610002146362000F08EF810BD10B5044614B176
:10962000204600F0ABF8342000F098F810BD10B5DB
:109630000446204600F0A2F820785C2802D020786A
:109640002F2803D10021642000F008F9322000F017
:1096500085F810BD10B5682000F04CF810BD000072
:1096600010B5222024F012FA24F005FA04464FF433
:109670008051024801F0D0F9204610BD000402409C
:109680002DE9F04124F0F7F9044624F0F4F90546F9
:1096900024F0F1F9064624F0EEF907464FF4805124
:1096A000054801F0B9F944EA052040EA064040EADD
:1096B0000760BDE8F08100000004024070B5044678
:1096C000272024F0E3F924F0D6F90646054646B1F2
:1096D00000BF24F0D0F92070641C701EC0B2061EBA
:1096E000F7D14FF48051024801F096F9284670BD39
:1096F0000004024010B504460C2024F0C7F92046AF
:1097000024F0E4F9FFF7BCFF10BD000070B504467B
:109710000A2024F0BBF9204624F0D8F924F0ABF954
:1097200005464FF48051024801F076F9284670BD95
:109730000004024070B505460C46284624F0A6F900
:10974000204624F0C3F94FF48051034801F064F936
:1097500022F050FB70BD00000004024010B504462A
:10976000204624F093F94FF48051034801F054F956
:1097700022F040FB10BD0000000402402DE9F04142
:109780000646012024F082F924F075F943282BDAEB
:109790002B20FFF7BBFF102826DA2F2024F076F9C4
:1097A000002024F093F93220FFF7D8FF0446142C50
:1097B0001AD1CF20FFF7AAFF0446ACB14C20FFF727
:1097C00099FF00EB042739464C2000F047F8502061
:1097D000FFF790FF00EB04273946502000F03EF8D9
:1097E0000021702000F03AF82F2024F04FF935784E
:1097F000284624F06BF909E0761C35785C2D01D001
:109800002F2D00D10025284624F060F9002DF3D13A
:109810004FF48051024801F0FFF8BDE8F0810000EC
:109820000004024070B504462D2024F02FF924F0E6
:1098300022F90646054646B100BF207824F046F9D5
:10984000641C701EC0B2061EF7D14FF4805102484E
:1098500001F0E2F8284670BD0004024070B50546EC
:109860000C460D2024F012F9284624F02FF9E0B21E
:1098700024F02CF9C4F3072024F028F9C4F307409E
:1098800024F024F9200E24F021F94FF480510248ED
:1098900001F0C2F870BD00000004024070B502463D
:1098A0000C46FF25FF2309E012F8010B80EA0501B1
:1098B0000648405C80EA03050548435C201EA4F18D
:1098C0000106B4B2F0D145EA032070BD9B2F030816
:1098D0009B3003082DE9F04103460C460020014669
:1098E000024606E013F8010B411842F10002601E27
:1098F00084B2002CF6DC080C40EA024C100C8DB24D
:109900001CEB050140F10002080C40EA024041183E
:109910006FEA010080B2BDE8F08130B50246002058
:10992000002305E012F8015B2C18E0B25C1CE3B2E6
:109930008B42F7DB30BD10B513F0A4FB10BD10B5A2
:1099400013F03EFB10BD10B513F00AFB10BD10B5AF
:1099500013F066FB10BD10B515F0F2FA10BD10B58E
:109960001DF066FB10BD00000246094B9A4201D271
:10997000084801E00648103801F000531BB1064BBF
:109980000B40C36002E0044B0B4083607047000053
:1099900010640240006002407D0F7D0F21B102681B
:1099A00042F00102026003E0026822F0010202605C
:1099B00070470000016821F0010101600021016091
:1099C00041608160C1600161212141614A49884251
:1099D00004D13D21484A103A91608CE04649183143
:1099E000884205D14FF47461434A103A916082E095
:1099F00041493031884205D14FF474113E4A103A42
:109A0000916078E03C494831884205D14FF074615B
:109A1000394A103A91606EE037496031884204D18A
:109A20003649354A103AD16065E033497831884289
:109A300004D13349304A103AD1605CE02E4990316C
:109A4000884204D12F492C4A103AD16053E02A4968
:109A5000A831884205D14FF03D51274A103AD160D4
:109A600049E02949884204D13D21274A083A11603A
:109A700041E025491831884205D14FF47461224AEA
:109A8000083A116037E020493031884205D14FF45F
:109A900074111D4A083A11602DE01B494831884273
:109AA00005D14FF07461184A083A116023E0164955
:109AB0006031884204D11149134A121F11601AE023
:109AC00011497831884204D10D490F4A121F1160A3
:109AD00011E00D499031884204D10A490A4A121F07
:109AE000116008E00849A831884204D14FF03D5187
:109AF000054A121F11607047106002403D000020AF
:109B0000400F002000003D201064024010B501F01D
:109B100080034BB122B1436943F08003436103E00A
:109B2000436923F08003436180290BD02AB1036885
:109B300001F01E042343036004E0036801F01E04E7
:109B4000A343036010BD000010B500220268134B50
:109B50001A40CC680B6823434C6923438C69234328
:109B6000CC6923430C6A23434C6A23438C6A234306
:109B70004C6B23438C6B23431A430260426922F0EF
:109B80000702D1E90B3423431A4342610B69436056
:109B90004B6883608B68C36010BD00003F801CF081
:109BA0001CB50024012120201DF068FE302000900B
:109BB00001208DF8040000208DF8060003208DF8A8
:109BC000050000208DF807006946184800F0AEFE39
:109BD0003021164800F020FF0021154880F87C163F
:109BE00000201449887001204870C8704FF4FA7042
:109BF000886000F025F80E4890F8F003802813D113
:109C000000200D49C86524200C49487108200871BE
:109C10003020C8701420887020204870002104482B
:109C200080F8F01300F050F81CBD00000014024052
:109C3000BC22002038290020BC120020AC260020C5
:109C40001CB523F0E7FDD02023F0B0FD23F016FE75
:109C5000002023F0ABFD23F011FE23F0DBFDD1202B
:109C600023F0A4FD23F00AFE00240EE0062C05DA02
:109C7000012023F06BFD0DF8040004E0002023F028
:109C800065FD0DF80400601CC4B2072CEEDB23F068
:109C9000DBFD9DF806000A4948719DF80500087132
:109CA0009DF80400C8709DF8020088709DF80100BE
:109CB00048709DF80010034880F8F0131CBD0000A8
:109CC000AC260020BC2200201CB500241B4890F8C4
:109CD000F0038DF800001A4840788DF8010018480C
:109CE00080788DF8020001208DF803001448C078B8
:109CF0008DF80400124800798DF80500104840796D
:109D00008DF8060023F086FDD02023F04FFD23F0D0
:109D1000B5FD002023F04AFD23F0B0FD00BF07E0B1
:109D20001DF8040023F042FD23F0A8FD601CC4B21E
:109D3000072CF5DB23F088FD1CBD0000BC220020B1
:109D4000AC26002070B502460C460025002309E031
:109D500012F8010B80EA05010648405C80EA030521
:109D60000548435C201EA4F10106B4B2F0D145EAD7
:109D7000032070BD9B2F03089B30030810B50446D9
:109D80000B460021072A00DD072244EA0420014691
:109D90002BB901FA02F081B20912084610BD012B5D
:109DA00002D11141C8B2F9E700BFF7E7704710B51B
:109DB00004460B460021072A00DD072244EA04205E
:109DC000014613B91141C8B210BD012B05D101FAEA
:109DD00002F081B209120846F6E700BFF4E700007E
:109DE000F0B5ADF5317D04460D460020B090AF9042
:109DF000002604EB4400544901EBC000408AA8420D
:109E000003DC00200DF5317DF0BD0020AF9094E023
:109E10004D480122C1684D4800F0A2FA4A48406806
:109E200000788DF800009DF8000038287DD104EB03
:109E30004400454B03EBC000C06804EB4403424FB1
:109E400007EBC3031B8A03FB050104EB44003B46FD
:109E500003EBC000028A3D4800F082FA0020B09077
:109E600011E004EB4400384901EBC0004068BDF844
:109E7000C012405CBDF8C0220DF80200BDF8C0025F
:109E8000401C80B2B09004EB44002F4901EBC000AD
:109E9000008ABDF8C0128842E3DC04EB44002A4A81
:109EA00002EBC000008A401E81B2684600F01EFB33
:109EB000064604EB4400244901EBC000008A401E22
:109EC0001DF80000B04230D10020B0901FE004EB3C
:109ED00044001D4901EBC0004068BDF8C012415C60
:109EE00004EB4400184A02EBC0008068BDF8C022B1
:109EF000024404EB4400144B03EBC000008A401EF4
:109F000068431154BDF8C002401C80B2B09004EB0D
:109F100044000D4901EBC000008A401EBDF8C0128C
:109F20008842D4DC01206DE7FFE7642023F096FB34
:109F3000BDF8BC02401C80B2AF90BDF8BC02062840
:109F4000FFF666AF00205DE7C0E00208D8580020A9
:109F50002DE9F041ADF5307D04460E460025002781
:109F6000A8460020009004EB4400474901EBC000E4
:109F7000408AB04204DC00200DF5307DBDE8F08160
:109F800000210846FFF72CFF01287AD1002520E0A8
:109F900004EB44003C4901EBC0008068411904EB2C
:109FA0004400394A02EBC000008A401E7043085C3E
:109FB00004EB440102EBC1014968485504EB44003D
:109FC000114601EBC0004068405D01A94855681C7E
:109FD00085B204EB44002C4901EBC000008AA84282
:109FE000D6DC00274BE004EB4400274B03EBC0001A
:109FF000C06804EB4403DFF890C00CEBC3031B8A7A
:10A0000003FB060104EB4400634603EBC000008A37
:10A01000401E82B21D4800F025FA04EB44001A4AA3
:10A0200002EBC000008A401E81B201A800F05EFA77
:10A03000009004EB4400144A02EBC000C06804EB3B
:10A040004402114B03EBC202128A104404EB440297
:10A0500003EBC202128A02FB0600411E012268467F
:10A0600000F000FA31462046FFF7BAFE012801D180
:10A0700082E706E0642023F0F1FA781C87B2062F0D
:10A08000B1DB002078E70000C0E00208D8580020CB
:10A0900070B5ADF5307D00250024002000905149B9
:10A0A000088080E000256FE0002414E04D4800881F
:10A0B00000EB40004C4951F83000005D49490988E7
:10A0C00001EB4101484A02EBC1014968085501A969
:10A0D0000855601C84B24348008800EB40004249A8
:10A0E00001EBC000008A401EA042DFDC3D48008832
:10A0F00000EB40000A4602EBC000008A401E81B21D
:10A1000001A800F0F3F900903648008800EB400009
:10A11000354B03EBC000C068324B1B8803EB430395
:10A12000314E06EBC3031B8A03FB05012D48008853
:10A1300000EB4000334603EBC000008A401E82B2B1
:10A140002A4800F08FF92748008800EB400032468B
:10A1500002EBC000C068234A128802EB4202334679
:10A1600003EBC202128A10441E4A128802EB42021A
:10A1700003EBC202128A02FB0500411E012268465F
:10A1800000F070F9681C85B21648008800EB4000AA
:10A19000154901EBC000408AA84285DC11480088BF
:10A1A000401C104908800F4800880B28FFF67AAF42
:10A1B0000F4890F8E00120F001010D4880F8E0110F
:10A1C00090F8E00120F00600801D094981F8E001C7
:10A1D0000021084841800120FFF7BAFE0DF5307DCF
:10A1E00070BD000010000020C0E00208D858002018
:10A1F000BC2200209C2400201CB5012108461DF033
:10A200003DFB01208DF8040002208DF805000020A0
:10A210008DF8060001208DF807001820009069468F
:10A22000144800F083FB05221146124800F0C6FBDB
:10A23000052206210F4800F0C1FB052207210D4829
:10A2400000F0BCFBA020009002208DF80400032049
:10A250008DF8050000208DF806008DF8070069468E
:10A26000044800F063FB402000906946014800F07C
:10A270005DFB1CBD000002402DE9F84300240027CF
:10A28000A046002000900025FFF7B6FF00F0BAF8C6
:10A2900000BF00E06D1C2D488542FBD36E460821AF
:10A2A0002B4800F0B7FB1021294800F0B5FB062031
:10A2B00000F08CF80821264800F0AEFB0821244865
:10A2C00000F0A8FB1021224800F0A6FB012000F0BE
:10A2D0007DF8002000F07AF808211D4800F09CFB72
:10A2E0001C48D0F8FC10B0F80021B0F8020102FBC5
:10A2F0000010B0F5003F02D900BE00BFFEE71648CF
:10A30000006808B9FFF7C4FE00201449088017E070
:10A31000002406E0114908782146FFF761FD601C22
:10A3200084B20E48008800EB40000A4901EBC000EF
:10A33000408AA042EEDC09480088401C074908809A
:10A34000064800880B28E3DBBDE8F883FFFF0F0019
:10A3500000000240C0E002081C024342100000203E
:10A360002DE9F04105460C4616460027012022F053
:10A3700031FF0821144800F04DFB1021124800F075
:10A380004BFB032000F022F8C4F3074000F01EF856
:10A39000C4F3072000F01AF8E0B200F017F800BF8D
:10A3A00006E0002000F012F828706D1C781C87B2BF
:10A3B000B742F6DB0821044800F02EFB002022F013
:10A3C00009FFBDE8F08100000000024010B504461E
:10A3D00000BF02210A481DF07BFC0028F9D021466D
:10A3E00007481DF081FC00BF012105481DF070FCED
:10A3F0000028F9D002481DF074FCC0B210BD000066
:10A400000030014000B585B0012108031DF086FA37
:10A4100013481DF031FC0020ADF80000ADF8040039
:10A42000ADF80600ADF808004FF40070ADF80A0072
:10A430003820ADF80C000020ADF80E000720ADF874
:10A4400010004FF48270ADF80200694604481DF018
:10A450004DFC012102481DF003FC05B000BD0000C9
:10A46000003001402DE9F04105460C461646002714
:10A47000012022F0AFFE08211B4800F0CBFA10218A
:10A48000194800F0C9FA0620FFF7A0FF0821164876
:10A4900000F0C2FA0821144800F0BCFA102112485A
:10A4A00000F0BAFA0220FFF791FFC4F30740FFF76C
:10A4B0008DFFC4F30720FFF789FFE0B2FFF786FFA7
:10A4C00000BF05E02878FFF781FF6D1C781C87B27C
:10A4D000B742F7DB0821044800F09EFA002022F082
:10A4E00079FEBDE8F08100000000024010B5024690
:10A4F000107803E012F8014B2318D8B20B1EA1F11B
:10A500000104A1B2F6D110BD2C48807C012854D1A1
:10A5100000212A4881742A480078C0B901202849BE
:10A52000087028480068C0002749D1F8301240EA76
:10A5300081002549D1F82C1240EA41002249D1F886
:10A54000281208430F2181432048017017E00020A2
:10A550001B4908701B480068C0001B49D1F8301225
:10A5600040EA81001849D1F82C1240EA410016490E
:10A57000D1F8281208430F21814315480170134870
:10A58000007813490978884217D11048007811499A
:10A590000870084600781049097888420DD00D48A7
:10A5A0000078064908730B4800780B490870094881
:10A5B000007810B101200149C8727047BC12002018
:10A5C000DE0A00203402424200004242DF0A00203C
:10A5D000E00A0020E10A0020DD0A002010B5ADF5F8
:10A5E0007C7D00247DA00068FB9000200090FFF798
:10A5F00003F814287CD17A48FFF719F879490870D4
:10A6000008460078142874D1FFF724F80021764A10
:10A6100003C2BDF80000FEF76BFF6A464FF4FA7103
:10A6200001A8FEF783FF71A101A823F0CBF97149BE
:10A6300008800846008810B300BF04E000216E487F
:10A640000155601C84B2282CF8DB01A9694A1288E4
:10A6500088186AA123F0B6F969490880002409E046
:10A6600064480088C01C204401A9095C6248015567
:10A67000601C84B262480088001FA042F0DC61A127
:10A6800001A823F09FF95B4908800846008820B3A1
:10A69000002405E00021584828300155601C84B290
:10A6A000282CF7DB01A9534A1288881853A123F0FC
:10A6B00089F95349088000240AE04E480088083090
:10A6C000204401A9095C4C4828300155601C84B223
:10A6D0004B4800880938A042EFDC4DA101A823F0C7
:10A6E00071F9444908800846008830B3002407E027
:10A6F0006BE05BE00021404850300155601C84B2A3
:10A70000142CF7DB01A93B4A128888183BA123F0DF
:10A7100059F93B49088000240AE0364800880C308B
:10A72000204401A9095C344850300155601C84B2B2
:10A73000334800880D38A042EFDC39A101A823F08E
:10A7400041F92C4908800846008820B3002405E020
:10A750000020294946390855601C84B2322CF7DBA9
:10A7600001A9244A1288881824A123F02BF924492E
:10A77000088000240AE01F480088801D204401A9A9
:10A78000085C1D4946390855601C84B21C48008885
:10A79000C01FA042EFDC00210320FFF7D9FB0120FE
:10A7A000FEF734FF01200DF57C7D10BD0D480078CB
:10A7B000422803D10A48FEF730FF0CE00120FEF7E3
:10A7C00025FF00200749087005E00021164880F8A1
:10A7D000EF1323F089F800BFE5E700000D0A000041
:10A7E000480A0020380A0020400A002041504E3D0F
:10A7F000000000005E0A0020082A00203B00000044
:10A800005C0A0020574946494E414D453D00000035
:10A810005749464950415353574F52443D00000059
:10A820005345525645523D00BC22002010B5044607
:10A830003548844208D1012108461DF02FF8002137
:10A8400001201DF02BF85EE03048844208D1012140
:10A8500002201DF023F8002102201DF01FF852E015
:10A860002B48844208D1012104201DF017F8002153
:10A8700004201DF013F846E02648844208D1012147
:10A8800008201DF00BF8002108201DF007F83AE021
:10A890002148844208D1012110201CF0FFFF002133
:10A8A00010201CF0FBFF2EE01C48844208D101213F
:10A8B00020201CF0F3FF002120201CF0EFFF22E0FD
:10A8C0001748844208D1012140201CF0E7FF0021F5
:10A8D00040201CF0E3FF16E01248844208D1012119
:10A8E00080201CF0DBFF002180201CF0D7FF0AE055
:10A8F0000D48844207D1012180151CF0CFFF0021B3
:10A90000A0151CF0CBFF10BD000002400004024067
:10A9100000080240000C02400010024000140240F7
:10A9200000180240001C024000200240F0B50A4618
:10A9300000210023002400BF3DE0012505FA01F3BA
:10A94000156805EA03049C4234D105684F000326CC
:10A95000BE40B543056015794E00B54006683543E5
:10A9600005601579012D02D01579022D16D1856863
:10A970004F000326BE40B543856055794E00B54073
:10A98000866835438560456801268E40B54345603D
:10A99000456896798E40B6B235434560C5684F002C
:10A9A0000326BE40B543C560D5794E00B540C668A4
:10A9B0003543C560491C1029BFD3F0BDF0B5002355
:10A9C00000244D07ED0E02FA05F3CE1000F120052C
:10A9D00055F826504E07F70E0F26BE40B543CF1050
:10A9E00000F1200646F82750CE1000F1200555F85A
:10A9F000265045EA0304CE1000F1200545F8264014
:10AA0000F0BD0246002013690B400BB1012000E0AD
:10AA10000020704741837047018370470249087BDB
:10AA20000021014A11737047BC12002003480068DE
:10AA300000F0010000B100BE00BFFEE7F0ED00E055
:10AA40004AF6AA2001490860704700000030004023
:10AA500030B502460024002305E012F8015B2819F6
:10AA6000C4B2581CC3B28B42F7DB6042C0B230BDE7
:10AA700010B5002422F038FF642022F0EFFD10BD55
:10AA80002DE9F043ADF2DC7D80460E461446994632
:10AA90000025002783A00068CDF8D807002001908A
:10AAA000042C7CDC80480079302101EB101004EB91
:10AAB000C40101EB04117D4A114408717A48007900
:10AAC00000F00F00303004EBC40101EB041111441D
:10AAD00048717548C078302101EB101004EBC401B7
:10AAE00001EB0411114488716F48C07800F00F0029
:10AAF000303004EBC40101EB04111144C871FEF7BE
:10AB00007BFD14287ED16A480078142809D004EB14
:10AB1000C40101EB0411654A8818FEF788FD6449F9
:10AB200008706348007814286DD1B6F57A7F01DD8E
:10AB30004FF47A76FEF78EFD00215E4A03C25D482F
:10AB40000068FEF7D5FC5848C078302101EB1010A2
:10AB50008DF808005448C07800F00F0030308DF8B0
:10AB600009005148807801EB10108DF80A004E481A
:10AB7000807800F00F0030308DF80B004A484078A4
:10AB800001EB10108DF80C004748407800F00F00E2
:10AB900030308DF80D00484890F8F00300E07CE07C
:10ABA00001EB10108DF80E00434890F8F00300F010
:10ABB0000F0030308DF80F00B9F1000F03D1542091
:10ABC0008DF8100005E0B9F1010F02D152208DF887
:10ABD00010003A208DF8110000252CE0284605EBE6
:10ABE000D071491018F801100F110A2097FBF0F0EE
:10ABF000C0EBC00107F130000844C1B202AA05F160
:10AC00000A0001E043E02EE01154284605EBD07124
:10AC1000491018F8011001F00F070A2097FBF0F017
:10AC2000C0EBC00107F130000844C1B205F10B00D0
:10AC30001154A81C85B2B5EB460FCFDB0A2000EB00
:10AC4000460081B201AA02A8FEF7A2FC01AA0221D5
:10AC50000DF5FB60FEF79CFC0120FEF7D7FC002001
:10AC60001349087019E012480078422808D104EB13
:10AC7000C40101EB04110D4A8818FEF7CEFC0CE06C
:10AC80000120FEF7C3FC00200949087005E00021FF
:10AC9000094880F8EF1322F027FE0DF2DC7DBDE8B5
:10ACA000F08300000D0A0000AC260020600A00209E
:10ACB000380A0020400A0020BC22002070B5B8B03D
:10ACC0000021369135913491339132913191309107
:10ACD00000222E922F922C922D922B912A91299123
:10ACE00028912791269125912391159114911391E3
:10ACF0001291119110910F919FEDFD0A8DED0E0AA9
:10AD0000FCA006C8CDE90C12FCA006C8CDE90A12C9
:10AD1000BBE0FC48807858B30020FA498870FA48B4
:10AD2000B0F8C805F9490968C1F57A7188421FD1A0
:10AD3000F6480068C0F57A7081B2F348A0F8C015F3
:10AD40000021F248001FFEF729FEF149EF48001FDD
:10AD5000FEF70AFE0120EF4908704FF47A70EB49C4
:10AD60008C39C1F88C000121E848001FFEF716FE5F
:10AD7000E448807B50B30021E2488173E648408874
:10AD8000E2498C39496CC1F57A7188421ED1DF489D
:10AD90008C38406CC0F57A70DF4908394880002152
:10ADA000DA484C38FEF7FAFDDC49D8484C38FEF753
:10ADB000DBFD0120DA4908704FF47A70D3498C39F1
:10ADC00048640121D1484C38FEF7E8FDCD48807E2B
:10ADD00050B30021CB488176CF488088CB498C394D
:10ADE0004969C1F57A7188421ED1C8488C384069DA
:10ADF000C0F57A70C849083988800021C3487C387A
:10AE0000FEF7CCFDC749C1487C38FEF7ADFD0120F7
:10AE1000C54908704FF47A70BC498C3948610121EA
:10AE2000BA487C38FEF7BAFDB64890F8260060B301
:10AE30000021B44880F82610B748C088B3498C393F
:10AE4000C96AC1F57A7188421FD1B0488C38C06A8E
:10AE5000C0F57A7081B2B0480838C1800021AB4893
:10AE60006438FEF79BFDB149A8486438FEF77CFDC5
:10AE70000120AF4908704FF47A70A4498C39C86238
:10AE80000121A2486438FEF789FD9E488178807BC5
:10AE900001449C48807E01449A4890F8260008446A
:10AEA00000287FF436AF0BF0E1BA9A48007820B161
:10AEB0000020984908702B9019E09948007828B133
:10AEC00000209749087001202B9010E096480078E8
:10AED00028B100209449087002202B9007E0944884
:10AEE000007820B100209249087003212B919DF831
:10AEF000AC1001EB4100C0EBC1108E4911F83000DD
:10AF0000C12836D19DF8AC1001EB4100C0EBC11156
:10AF1000884800EBC100807808282AD101217A48AE
:10AF200080F818169DF8AC0030B101280AD002282C
:10AF30000ED0032818D111E04FF480417E48FFF76E
:10AF400069FD11E04FF400517B48FFF763FD0BE012
:10AF50004FF480517848FFF75DFD05E04FF4006144
:10AF60007548FFF757FD00BF00BF00207349086018
:10AF700099E764480C389DF8AC1010F811000121D5
:10AF8000B1EBD01F4BF0D0809DF8AC0000EB40013E
:10AF900001EB00116A4800EB0110407B022841F0F0
:10AFA000FA8101F0EEB99DF8AC0000EB4001C1EB75
:10AFB000C010604901EBC000007C01069DF8AC00A8
:10AFC00000EB4002C2EBC0105A4A02EBC000407CCA
:10AFD00041EA00419DF8AC0000EB4002C2EBC0101A
:10AFE000544A02EBC000807C41EA00219DF8AC008D
:10AFF00000EB4002C2EBC0104E4A02EBC000C07C26
:10B00000084312904F489DF8AC1050F82120129838
:10B0100082426CD04B4A9DF8AC00129942F8201045
:10B020009DF8AC1001EB4100C0EBC110414901EBB0
:10B03000C000C17B9DF8AC0000EB4002C2EBC01029
:10B040003C4A02EBC000807B41EA00212891324952
:10B0500008399DF8AC0031F81010BDF8A0000A3096
:10B06000814211DB2C4908399DF8AC0031F81010F1
:10B07000BDF8A0000A30081A81B2274A083A9DF8A4
:10B08000AC0022F8101007E00020234908399DF891
:10B09000AC2021F81200FCE39DF8AC0000EB40016D
:10B0A000C1EBC010234901EBC000C01D0990BDF8E1
:10B0B000A010FEF7F3FB11909DF8AC0000EB4001EF
:10B0C000C1EBC0101B4901EBC002BDF8A000083065
:10B0D000125C9DF8AC0000EB4001C1EBC0101549BB
:10B0E00001EBC003BDF8A000C01D185C2CE0FCE320
:10B0F0000000000001693230313030000169323027
:10B1000045303000102E0020BC5200208C600240E0
:10B1100000880020120000208458002000802010A9
:10B120001300002020800010140000200088001070
:10B1300015000020246600200018024088024242C8
:10B140003C3000200C76002042EA00221198824216
:10B1500072D19DF8AC1001EB4100C0EBC110FE496B
:10B1600001EBC000407C00F00F0101EBD1700991B0
:10B1700041100998A0EB4100C1B214919DF8AC10A8
:10B1800001EB4100C0EBC110F34901EBC000C07CF2
:10B1900000F00F0101EBD1704010099113900020D5
:10B1A000369025E09DF8AC1001EB4100C0EBC110DA
:10B1B000E94901EBC001BDF8D8001430095C0991E0
:10B1C000DDE913210998FEF7D9FD01469DF8AC0091
:10B1D00000EB4002C2EBC010DF4A02EBC002BDF838
:10B1E000D80014301154BDF8D800401C81B23691FB
:10B1F000BDF8A000C01FBDF8D8108842D2DCD748E7
:10B2000090F8EF03A8B1BDF8A000801C81B20991AD
:10B210009DF8AC1001EB4100C0EBC111CE4800EB32
:10B22000C100C01D012308909DF8AC200999FFF7CB
:10B2300027FC002135914BE0FCE3002136912AE008
:10B240009DF8AC10C1EBC10000EB8111C44800EBCC
:10B250004111C91DBDF8D40000EB400202EBC00053
:10B2600001EB4001891CBDF8D800095C9DF8AC00D9
:10B2700000EB4002C2EBC010B74A02EBC002BDF8BF
:10B28000D8001430105C814200D008E0BDF8D8002E
:10B29000401C81B23691BDF8D8001428D0DB00BF25
:10B2A000BDF8D80014280ED1BDF8D400C1B29DF865
:10B2B000AC00C0EBC00202EB8012A94800EB4210C8
:10B2C00080F85F1008E0BDF8D400401C81B23591D1
:10B2D000BDF8D4000428B0DB00BFBDF8D4000428BA
:10B2E0005FD10020359057E09DF8AC00C0EBC00165
:10B2F00001EB80119A4800EB4110C01DBDF8D4103D
:10B3000001EB410202EBC10100EB41008078E8BB98
:10B310000020369027E09DF8AC0000EB4001C1EB27
:10B32000C0108D4901EBC001BDF8D80014300A5C93
:10B330009DF8AC00C0EBC00101EB8011884800EB28
:10B340004111C91DBDF8D40000EB400303EBC00060
:10B3500001EB4001891CBDF8D8000A54BDF8D800A3
:10B36000401C81B23691BDF8D8001428D3DBBDF85B
:10B37000D400C1B29DF8AC00C0EBC00202EB801259
:10B38000774800EB421080F85F1009E0FFE7BDF856
:10B39000D400401C81B23591BDF8D4000428A3DB51
:10B3A00000BF9DF8AC1001EB4100C0EBC1106A4931
:10B3B00001EBC00090F83210259133211091BDF8B7
:10B3C000940015287DD00FDCA0F10B000A2879D25B
:10B3D000DFE810F0340440044204410478007800AF
:10B3E000430444047800F706A1286CD006DC5028FA
:10B3F0006AD0512807D0522864D1F1E3A2287DD029
:10B40000A428F9D1F6E3BDF8A010BDF84000081A51
:10B41000C1B22391E8E39DF8AC1001EB4100C0EB11
:10B42000C1104D4901EBC001BDF84000095C2991F4
:10B43000BDF84000401C81B210919DF8AC1001EBAA
:10B440004100C0EBC110444901EBC001BDF8400010
:10B45000095C2A919DF8A80001287BD1BDF8400025
:10B46000401C81B210919DF8AC0000EB4001C1EB93
:10B47000C010394901EBC001BDF84000095C3391AF
:10B48000BDF84000401C81B210919DF8AC1001EB5A
:10B490004100C0EBC110304901EBC001BDF84000D4
:10B4A000095C3091BDF84000401C81B210919DF8BC
:10B4B000AC1001EB4100C0EBC110274901EBC0010A
:10B4C00003E0FDE3FDE394E396E3BDF84000095C8F
:10B4D0003191BDF84000401C81B210919DF8AC1034
:10B4E00001EB4100C0EBC1101B4901EBC001BDF8ED
:10B4F0004000095C3291BDF8400000E07BE3401C55
:10B5000081B21091BDF8401035912CE2BDF8400099
:10B51000401C81B210919DF8AC1001EB4100C0EBD2
:10B52000C1100D4901EBC001BDF84000095C249138
:10B53000BDF84000401C81B210919DF89000C0F30E
:10B54000801000287ED09DF890209DF8A40000EB8C
:10B55000400107E00DE2000024660020BC2200202C
:10B56000FC34002001EB0011F94800EB01113031EF
:10B570009DF89C0001EB001082709DF8A40000EB88
:10B58000400101EB0011F24800EB011030309DF852
:10B590009C1000EB01108078C0F3800020BB9DF868
:10B5A000A40000EB400101EB0011E94800EB0110A1
:10B5B00030309DF89C1000EB01108078C0F3C00083
:10B5C00090B99DF8A40000EB400101EB0011E048A8
:10B5D00000EB011030309DF89C1000EB01108078DA
:10B5E000C0F340000028ADD000202E902F90002105
:10B5F000369122E09DF8AC0000EB4001C1EBC01099
:10B60000D44901EBC001BDF84020BDF8D80010447A
:10B61000095CBDF8D800C0F10300C00001FA00F0D9
:10B62000C117DDE92E34184341EA0402CDE92E02A8
:10B63000BDF8D800401C80B23690BDF8D800042870
:10B64000D8DB00E079E19DF8A4002E9900EB4002E0
:10B6500002EB0012BE4800EB021230329DF89C0053
:10B6600002EB00104160BDF84000001D81B2109156
:10B6700000222E922F920021369122E09DF8AC10EC
:10B6800001EB4100C0EBC110B24901EBC001BDF8B4
:10B690004020BDF8D8001044095CBDF8D800C0F1C6
:10B6A0000300C00001FA00F0C117DDE92E34184391
:10B6B00041EA0402CDE92E02BDF8D800401C80B258
:10B6C0003690BDF8D8000428D8DB9DF8A4002E9948
:10B6D000C0EBC00202EB80129F4800EB42126032C6
:10B6E0009DF89C0000EB001002EBC000C0F81A109F
:10B6F000BDF84000001D81B2109100222E922F92C1
:10B700000021369122E09DF8AC1001EB4100C0EB26
:10B71000C110904901EBC001BDF84020BDF8D80030
:10B720001044095CBDF8D800C0F10300C00001FA64
:10B7300000F0C117DDE92E34184341EA0402CDE9D7
:10B740002E02BDF8D800401C80B23690BDF8D8005B
:10B750000428D8DB9DF8A4002E99C0EBC00202EBB0
:10B7600080127D4800EB421260329DF89C0000EB95
:10B77000001002EBC000C0F81E10BDF84000001D14
:10B7800081B2109100222E922F920021369122E058
:10B790009DF8AC1001EB4100C0EBC1106D4901EB0D
:10B7A000C001BDF84020BDF8D8001044095CBDF8C8
:10B7B000D800C0F10200C00001FA00F0C117DDE9B5
:10B7C0002E24104341EA0402CDE92E02BDF8D80030
:10B7D000401C80B23690BDF8D8000328D8DB9DF815
:10B7E000A410C1EBC10000EB81115B4800EB4110DC
:10B7F00060309DF89C1001EB011100EBC10034306A
:10B80000099000682E99084309990860BDF8400026
:10B81000C01C80B2109000222E922F9200203690F1
:10B8200022E09DF8AC1001EB4100C0EBC11049498A
:10B8300001EBC001BDF84020BDF8D8001044095C00
:10B84000BDF8D800C0F10500C00001FA00F0C11732
:10B85000DDE92E34184341EA0402CDE92E02BDF899
:10B86000D800401C80B23690BDF8D8000628D8DB3E
:10B870009DF8A400DDE92E12C0EBC00303EB80139A
:10B88000354800EB431360339DF89C0000EB00103B
:10B8900000E0FDE303EBC00040F8221F4260BDF86A
:10B8A0004000801D81B2109100222E922F92002123
:10B8B000369124E09DF8AC1001EB4100C0EBC110C3
:10B8C000244901EBC001BDF84020BDF8D800104468
:10B8D000095CBDF8D800C0F10500C00001FA00F015
:10B8E000C117DDE92E34184300E0FDE341EA04020C
:10B8F000CDE92E02BDF8D800401C80B23690BDF8CC
:10B90000D8000628D6DB9DF8A400DDE92E12C0EB96
:10B91000C00303EB8013104800EB431360339DF822
:10B920009C0000EB001003EBC00022308160C2607D
:10B93000BDF84000801D81B21091BDF84010BDF8E7
:10B94000D400091ABDF8C000801E814206DB0FE05A
:10B950003C30002024660020FC3400209DF89C0030
:10B96000401CC1B22791BDF8D40000287FF4CEADB1
:10B9700026E19DF8AC1001EB4100C0EBC110FE497F
:10B9800001EBC001BDF84000085C0328F0D1BDF810
:10B990004000401C81B210919DF8AC1001EB4100B9
:10B9A000C0EBC110F44901EBC001BDF84000095CD7
:10B9B0003391BDF84000401C81B210919DF8AC104D
:10B9C00001EB4100C0EBC110EB4901EBC001BDF838
:10B9D0004000095C3091BDF84000401C81B21091DC
:10B9E0009DF8AC0000EB4001C1EBC010E24901EB57
:10B9F000C001BDF84000095C3191BDF84000401C19
:10BA000081B210919DF8AC0000EB4001C1EBC01079
:10BA1000D94901EBC001BDF84000095C3291BDF885
:10BA20004000401C81B21091BDF8401035910021BA
:10BA30002791BFE0EDE3BDF84000401C81B21091BA
:10BA40009DF8AC0000EB4001C1EBC010CA4901EB0E
:10BA5000C001BDF84000095C2491BDF84000401CC5
:10BA600081B210919DF89000C0F38010F0B39DF862
:10BA700090209DF8A40000EB400101EB0011BF48AD
:10BA800000EB011130319DF89C0001EB0010827039
:10BA90009DF8A40000EB400101EB0011B74800EB5A
:10BAA000011030309DF89C1000EB01108078C0F33D
:10BAB0008000D8B100202E902F900021369129E0EF
:10BAC0009DF8AC0000EB4001C1EBC010AA4901EBAE
:10BAD000C001BDF84020BDF8D80010440A5C9DF8B4
:10BAE000A400C0EBC00101EB801100E052E0A448CB
:10BAF00000EB411160319DF89C0000EB001001EB60
:10BB0000C0013F31BDF8D8000A54BDF8D800401C30
:10BB100081B23691BDF8D8000A28D1DBBDF84000CB
:10BB20000A3081B2109100222E922F92002136917C
:10BB300027E09DF8AC1001EB4100C0EBC1108E492D
:10BB400001EBC001BDF84020BDF8D80010440A5CEC
:10BB50009DF8A400C0EBC00101EB8011884800EB08
:10BB6000411160319DF89C0000EB001001EBC00119
:10BB70005831BDF8D8000A54BDF8D800401C81B235
:10BB80003691BDF8D8000228D3DBBDF84000801CF8
:10BB900081B21091BDF84010BDF8D400091ABDF86B
:10BBA000C000801E814200DB09E09DF89C00401C23
:10BBB000C1B22791BDF8D40000287FF43CAF00BF8C
:10BBC000BDF84010BDF8A000801D81420ADCBDF820
:10BBD000A010891DBDF84000081AC1B2239103E0EE
:10BBE0003DE007E000202390239800287FF413AC69
:10BBF0000EE30DE30CE30BE39DF8AC1001EB410009
:10BC0000C0EBC1105C4901EBC001BDF84000095C0C
:10BC10009DF8AC00C0EBC00202EB8012584800EB6C
:10BC20004210817150219DF8AC00C0EBC00202EBC4
:10BC30008012534800EB42104171E9E20B219DF85C
:10BC4000AC00C0EBC00202EB80124D4800EB42108A
:10BC50004171DDE2DCE2DBE2DAE2D9E2D8E2522154
:10BC60009DF8AC00C0EBC00202EB8012444800EB30
:10BC700042104171BDF8A010BDF84000814207DDBF
:10BC8000BDF8A010BDF84000081AC1B2239101E030
:10BC9000002023909DF8AC0000EB4001C1EBC011E7
:10BCA000354800EBC101BDF840000A5C9DF8AC00CE
:10BCB000C0EBC00101EB8011314800EB411101E004
:10BCC00080E280E2C91D9DF8AC00C0EBC00303EB2D
:10BCD00080132B4800EB431090F85F0000EB40030B
:10BCE00003EBC00001EB40004270BDF84000401C77
:10BCF00081B210919DF8AC1001EB4100C0EBC11076
:10BD00001D4901EBC001BDF84000095C3491BDF84C
:10BD10004000401C81B210919DF8AC1001EB410035
:10BD2000C0EBC110144901EBC001BDF84000095C33
:10BD30003291BDF84000401C81B210910021359134
:10BD4000EBE19DF8AC1001EB4100C0EBC1100A49DA
:10BD500001EBC001BDF84000085C0A4981F82000F1
:10BD6000BDF84000401C81B2109100222E922F920B
:10BD7000002136912BE00000246600203C3000209A
:10BD8000FC340020BC1200209DF8AC1001EB4100F7
:10BD9000C0EBC110FE4901EBC001BDF84020BDF869
:10BDA000D8001044095CBDF8D800C0F10300C00001
:10BDB00001FA00F0C117DDE92E34184341EA04020C
:10BDC000CDE92E02BDF8D800401C80B23690BDF8F7
:10BDD000D8000428D8DBEF492E98C1F82100BDF81F
:10BDE0004000001D81B2109100222E922F9200215E
:10BDF000369122E09DF8AC1001EB4100C0EBC11080
:10BE0000E34901EBC001BDF84020BDF8D800104463
:10BE1000095CBDF8D800C0F10300C00001FA00F0D1
:10BE2000C117DDE92E34184341EA0402CDE92E02A0
:10BE3000BDF8D800401C80B23690BDF8D800042868
:10BE4000D8DBD4482E99C0F82510BDF84000001D5D
:10BE500081B2109100222E922F920021369122E081
:10BE60009DF8AC0000EB4001C1EBC010C84901EBEC
:10BE7000C001BDF84020BDF8D8001044095CBDF8F1
:10BE8000D800C0F10200C00001FA00F0C117DDE9DE
:10BE90002E34184341EA0402CDE92E02BDF8D80041
:10BEA000401C80B23690BDF8D8000328D8DBB949D1
:10BEB0002E98C1F82900BDF84000C01C81B2109135
:10BEC00000222E922F920021369122E09DF8AC00A4
:10BED00000EB4001C1EBC010AD4901EBC001BDF862
:10BEE0004020BDF8D8001044095CBDF8D800C0F16E
:10BEF0000500C00001FA00F0C117DDE92E34184337
:10BF000041EA0402CDE92E02BDF8D800401C80B2FF
:10BF10003690BDF8D8000628D8DB9E4A0D32DDE900
:10BF20002E1011625062BDF84000801D81B2109148
:10BF300000222E922F920021369122E09DF8AC0033
:10BF400000EB4001C1EBC010914901EBC001BDF80D
:10BF50004020BDF8D8001044095CBDF8D800C0F1FD
:10BF60000500C00001FA00F0C117DDE92E341843C6
:10BF700041EA0402CDE92E02BDF8D800401C80B28F
:10BF80003690BDF8D8000628D8DB82482D30DDE990
:10BF90002E128160C260BDF84000801D81B21091F8
:10BFA0009DF8AC0000EB4001C1EBC010784901EBFB
:10BFB000C001BDF84000095C764880F84610BDF825
:10BFC0004000401C81B210919DF8AC0000EB400194
:10BFD000C1EBC0106E4901EBC001BDF84000095C27
:10BFE0006C4880F84510BDF84000401C81B21091AB
:10BFF0009DF8AC0000EB4001C1EBC010644901EBBF
:10C00000C001BDF84000095C624880F84410BDF8EA
:10C010004000401C81B210919DF8AC0000EB400143
:10C02000C1EBC0105A4901EBC001BDF84000095CEA
:10C03000584880F84310BDF84000401C81B2109170
:10C040009DF8AC0000EB4001C1EBC010504901EB82
:10C05000C001BDF84000095C4E4880F84210BDF8B0
:10C060004000401C81B210919DF8AC1001EB4100E2
:10C07000C0EBC110464901EBC001BDF84000095CAE
:10C08000444880F84110BDF84000401C81B200E0F7
:10C090007FE1109100222E922F920021369122E012
:10C0A0009DF8AC1001EB4100C0EBC110384901EB29
:10C0B000C001BDF84020BDF8D8001044095CBDF8AF
:10C0C000D800C0F10300C00001FA00F0C117DDE99B
:10C0D0002E34184341EA0402CDE92E02BDF8D800FF
:10C0E000401C80B2369000E0B4E0BDF8D8000428CF
:10C0F000D6DB28492E98C1F847000846C06D81B2AA
:10C1000002200991FCF7E4FF00210620FDF720FF43
:10C11000BDF8D400401C81B23591BDF8D410BDF8F3
:10C12000D0008142FFF60DAE1A48C06D1949C98B87
:10C13000884206D21748C06DBDF8D0100844154992
:10C14000C86500210520FDF703FF01229DF8AC0022
:10C15000C0EBC00101EB80110F4800EB4111C91D7C
:10C160009DF8AC00C0EBC00303EB80130A4800EB62
:10C17000431090F85F0000EB400303EBC00001F8B0
:10C1800010200F2005490871BDF8401008E000009C
:10C1900024660020BC120020FC340020842A0020E9
:10C1A000BDF8A000801D814208DCBDF8A010891DEB
:10C1B000BDF84000081AC1B2239101E0002023908D
:10C1C00026E025E024E000219DF8AC00C0EBC00291
:10C1D00002EB8012FE4800EB42104171369112E0F2
:10C1E00000219DF8AC0000EB4002C2EBC010F94A00
:10C1F00002EBC002BDF8D8000D301154BDF8D800D4
:10C20000401C81B23691BDF8D8000528E8DB00BF9C
:10C2100027E00020369012E000219DF8AC0000EBF2
:10C220004002C2EBC010EB4A02EBC002BDF8D800DE
:10C230000D301154BDF8D800401C81B23691BDF8C4
:10C24000D8000528E8DB0020E3499DF8AC2021F860
:10C2500012009EE00021E0489DF8AC2020F812106A
:10C2600097E0DD489DF8AC1030F81100F0B39DF870
:10C27000AC1001EB4100C0EBC110D64901EBC0018D
:10C28000BDF8A0001130085CFA2802D111203590C9
:10C2900013E09DF8AC1001EB4100C0EBC110CD499B
:10C2A00001EBC001BDF8A0000A30085CFA2802D1F9
:10C2B0000A20359001E000203590BDF8D400002818
:10C2C00057DD0020369025E09DF8AC1001EB4100D1
:10C2D000C0EBC110BF4901EBC001BDF8A020BDF803
:10C2E000D4000244BDF8D800104400E049E0095CE5
:10C2F0009DF8AC0000EB4002C2EBC010B54A02EB67
:10C30000C002BDF8D800C01D1154BDF8D800401CB3
:10C3100081B23691B0499DF8AC0031F81010BDF8EB
:10C32000D8008142D0DC002036901DE00021BDF80D
:10C33000A020BDF8D4000244A74B9DF8AC0033F810
:10C3400010000244BDF8D80002449DF8AC0000EB98
:10C350004003C3EBC0109F4B03EBC0008154BDF8FA
:10C36000D800401C81B23691BDF8D8002828DDDB0A
:10C3700005E0002098499DF8AC2021F8120000202B
:10C38000289095489DF8AC1030F8110000287EF4F4
:10C390000AAE0AF06BB8914890F8EF03B0B18E493D
:10C3A0009DF8AC0031F8101009919DF8AC0000EB3D
:10C3B0004001C1EBC010874901EBC0010123089186
:10C3C0009DF8AC20DDE90801FEF75AFB9DF8AC10A2
:10C3D00001EB410000EB0111814800EB0110817974
:10C3E0002A919DF8A800092889F06886DFE810F0F6
:10C3F0000146090095114A20962CD22EDD325B377A
:10C4000004429DF8AC1001EB4100C0EBC110714932
:10C4100001EBC000417808460991002110F0BEFCF4
:10C42000C1B22791002134911CE09DF8AC1001EBC2
:10C43000410000EB01116A4800EB01113031BDF8F9
:10C44000D00001EB001041789DF89C00814204D19E
:10C45000BDF8D000C1B2279112E0BDF8D000401C59
:10C4600081B234919DF8AC1001EB410000EB011159
:10C470005B4800EB0110C179BDF8D0008142D4DCEB
:10C4800000BF9DF8AC1001EB4100C0EBC110514959
:10C4900001EBC000807800F0F000A0280DD19DF8DD
:10C4A000AC1001EB4100C0EBC1104A4901EBC000E8
:10C4B000807800F00F0128910AE09DF8AC1001EBA4
:10C4C0004100C0EBC110434901EBC00081782891C5
:10C4D000BDF8A00008B9102028909DF8AC1001EB21
:10C4E0004100C0EBC1103B4901EBC001BDF8A00009
:10C4F000401C095C2591BDF8A000401C81B2099147
:10C500009DF8AC0000EB4001C1EBC010314901EBDC
:10C51000C0010891DDE9080111F0D0F835909DF8CF
:10C52000AC1001EB4100C0EBC1102A4901EBC00186
:10C53000BDF8A000801C095CBDF8D400814242F027
:10C54000EA809DF8AC1001EB4100C0EBC11021491D
:10C5500001EBC0004078002842F3DD809DF8AC106C
:10C5600001EB4100C0EBC1101A4901EBC001BDF85D
:10C57000A000C01C0A5C9DF8AC00C0EBC00101EB40
:10C580008011134800EB411160319DF89C0000EBD5
:10C59000001001EBC00080F83C200021114A9DF8FA
:10C5A000AC0002EB00129DF89C0011540E48007F75
:10C5B000012850D19DF8AC1001EB410000EB0111B6
:10C5C000074800EB011030309DF89C100EE0000091
:10C5D000FC340020246600207C580020BC2200206F
:10C5E0003C300020702E0020BC12002000EB011017
:10C5F000801C0990007820F0800080300999087034
:10C60000BDF89400B62814D0C52819D0D52802D07A
:10C61000D9281CD106E0BDF8A000032801DA0020CB
:10C62000259017E0BDF8A000032801DA002025902E
:10C6300010E0BDF8A000032801DA0020259009E0F1
:10C64000BDF8A000032801DA0020259002E00020B8
:10C65000259000BF00BF9DF8AC1001EB410000EB3E
:10C660000111FE4800EB011030309DF89C1000EBEA
:10C670000110801C0990007820F04000403009999A
:10C680000870BDF89400C5287ED016DCB5287CD093
:10C690000CDC112801F0DA86122801F01987132822
:10C6A00001F0A287B22842F03580E8E3B6286DD0C9
:10C6B000B9286CD0C328F6D1EAE3D92868D007DCC2
:10C6C000CA2866D0CE2801F0E785D528EBD109E04D
:10C6D000E12801F0F485E52801F00486E728E2D19D
:10C6E00001F09DBE9DF8AC1001EB4100C0EBC11004
:10C6F000DB4901EBC000C178DA4880F8E6119DF80B
:10C70000AC10C1EBC10000EB8111D74800EB411127
:10C7100060319DF89C0000EB001011F830109DF87E
:10C72000AC00C0EBC00202EB8012CF4800EB42101D
:10C73000007981427EDA9DF8AC1001EB410000EBFC
:10C740000111C64800EB011030309DF89C1000EB41
:10C750000110801C0990C34890F8E6110120A0EB5D
:10C76000D1100999097860F3000109980170BD485A
:10C7700090F8E601C0F34010E8BB9DF8AC0000EB78
:10C78000400101EB001105E0FDE3FDE3FDE3FDE306
:10C79000FDE3FDE3B14800EB011030309DF89C1043
:10C7A00000EB01108078C0F3401020B39DF8AC007E
:10C7B00000EB400101EB0011A84800EB0110303004
:10C7C0009DF89C1000EB0110801C0990007820F06F
:10C7D0000200801C099908709DF8AC00C0EBC001F4
:10C7E00001EB8011A04800EB411060309DF89C10D7
:10C7F00001EB011100E00EE000EBC10018300990E0
:10C80000007820F00200801C099908709DF8AC1097
:10C810000220FDF79DFB00219DF8AC00C0EBC0029B
:10C8200002EB8012904800EB4210C17002229DF88A
:10C83000AC0000E020E0C0EBC00101EB80118A48B1
:10C8400000EB411160319DF89C0000EB001001F8F5
:10C850003020B6229DF8AC00C0EBC00101EB801186
:10C86000814800EB411060309DF89C1001EB0111F4
:10C8700000EBC10042717BE39DF8AC0000EB40018E
:10C8800001EB0011754800EB011030309DF89C1051
:10C8900000EB0110801C0990724890F8E60101211C
:10C8A000A1EBD01009990A7860F300020A709DF894
:10C8B000AC0000EB400101EB0011684800EB0110F7
:10C8C00030309DF89C1000EB0110801C09906548E9
:10C8D00090F8E60142090998007862F3410009994D
:10C8E00008709DF8AC0000EB400101EB00115B48C3
:10C8F00000EB011030309DF89C1000EB01108078A7
:10C90000C0F340029DF8AC00C0EBC00101EB801108
:10C91000554800EB411060309DF89C1001EB01116F
:10C9200000EBC100007EC0F3400082427ED09DF843
:10C93000AC10C1EBC10000EB81114B4800EB411082
:10C9400060309DF89C1001EB011100EBC100183024
:10C9500009909DF8AC0000EB400101EB00113F484D
:10C9600000EB011030309DF89C1000EB0110807836
:10C9700042080998007862F34100099908709DF80F
:10C98000AC1001EB410000EB0111344800EB011049
:10C9900030309DF89C1000EB01108078C0F340000F
:10C9A00090B1D9229DF8AC00C0EBC00101EB801121
:10C9B0002D4800EB411060309DF89C1001EB0111F7
:10C9C00000EBC100427138E001229DF8AC00C0EBE1
:10C9D000C00101EB8011244800EB411160319DF84A
:10C9E0009C0000EB001001EBC0004273D9229DF8BF
:10C9F000AC00C0EBC00101EB80111B4800EB411102
:10CA000060319DF89C0000EB001001EBC00042710A
:10CA100001229DF8AC00C0EBC00101EB801112486F
:10CA200000EB411060309DF89C1000E00AE001EB43
:10CA3000011100EBC10080F83E209DF8AC100220EF
:10CA4000FDF786FA9DF8AC1001EB410000EB0111F7
:10CA5000024800EB0111303108E000003C300020BA
:10CA600024660020BC220020FC3400209DF89C009D
:10CA700001EB0010807800F001029DF8AC00C0EBE3
:10CA8000C00101EB8011FE4800EB411060309DF8C1
:10CA90009C1001EB011100EBC100007E00F00100D1
:10CAA000824276D09DF8AC10C1EBC10000EB811141
:10CAB000F34800EB411060309DF89C1001EB011130
:10CAC00000EBC100183009909DF8AC1001EB41005B
:10CAD00000EB0111EB4800EB011030309DF89C1089
:10CAE00000EB0110807809990A7860F300020A705F
:10CAF0009DF8AC1001EB410000EB0111E14800EBA7
:10CB0000011030309DF89C1000EB0110807800F08F
:10CB10000100E8BB9DF8AC1001EB410000EB0111F6
:10CB2000D84800EB011030309DF89C1000EB01104C
:10CB30008078C0F3401068B39DF8AC10C1EBC10021
:10CB400000EB8111CE4800EB411060309DF89C1045
:10CB500001EB011100EBC10090F83E00D0B99DF847
:10CB6000AC10C1EBC10000EB8111C54800EB4110D6
:10CB700060309DF89C1001EB011100EBC100407B7F
:10CB800040B99DF8AC1001EB410000EB011102E04F
:10CB900058E080E142E0BB4800EB011030309DF8E6
:10CBA0009C1000EB01108078C0F34000B0BB012264
:10CBB0009DF8AC00C0EBC00101EB8011B04800EB68
:10CBC000411160319DF89C0000EB001001EBC000AA
:10CBD0004273D9229DF8AC00C0EBC00101EB80117B
:10CBE000A74800EB411160319DF89C0000EB00105C
:10CBF00001EBC000427101229DF8AC00C0EBC00106
:10CC000001EB80119E4800EB411060309DF89C10B4
:10CC100001EB011100EBC10080F83E2000229DF8DD
:10CC2000AC00C0EBC00101EB8011954800EB411056
:10CC300060309DF89C1001EB011100EBC10080F801
:10CC40003D2018E19DF8AC10C1EBC10000EB811153
:10CC50008B4800EB411060309DF89C1001EB0111F6
:10CC600000EBC10090F83E0098B901229DF8AC009D
:10CC7000C0EBC00101EB8011814800EB4110603036
:10CC80009DF89C1001EB011100EBC10080F83D20E4
:10CC900027E000229DF8AC00C0EBC00101EB801141
:10CCA000774800EB411160319DF89C0000EB0010CB
:10CCB00001EBC00080F83D209DF8AC1001EB410075
:10CCC00000EB01116F4800EB011130319DF89C0021
:10CCD00001EB0010801C0990007820F001020998F7
:10CCE0000270694890F8C80780B19DF8AC1001EB5C
:10CCF000410000EB0111634800EB011030309DF85A
:10CD00009C1000EB0110807A02286FD15F48407FB1
:10CD100001286BD15D48C06D5C49C98B884265D2E2
:10CD20009DF8AC10C1EBC10000EB8111544800EB41
:10CD3000411060309DF89C1001EB011100EBC10027
:10CD400090F83D00012851D19DF8AC10C1EBC10015
:10CD500000EB81114A4800EB411060309DF89C10B7
:10CD600001EB011100EBC10090F87700F0BB9DF8DA
:10CD7000AC1001EB410000EB0111424800EB011146
:10CD800030319DF89C0001EB001001789DF8AC005B
:10CD9000C0EBC00202EB8012394800EB4210417038
:10CDA000C3229DF8AC00C0EBC00101EB80113448F8
:10CDB00000EB411160319DF89C0000EB001001EB8D
:10CDC000C000427100229DF8AC0000EB400101EB75
:10CDD00000112C4800EB011130319DF89C0001EB53
:10CDE000001042609DF8AC10022000E043E0FDF727
:10CDF000AFF80021369119E000229DF8AC00C0EB9D
:10CE0000C00101EB80111E4800EB411160319DF81B
:10CE10009C0000EB001001EBC0013F31BDF8D800D1
:10CE20000A54BDF8D800401C81B23691BDF8D80034
:10CE30001428E1DB0020369019E000229DF8AC00B8
:10CE4000C0EBC00101EB80110D4800EB41116031D6
:10CE50009DF89C0000EB001001EBC0015B31BDF8B8
:10CE6000D8000A54BDF8D800401C81B23691BDF8F4
:10CE7000D8000A28E1DB9DF8AC10022009E0F5E3B8
:10CE8000FC3400203C300020BC220020BC120020DA
:10CE9000B8E3FDF75DF89DF8AC1001EB410000EB45
:10CEA0000111FE4800EB011030309DF89C1000EBA2
:10CEB00001108078C0F3400088B1D9229DF8AC0001
:10CEC000C0EBC00101EB8011F54800EB4110603070
:10CED0009DF89C1001EB011100EBC10042719DF81F
:10CEE000AC10C1EBC10000EB8111ED4800EB41102B
:10CEF00060309DF89C1001EB011100EBC1008078BF
:10CF0000B22835D19DF8AC1001EB410000EB0111C6
:10CF1000E24800EB011030309DF89C1000EB01104E
:10CF20008078C0F3400018BB9DF8AC0000EB4001D6
:10CF300001EB0011D94800EB011030309DF89C1036
:10CF400000EB01108078C0F3401088B9E5229DF80D
:10CF5000AC00C0EBC00101EB8011D14800EB4110E7
:10CF600060309DF89C1001EB011100EBC100427193
:10CF70009DF8AC0000EB400101EB0011C74800EB4D
:10CF80000110303005E0F9E384E3F8E3F8E313E15E
:10CF90006DE39DF89C1000EB011080780121B1EB4E
:10CFA000D01F4FD19DF8AC0000EB400101EB001108
:10CFB000BA4800EB011030309DF89C1000EB0110D6
:10CFC000807800F00100E8BB9DF8AC00C0EBC00128
:10CFD00001EB8011B24800EB411060309DF89C10CD
:10CFE00001EB011100EBC10090F83E0050BB9DF831
:10CFF000AC0000EB400101EB0011A84800EB011070
:10D0000030309DF89C1000EB01108078C0F3C00018
:10D01000C0B99DF8AC0000EB400101EB00119F4846
:10D0200000EB011030309DF89C1000EB0110407AAD
:10D0300000F0010030B19DF8AC00C0EBC00101EB85
:10D04000801100E049E0964800EB411060309DF807
:10D050009C1001EB011100EBC10090F8860000F07C
:10D060000100D0BB9DF8AC00C0EBC00101EB80110A
:10D070008B4800EB411060309DF89C1001EB0111D2
:10D0800000EBC10090F8780038B3002036902AE019
:10D090009DF8AC00C0EBC00101EB8011804800EBB3
:10D0A000411160319DF89C0000EB001001EBC000C5
:10D0B00000F17901BDF8D8000A5C9DF8AC0000EBE6
:10D0C000400101EB0011754800EB01100E30BDF876
:10D0D000D810405C824201D009E06CE0BDF8D80075
:10D0E000401C81B23691BDF8D8000628D0DB00BFC5
:10D0F000BDF8D80006285ED1369029E09DF8AC0036
:10D10000C0EBC00101EB8011654800EB41116031BB
:10D110009DF89C0000EB001001EBC00000F17901CC
:10D12000BDF8D8000A5C9DF8AC0000EB400101EBB3
:10D1300000115A4800EB01100E30BDF8D810405CC9
:10D14000824200D008E0BDF8D800401C81B2369180
:10D15000BDF8D8000A28D1DB00BFBDF8D8000A28E6
:10D1600029D09DF8AC00C0EBC00101EB80114C4808
:10D1700000EB411060309DF89C1001EB011100EBB9
:10D18000C10086300990007820F00100401C099908
:10D19000087012229DF8AC00C0EBC00101EB8011B9
:10D1A0003F4800EB411060309DF89C1001EB0111ED
:10D1B00000EBC1004271FCE39DF8AC0000EB4001C4
:10D1C00001EB0011354800EB0110007BD0BBBDF82E
:10D1D000A000082800D0EEE70020369028E09DF857
:10D1E000AC0000EB4001C1EBC0102E4901EBC001C7
:10D1F000BDF8D800C01C085C00F00F00092800DD55
:10D200001AE09DF8AC0000EB4001C1EBC0102549CD
:10D2100001EBC001BDF8D800C01C085C00F0F000B4
:10D22000902800DD08E0BDF8D800401C81B236919E
:10D23000BDF8D8000628D2DB00BFBDF8D80006280C
:10D2400001DAB8E770E09DF8AC0000EB4001C1EBFB
:10D25000C010144901EBC000C07801049DF8AC0077
:10D2600000EB4002C2EBC0100E4A02EBC000007996
:10D2700041EA00219DF8AC0000EB4002C2EBC01077
:10D28000084A02EBC000407901439DF8AC00C0EBB6
:10D29000C00202EB8012024806E000003C30002091
:10D2A000FC3400202466002000EB421260329DF81E
:10D2B0009C0000EB001002EBC000C0F81A109DF8B3
:10D2C000AC0000EB4001C1EBC010FE4901EBC00017
:10D2D000807901049DF8AC0000EB4002C2EBC01065
:10D2E000F84A02EBC000C07941EA00219DF8AC0089
:10D2F00000EB4002C2EBC010F24A02EBC000007A21
:10D3000001439DF8AC00C0EBC00202EB8012EE4876
:10D3100000EB421060309DF89C2002EB021200EB03
:10D32000C200C0F81E10BAE0BDF8A0000A2800D064
:10D3300041E70020369028E09DF8AC1001EB410059
:10D34000C0EBC110DF4901EBC001BDF8D800C01C23
:10D35000085C00F00F00092800DD1AE09DF8AC1011
:10D3600001EB4100C0EBC110D64901EBC001BDF893
:10D37000D800C01C085C00F0F000902800DD08E038
:10D38000BDF8D800401C81B23691BDF8D8000828FD
:10D39000D2DB00BFBDF8D800082800DA0BE79DF803
:10D3A000AC1001EB4100C0EBC110C64901EBC0005D
:10D3B000C07801069DF8AC0000EB4002C2EBC01043
:10D3C000C04A02EBC000007941EA00419DF8AC0080
:10D3D00000EB4002C2EBC010BA4A02EBC000407939
:10D3E00041EA00219DF8AC0000EB4002C2EBC01006
:10D3F000B44A02EBC000807901439DF8AC00C0EB59
:10D40000C00202EB8012B04800EB421260329DF87D
:10D410009C0000EB001002EBC000C0F81A109DF851
:10D42000AC1001EB4100C0EBC110A64901EBC000FC
:10D43000C07901069DF8AC0000EB4002C2EBC010C1
:10D44000A04A02EBC000007A41EA00419DF8AC001E
:10D4500000EB4002C2EBC0109A4A02EBC000407AD7
:10D4600041EA00219DF8AC0000EB4002C2EBC01085
:10D47000944A02EBC000807A01439DF8AC00C0EBF7
:10D48000C00202EB8012904800EB421060309DF821
:10D490009C2002EB021200EBC200C0F81E109DF8A7
:10D4A000AC10C1EBC10000EB8111874800EB4111CA
:10D4B00060319DF89C0000EB001011F830109DF8D1
:10D4C000AC00C0EBC00202EB80127F4800EB4210C0
:10D4D000007981422EDA00219DF8AC00C0EBC00239
:10D4E00002EB8012784800EB4210C17004229DF8D4
:10D4F000AC00C0EBC00101EB8011734800EB41119F
:10D5000060319DF89C0000EB001001F83020C5222E
:10D510009DF8AC00C0EBC00101EB80116A4800EB44
:10D52000411060309DF89C1001EB011100EBC1002F
:10D53000427166E09DF8AC1001EB410000EB011177
:10D54000624800EB011030309DF89C1000EB011098
:10D550008078C0F3400090B1D5229DF8AC00C0EBBC
:10D56000C00101EB8011584800EB411060309DF87C
:10D570009C1001EB011100EBC100427141E09DF8EC
:10D58000AC10C1EBC10000EB81114F4800EB411022
:10D5900060309DF89C1001EB011100EBC100807B15
:10D5A00001282ED100229DF8AC00C0EBC00101EB98
:10D5B0008011454800EB411160319DF89C0000EB63
:10D5C000001001EBC0008273B6229DF8AC00C0EBE6
:10D5D000C00101EB80113C4800EB411160319DF826
:10D5E0009C0000EB001001EBC000427100219DF88F
:10D5F000AC00C0EBC00202EB8012334800EB4210DB
:10D60000C170D8E5D5229DF8AC00C0EBC00101EB9C
:10D6100080112D4800EB411160319DF89C0000EB1A
:10D62000001001EBC000427101219DF8AC00C0EB7D
:10D63000C00202EB8012244800EB4210C1709DF83A
:10D64000AC1001EB410000EB0111204800EB01118F
:10D6500030319DF89C0001EB0010801C099000788F
:10D6600020F02000203009990870A4E51FE2D5229F
:10D670009DF8AC00C0EBC00101EB8011124800EB3B
:10D68000411060309DF89C1001EB011100EBC100CE
:10D69000427190E59DF8AC10C1EBC10000EB811127
:10D6A000094800EB41106030BDF8D01001EB0111CA
:10D6B00000EBC1008079012842D100229DF8AC0026
:10D6C00006E0000024660020FC3400203C300020EE
:10D6D000C0EBC00101EB8011FE4800EB411160314D
:10D6E000BDF8D00000EB001001EBC0008271D92220
:10D6F0009DF8AC00C0EBC00101EB8011F54800EBD8
:10D70000411160319DF89C0000EB001001EBC0005E
:10D7100042719DF8AC1001EB410000EB0111EE48A5
:10D7200000EB011030309DF89C1000EB0110801CC4
:10D730000990007820F00400001D099908701CE091
:10D74000C3229DF8AC00C0EBC00101EB8011E148A1
:10D7500000EB411160319DF89C0000EB001001EBE3
:10D76000C000427100219DF8AC00C0EBC00202EB8A
:10D770008012D84800EB4210C1701CE5D2E16CE089
:10D78000FFE79DF8AC10C1EBC10000EB8111D1485F
:10D7900000EB41106030BDF8D01001EB011100EB3F
:10D7A000C100807901283AD100229DF8AC00C0EB7D
:10D7B000C00101EB8011C74800EB41116031BDF899
:10D7C000D00000EB001001EBC0008271D9229DF85F
:10D7D000AC00C0EBC00101EB8011BE4800EB411171
:10D7E00060319DF89C0000EB001001EBC00042711D
:10D7F0009DF8AC1001EB410000EB0111B64800EBC5
:10D80000011130319DF89C0001EB0010801C099043
:10D81000007820F00400001D099908701CE0C32264
:10D820009DF8AC00C0EBC00101EB8011A94800EBF2
:10D83000411160319DF89C0000EB001001EBC0002D
:10D84000427100219DF8AC00C0EBC00202EB8012D7
:10D85000A04800EB4210C170ADE49DF8AC1001EBA4
:10D86000410000EB01119C4800EB0110007B38BB2C
:10D870009DF8AC1001EB4100C0EBC110974901EBE2
:10D88000C00001799DF8AC0000EB4002C2EBC01073
:10D89000924A02EBC000C07841EA00229DF8AC0039
:10D8A000C0EBC00101EB80118A4800EB41106030F1
:10D8B0009DF89C1001EB011100EBC100426332E0C6
:10D8C0009DF8AC1001EB4100C0EBC110834901EBA6
:10D8D000C000C07801049DF8AC0000EB4002C2EB30
:10D8E000C0107E4A02EBC000007941EA00219DF899
:10D8F000AC0000EB4002C2EBC010784A02EBC00063
:10D90000407901439DF8AC00C0EBC00202EB8012ED
:10D91000704800EB421060309DF89C2002EB021230
:10D9200000EBC20041639DF8AC10C1EBC10000EBFD
:10D930008111684800EB411160319DF89C0000EBBB
:10D94000001011F830109DF8AC00C0EBC00202EBE3
:10D950008012604800EB42100079814230DA0021E9
:10D960009DF8AC00C0EBC00202EB8012594800EBFE
:10D970004210C17003229DF8AC00C0EBC00101EB66
:10D980008011544800EB411160319DF89C0000EB80
:10D99000001001F83020D9229DF8AC00C0EBC00186
:10D9A00001EB80114B4800EB411060309DF89C105A
:10D9B00000E0FDE301EB011100EBC100427175E0F5
:10D9C0009DF8AC10C1EBC10000EB8111414800EBA8
:10D9D00041106030BDF8D01001EB011100EBC10027
:10D9E0008079012845D100229DF8AC00C0EBC00130
:10D9F00001EB8011374800EB41116031BDF8D000D8
:10DA000000EB001001EBC0008271D9229DF8AC0040
:10DA1000C0EBC00101EB80112E4800EB41116031D9
:10DA20009DF89C0000EB001001EBC00042719DF8D6
:10DA3000AC1001EB410000EB0111274800EB011194
:10DA400030319DF89C0001EB0010801C099000789B
:10DA500020F00400001D0999087001229DF8AC0017
:10DA6000C0EBC00101EB80111A4800EB4110C270FD
:10DA70001CE0C5229DF8AC00C0EBC00101EB801199
:10DA8000144800EB411160319DF89C0000EB001040
:10DA900001EBC000427100219DF8AC00C0EBC00258
:10DAA00002EB80120B4800EB4210C17080E30021B2
:10DAB0009DF8AC00C0EBC00202EB8012054800EB01
:10DAC0004210C1709DF8AC1001EB410000EB011158
:10DAD000014805E0FC3400203C3000202466002092
:10DAE00000EB011130319DF89C0001EB0010801C0F
:10DAF0000990007820F00400001D09990870D522D3
:10DB00009DF8AC00C0EBC00101EB8011FE4800EBBA
:10DB1000411060309DF89C1001EB011100EBC10039
:10DB2000427145E39DF8AC1001EB410000EB01119F
:10DB3000F64800EB0110007BD0BBBDF8A0000C281C
:10DB400000D035E30020369028E09DF8AC1001EBC2
:10DB50004100C0EBC110EE4901EBC001BDF8D80097
:10DB6000C01C085C00F00F00092800DD1AE09DF8D9
:10DB7000AC1001EB4100C0EBC110E54901EBC00165
:10DB8000BDF8D800C01C085C00F0F000902800DD53
:10DB900008E0BDF8D800401C81B23691BDF8D8002D
:10DBA0000A28D2DB00BFBDF8D8000A2801DAFFE25C
:10DBB0007CE000202C902D90002136911EE0DDE9C4
:10DBC0002C10000240EA11620902CDE92C129DF8E6
:10DBD000AC1001EB4100C0EBC110CD4901EBC0011D
:10DBE000BDF8D800C01C085CDDE92C341843CDE931
:10DBF0002C04BDF8D800401C80B23690BDF8D80087
:10DC00000528DCDB9DF8AC00DDE92C21C0EBC0036E
:10DC100003EB8013BC4800EB431360339DF89C007A
:10DC200000EB001003EBC00040F8222F41600022FF
:10DC30002C922D92002136911EE0DDE92C1000027D
:10DC400040EA11620902CDE92C129DF8AC1001EBFB
:10DC50004100C0EBC110AE4901EBC001BDF8D800D6
:10DC60000830085CDDE92C341843CDE92C04BDF8FC
:10DC7000D800401C80B23690BDF8D8000528DCDB07
:10DC80009DF8AC00DDE92C12C0EBC00303EB801360
:10DC90009D4800EB431060309DF89C3003EB03136C
:10DCA00000EBC30022308160C260B6E0BDF8A00086
:10DCB0000E2800D07CE20020369028E09DF8AC10C1
:10DCC00001EB4100C0EBC110914901EBC001BDF86F
:10DCD000D800C01C085C00F00F00092800DD1AE025
:10DCE0009DF8AC1001EB4100C0EBC110884901EB7D
:10DCF000C001BDF8D800C01C085C00F0F0009028FE
:10DD000000DD08E0BDF8D800401C81B23691BDF8B6
:10DD1000D8000C28D2DB00BFBDF8D8000C2800DAF0
:10DD200046E200202C902D90002136911EE0DDE986
:10DD30002C10000240EA11620902CDE92C129DF874
:10DD4000AC1001EB4100C0EBC110714901EBC00107
:10DD5000BDF8D800C01C085CDDE92C341843CDE9BF
:10DD60002C04BDF8D800401C80B23690BDF8D80015
:10DD70000628DCDB9DF8AC00DDE92C12C0EBC0030B
:10DD800003EB8013604800EB431360339DF89C0065
:10DD900000EB001003EBC00040F8221F426000229D
:10DDA0002C922D92002136911EE0DDE92C1000020C
:10DDB00040EA11620902CDE92C129DF8AC1001EB8A
:10DDC0004100C0EBC110524901EBC001BDF8D800C1
:10DDD0000930085CDDE92C341843CDE92C04BDF88A
:10DDE000D800401C80B23690BDF8D8000628DCDB95
:10DDF0009DF8AC00DDE92C21C0EBC00303EB8013E0
:10DE0000414800EB431060309DF89C3003EB031356
:10DE100000EBC30022308260C1609DF8AC10C1EB02
:10DE2000C10000EB8111384800EB411160319DF8D1
:10DE30009C0000EB001011F830109DF8AC00C0EB16
:10DE4000C00202EB8012304800EB421000798142A0
:10DE50007ED1304890F8C80780B19DF8AC1001EB36
:10DE6000410000EB0111294800EB011030309DF812
:10DE70009C1000EB0110807A02286AD1002126480C
:10DE8000C0F83D109DF8AC10C1EBC10000EB811152
:10DE90001D4800EB411060309DF89C1001EB011112
:10DEA00000EBC10022301022014609901A482D30A3
:10DEB000FAF7CBF99DF8AC10C1EBC10000EB811172
:10DEC000114800EB411160319DF89C0000EB0010FF
:10DED00001EBC0011048401C51F81A2F026249683A
:10DEE00041629DF8AC1001EB410000EB01110748C5
:10DEF00000EB011130319DF89C0001EB001000781F
:10DF0000054981F8200009E0FC3400203C30002065
:10DF100024660020BC220020BC12002001F1210058
:10DF200001F59C510A6F0262B1F8741081849DF86A
:10DF3000AC10C1EBC10000EB8111FE4800EB4111B8
:10DF400060319DF89C0000EB001001EBC00001E087
:10DF50003EE144E0416BF848C0F829109DF8AC1050
:10DF600001EB410000EB0111F44800EB01113031ED
:10DF70009DF89C0001EB00104168EF48C0F8471085
:10DF8000C06D81B202200991FBF7A2F800210620A2
:10DF9000FBF7DEFFE848C06DE749C98B884204D231
:10DFA000E548C06D401CE449C86500210520FBF729
:10DFB000CFFF9DF8AC1001EB410000EB0111DF48F1
:10DFC00000EB011030309DF89C1000EB0110801C1C
:10DFD0000990007820F008020998027015E09DF879
:10DFE000AC0000EB400101EB0011D44800EB011044
:10DFF00030309DF89C1000EB0110801C09900078D7
:10E0000020F008000830099908709DF8AC0000EB7A
:10E01000400101EB0011C94800EB011030309DF8C0
:10E020009C1000EB0110801C0990007820F0200269
:10E03000099802709DF8AC100220FBF789FF9DF84B
:10E04000AC009DF89C1001EB0010C217CDE92C022A
:10E0500000222C9800EB8001C1EB8011B64864309F
:10E060000844C0F81D209DF8AC00C0EBC00101EBD6
:10E070008011B04800EB411060309DF89C1001EB1E
:10E08000011100EBC100223009902C9800EB8001B7
:10E09000C1EB8011A848643001440D311022089171
:10E0A000DDE90801FAF7D1F89DF8AC00C0EBC0013A
:10E0B00001EB80119F4800EB411160319DF89C00FD
:10E0C00000EB001001EBC0012C9800EB8002C2EBCA
:10E0D000801299486430104451F81A2F40F8012FEB
:10E0E000496841609DF8AC0000EB400101EB001174
:10E0F000924800EB011130319DF89C0001EB0010BB
:10E1000001782C9800EB8002C2EB80128A486430C0
:10E1100081542C9800EB8001C1EB8011864864305B
:10E1200001448748026F41F8212FB0F874008880BD
:10E130009DF8AC00C0EBC00101EB80117D4800EB05
:10E14000411160319DF89C0000EB001001EBC00014
:10E15000416B2C9800EB8002C2EB80127648643051
:10E160001044C0F809109DF8AC0000EB400101EB31
:10E170000011724800EB011130319DF89C0001EB59
:10E18000001041682C9800EB8002C2EB80126A48B4
:10E1900064301044C0F827102C9881B208200991EF
:10E1A000FBF7D6FE00229DF8AC00C0EBC00100E0FA
:10E1B00019E201EB80115F4800EB411060309DF8DF
:10E1C0009C1001EB011100EBC10080F83E2050E0F3
:10E1D0009DF8AC0000EB400101EB0011574800EB4B
:10E1E000011030309DF89C1000EB0110801C09904C
:10E1F000007820F00400001D099908709DF8AC001B
:10E2000000EB400101EB00114C4800EB01103030F5
:10E210009DF89C1000EB0110801C0990007820F004
:10E22000800080300999087001229DF8AC00C0EB95
:10E23000C00101EB80113F4800EB4110C2709DF816
:10E24000AC00C0EBC00101EB80113A4800EB41107B
:10E2500002799DF8AC00C0EBC00101EB801135489C
:10E2600000EB411060309DF89C1001EB011100F8AB
:10E270003120D5229DF8AC00C0EBC00101EB80112C
:10E280002C4800EB411060309DF89C1001EB01110F
:10E2900000EBC10042713DE2D5229DF8AC00C0EB1D
:10E2A000C00101EB8011234800EB411060309DF864
:10E2B0009C1001EB011100EBC10042712AE2D52252
:10E2C0009DF8AC00C0EBC00101EB8011194800EBD8
:10E2D000411060309DF89C1001EB011100EBC10072
:10E2E000427117E20121174880F8EC169DF8AC0046
:10E2F000C0EBC00101EB80110E4800EB4111603111
:10E300009DF89C0000EB001011F830109DF8AC0057
:10E31000C0EBC00202EB8012064800EB421000790D
:10E32000814239DA00219DF8AC00C0EBC00202EB5B
:10E33000801209E0FC340020BC1200203C30002098
:10E340003C260020BC220020FA4800EB4210C1709D
:10E3500001229DF8AC00C0EBC00101EB8011F54833
:10E3600000EB411160319DF89C0000EB001001F8BA
:10E37000302011229DF8AC00C0EBC00101EB8011F0
:10E38000EC4800EB411060309DF89C1001EB01114E
:10E3900000EBC100427141E09DF8AC00C0EBC00150
:10E3A00001EB8011E34800EB411060309DF89C10B8
:10E3B00001EB011100EBC1008078B2282ED10021C1
:10E3C0009DF8AC00C0EBC00202EB8012D94800EB14
:10E3D0004210C170B2229DF8AC00C0EBC00101EB4D
:10E3E0008011D44800EB411160319DF89C0000EB96
:10E3F000001001EBC000427100229DF8AC00C0EBA0
:10E40000C00101EB8011CB4800EB411060309DF85A
:10E410009C1001EB011100EBC10082707AE1002138
:10E42000C54880F8EC16D5229DF8AC00C0EBC001C1
:10E4300001EB8011BF4800EB411060309DF89C104B
:10E4400001EB011100EBC100427163E101229DF873
:10E45000AC00C0EBC00101EB8011B64800EB4111EC
:10E4600060319DF89C0000EB001001EBC00080F8CB
:10E4700078200021369126E09DF8AC1001EB410098
:10E48000C0EBC110AD4901EBC001BDF8D800C01C04
:10E490000A5C9DF8AC00C0EBC00101EB8011A548FF
:10E4A00000EB411160319DF89C0000EB001001EB86
:10E4B000C00000F17901BDF8D8000A54BDF8D800B9
:10E4C000401C81B23691BDF8D8000A28D4DB21E186
:10E4D0009DF8AC1001EB4100C0EBC111974800EB77
:10E4E000C100C07801049DF8AC0000EB4002C2EB13
:10E4F000C010924A02EBC000007941EA00209DF86A
:10E50000AC1001EB4102C2EBC1118C4A02EBC1011C
:10E5100049790843B0F5E13F65D19DF8AC1001EBB6
:10E52000410000EB0111864800EB011030309DF8EE
:10E530009C1000EB0110801C0990007820F0040270
:10E540000998027000229DF8AC00C0EBC00101EBFD
:10E550008011784800EB411060309DF89C1001EB71
:10E56000011100EBC100A0F8842013229DF8AC003B
:10E57000C0EBC00101EB80116E4800EB4110603030
:10E580009DF89C1001EB011100EBC10042719DF858
:10E59000AC1001EB410000EB0111694800EB0110E8
:10E5A000407903464FF480524FF4E13109909DF8D1
:10E5B000AC000FF095F89DF8AC10C1EBC10000EB7A
:10E5C00081115C4800EB411160319DF89C0000EB2B
:10E5D000001001EBC00086300990007820F00800A0
:10E5E00008300999087095E09DF8AC1001EB4100E6
:10E5F000C0EBC110514901EBC00001799DF8AC009E
:10E6000000EB4002C2EBC0104C4A02EBC000C078E5
:10E6100041EA00229DF8AC00C0EBC00101EB801183
:10E62000444800EB411160319DF89C0000EB001064
:10E6300001EBC000A0F884209DF8AC10C1EBC10034
:10E6400000EB81113B4800EB411160319DF89C00CB
:10E6500000EB001001EBC000B0F884109DF8AC0096
:10E6600000EB400202EB0012354800EB0210408B39
:10E6700081424EDBE5229DF8AC00C0EBC00101EB0E
:10E6800080112C4800EB411160319DF89C0000EB9B
:10E69000001001EBC000427100229DF8AC00C0EBFD
:10E6A000C00101EB8011234800EB411160319DF85E
:10E6B0009C0000EB001001F830209DF8AC1001EB3D
:10E6C000410000EB01111E4800EB011130319DF8B3
:10E6D0009C0001EB0010801C0990007820F0800263
:10E6E000099802709DF8AC10C1EBC10000EB8111DC
:10E6F000104800EB411060309DF89C1001EB0111B7
:10E7000000EBC10086300990007820F001020998E2
:10E71000027000BF00BF07F0D1BC9DF8AC1001EB48
:10E720004100C0EBC110054911F83000042809D19F
:10E73000259013E0FC340020BC2200202466002039
:10E740003C3000209DF8AC1001EB4100C0EBC11043
:10E75000FE4911F83000152800D125909DF8AC1025
:10E7600001EB4100C0EBC110F84901EBC00041785A
:10E770009DF8AC0000EB4002C2EBC010F34A12F867
:10E78000300041EA002041F23001884202D1A62146
:10E7900025913DE09DF8AC1001EB4100C0EBC110AC
:10E7A000EA4901EBC00041789DF8AC0000EB400263
:10E7B000C2EBC010E54A12F8300041EA002041F2F5
:10E7C0003101884202D1A721259121E09DF8AC10AA
:10E7D00001EB4100C0EBC110DC4911F83000022808
:10E7E00016D19DF8AC1001EB4100C0EBC110D74928
:10E7F00001EBC00001799DF8AC0000EB4002C2EBD8
:10E80000C010D24A02EBC000C07841EA0021259135
:10E810009DF8AC10C1EBC10000EB8111CC4800EBBE
:10E820004110817827910021CA4A9DF8AC0002EB83
:10E8300000129DF89C001154C748007F012815D193
:10E840009DF8AC1001EB410000EB0111C34800EB57
:10E85000011030309DF89C1000EB0110801C0990D5
:10E86000007820F080008030099908709DF8AC1085
:10E8700001EB410000EB0111B84800EB0110303012
:10E880009DF89C1000EB0110801C0990007820F08E
:10E890004001403109980170BDF8941043F23002F4
:10E8A000881A91427ED009DC04297CD015297BD0BE
:10E8B000A6290DD0A72941F0E2852EE1B0F5C06F61
:10E8C00073D0A0F20160002870D00428F3D1FDE3DA
:10E8D00000219DF8AC00C0EBC00202EB80129C4806
:10E8E00000EB4210C1709DF8AC10C1EBC10000EB11
:10E8F0008111974800EB411060309DF89C1001EBAE
:10E90000011110F83100032823DC04229DF8AC002B
:10E91000C0EBC00101EB80118D4800EB411160316B
:10E920009DF89C0000EB001001F83020A8229DF813
:10E93000AC00C0EBC00101EB8011854800EB411039
:10E9400060309DF89C1001EB011100EBC100427199
:10E95000E1E09DF8AC10C1EBC10000EB81117C48F7
:10E9600000EB411060309DF89C1001EB011110F894
:10E970003100082829DC09229DF8AC00C0EBC00159
:10E9800001EB8011724800EB411160319DF89C0051
:10E9900000EB001001F83020A9229DF8AC00C0EB7C
:10E9A000C00104E076E1EAE1F9E3F9E3F9E301EB20
:10E9B0008011674800EB411060309DF89C1001EB1E
:10E9C000011100EBC1004271A5E09DF8AC10C1EB54
:10E9D000C10000EB81115E4800EB411060309DF8F2
:10E9E0009C1001EB011110F831000D2823DC0E22E0
:10E9F0009DF8AC00C0EBC00101EB8011544800EB66
:10EA0000411160319DF89C0000EB001001F83020AE
:10EA1000A2229DF8AC00C0EBC00101EB80114C4874
:10EA200000EB411060309DF89C1001EB011100EBF0
:10EA3000C10042716FE09DF8AC00C0EBC00101EB7A
:10EA40008011434800EB411060309DF89C1001EBB1
:10EA5000011100EBC1004079A52815D19DF8AC103B
:10EA600001EB410000EB01113C4800EB011030309C
:10EA70009DF89C1000EB0110801C0990007820F09C
:10EA80000400001D099908709DF8AC10C1EBC1008D
:10EA900000EB81112E4800EB411060309DF89C1076
:10EAA00001EB011100EBC1008078A12833D09DF863
:10EAB000AC00C0EBC00101EB8011254800EB411117
:10EAC00060319DF89C0000EB001001EBC0008278E3
:10EAD0009DF8AC00C0EBC00101EB80111C4800EBBD
:10EAE000411160319DF89C0000EB001001EBC0006B
:10EAF0004271A1229DF8AC00C0EBC00101EB801176
:10EB0000134800EB411060309DF89C1001EB01119F
:10EB100000EBC100827001F0B2BC00219DF8AC0096
:10EB2000C0EBC00202EB8012094800EB4210C1703A
:10EB30009DF8AC10C1EBC10000EB8111044800EB63
:10EB4000411060309DF89C100AE00000246600200F
:10EB5000FC340020702E0020BC1200203C3000202D
:10EB600001EB011110F8310005281CDC00219DF893
:10EB7000AC00C0EBC00202EB8012FE4800EB42107A
:10EB8000C17006229DF8AC00C0EBC00101EB801102
:10EB9000F84800EB411060309DF89C1001EB01112A
:10EBA00000F8312022E09DF8AC10C1EBC10000EB71
:10EBB0008111F04800EB411060309DF89C1001EB92
:10EBC000011110F83100092810DC0A229DF8AC0070
:10EBD000C0EBC00101EB8011E64800EB4110603052
:10EBE0009DF89C1001EB011100F831209DF8AC104C
:10EBF000C1EBC10000EB8111DE4800EB4110603039
:10EC00009DF89C1001EB011100EBC1004079A42894
:10EC10002DD19DF8AC1001EB410000EB0111D6485D
:10EC200000EB011030309DF89C1000EB0110801CAF
:10EC30000990007820F02000203009990870002207
:10EC40009DF8AC00C0EBC00101EB8011C94800EB9E
:10EC5000411060309DF89C1001EB011100EBC100E8
:10EC600080F83D209DF8AC100220FBF771F9A1223D
:10EC70009DF8AC00C0EBC00101EB8011BD4800EB7A
:10EC8000411060309DF89C1001EB011100EBC100B8
:10EC9000427140E70020369015E09DF8AC1001EB82
:10ECA0004100C0EBC110B54901EBC001BDF8D8006F
:10ECB000C01C095C16AABDF8D8001154BDF8D800D4
:10ECC000401C81B23691BDF8D8000628E5DB06214C
:10ECD00016A81EF0DBFC0021CDE92E01DDE92E2176
:10ECE000100A40EA01602E9BC01841EB21214FF42D
:10ECF00080724FF00003CDE90801F9F763FA9DF83F
:10ED0000AC00C0EBC00101EB80119A4800EB411050
:10ED100060309DF89C1001EB011100EBC100027105
:10ED200000229DF8AC00C0EBC00101EB80119148BE
:10ED300000EB4110C27001229DF8AC00C0EBC00195
:10ED400001EB80118B4800EB411060309DF89C1066
:10ED500001EB011100F83120A7229DF8AC00C0EBB7
:10ED6000C00101EB8011834800EB411060309DF839
:10ED70009C1001EB011100EBC1004271CBE69DF844
:10ED8000AC10C1EBC10000EB81117A4800EB4110DF
:10ED900060309DF89C1001EB011110F8310006283D
:10EDA0002DDC00219DF8AC00C0EBC00202EB80120C
:10EDB000704800EB4210C17007229DF8AC00C0EB18
:10EDC000C00101EB80116B4800EB411160319DF8EF
:10EDD0009C0000EB001001F83020A7229DF8AC0049
:10EDE000C0EBC00101EB8011624800EB41106030C4
:10EDF0009DF89C1001EB011100EBC10042719DF8E0
:10EE0000AC10C1EBC10000EB81115A4800EB41107E
:10EE100060309DF89C1001EB011110F831000128C1
:10EE20002EDC00219DF8AC00C0EBC00202EB80128A
:10EE3000504800EB4210C17002229DF8AC00C0EBBC
:10EE4000C00101EB80114B4800EB411160319DF88E
:10EE50009C0000EB001001F83020A3229DF8AC00CC
:10EE6000C0EBC00101EB8011424800EB4110603063
:10EE70009DF89C1001EB011100EBC100427116E2FC
:10EE80009DF8AC10C1EBC10000EB8111394800EBDB
:10EE9000411060309DF89C1001EB011110F8310019
:10EEA00007282EDC00219DF8AC00C0EBC00202EB6D
:10EEB0008012304800EB4210C17008229DF8AC006F
:10EEC000C0EBC00101EB80112A4800EB4111603119
:10EED0009DF89C0000EB001001F83020A3229DF863
:10EEE000AC00C0EBC00101EB8011224800EB4110E7
:10EEF00060309DF89C1001EB011100EBC1004271E4
:10EF0000D5E19DF8AC10C1EBC10000EB81111948AF
:10EF100000EB411060309DF89C1001EB011110F8DE
:10EF200031000B2835DC00219DF8AC00C0EBC0029D
:10EF300002EB80120F4800EB4210C1700C229DF8CA
:10EF4000AC00C0EBC00101EB80110A4800EB41119D
:10EF500060319DF89C0000EB001001F83020A122E8
:10EF60009DF8AC00C0EBC00101EB8011014800EB43
:10EF7000411005E0FC3400203C30002024660020D5
:10EF800060309DF89C1001EB011100EBC100427153
:10EF90008DE19DF8AC10C1EBC10000EB8111FC4884
:10EFA00000EB411060309DF89C1001EB011110F84E
:10EFB00031000C282EDC00219DF8AC00C0EBC00213
:10EFC00002EB8012F24800EB4210C1700D229DF856
:10EFD000AC00C0EBC00101EB8011ED4800EB41112A
:10EFE00060319DF89C0000EB001001F83020A32256
:10EFF0009DF8AC00C0EBC00101EB8011E44800EBD0
:10F00000411060309DF89C1001EB011100EBC10034
:10F0100042714CE19DF8AC10C1EBC10000EB8111D5
:10F02000DB4800EB411060309DF89C1001EB0111B2
:10F0300010F831000E287DDC0F229DF8AC00C0EBEB
:10F04000C00101EB8011D24800EB411160319DF805
:10F050009C0000EB001001F83020A1229DF8AC00CC
:10F06000C0EBC00101EB8011C94800EB41116031D8
:10F070009DF89C0000EB001001EBC00042719DF870
:10F08000AC00C0EBC00101EB8011C14800EB4111A5
:10F0900060319DF89C0000EB001001EBC000827015
:10F0A0009DF8AC1001EB410000EB0111B94800EBF9
:10F0B000011130319DF89C0001EB0010801C09907B
:10F0C000007820F080008030099900E0FDE30870AE
:10F0D0009DF8AC0000EB400101EB0011AD4800EBE6
:10F0E000011030309DF89C1000EB0110801C09903D
:10F0F000007820F00400001D099908709DF8AC000C
:10F1000000EB400101EB0011A24800EB0110303090
:10F110009DF89C1000EB01108078C0F34010E8B31C
:10F120009DF8AC0000EB400101EB0011994800EBA9
:10F13000011000E03EE030309DF89C1000EB011023
:10F14000801C0990007820F02002099802709DF838
:10F15000AC0000EB400101EB00118E4800EB011008
:10F1600030309DF89C1000EB01108078C0F3400017
:10F17000D0B99DF8AC0000EB400101EB00118548CF
:10F1800000EB011030309DF89C1000EB0110801C4A
:10F190000990007820F00800083003E069E087E07B
:10F1A000B5E0F9E0099908709DF8AC100220FAF773
:10F1B000CFFE7CE09DF8AC00C0EBC00101EB8011FC
:10F1C000734800EB411160319DF89C0000EB00108A
:10F1D00011F830109DF8AC00C0EBC00202EB8012B9
:10F1E0006B4800EB42100079814260D19DF8AC0081
:10F1F000C0EBC00101EB8011654800EB41106030AD
:10F200009DF89C1001EB011100EBC1008078A12852
:10F2100030D0A3229DF8AC00C0EBC00101EB8011FF
:10F220005B4800EB411160319DF89C0000EB001041
:10F2300001EBC00042719DF8AC00C0EBC00101EBD6
:10F240008011534800EB411060309DF89C1001EB99
:10F25000011100EBC1008078A22828D000219DF880
:10F26000AC00C0EBC00202EB8012494800EB421038
:10F27000C1701CE0A1229DF8AC00C0EBC00101EB05
:10F280008011434800EB411160319DF89C0000EB78
:10F29000001001EBC000427101219DF8AC00C0EBF1
:10F2A000C00202EB80123A4800EB4210C17032E417
:10F2B000A1229DF8AC00C0EBC00101EB80113448E5
:10F2C00000EB411160319DF89C0000EB001001EB58
:10F2D000C00082709DF8AC00C0EBC00101EB801152
:10F2E0002B4800EB411160319DF89C0000EB0010B1
:10F2F00001EBC000427100219DF8AC00C0EBC002E0
:10F3000002EB8012224800EB4210C170C1E49DF86C
:10F31000AC00C0EBC00101EB80111D4800EB4110B7
:10F3200060309DF89C1001EB011110F831000628A7
:10F330002DDC00219DF8AC00C0EBC00202EB801276
:10F34000134800EB4210C17007229DF8AC00C0EBDF
:10F35000C00101EB80110E4800EB411160319DF8B6
:10F360009C0000EB001001F83020A7229DF8AC00B3
:10F37000C0EBC00101EB8011054800EB411060308B
:10F380009DF89C1001EB011100EBC100427180E47B
:10F39000FC3400203C30002000219DF8AC00C0EB84
:10F3A000C00202EB8012FE4800EB4210C170A7229F
:10F3B0009DF8AC00C0EBC00101EB8011F84800EBF8
:10F3C000411160319DF89C0000EB001001EBC00082
:10F3D00042719DF8AC0000EB4001C1EBC010F14957
:10F3E00001EBC000407930287DD19DF8AC00C0EB26
:10F3F000C00101EB8011EA4800EB411160319DF83A
:10F400009C0000EB001011F830109DF8AC00C0EB30
:10F41000C00202EB8012E24800EB42100079814208
:10F4200061D19DF8AC0000EB400101EB0011DE481A
:10F4300000EB011030309DF89C1000EB0110801C97
:10F440000990007820F00102099802709DF8AC0044
:10F4500000EB400101EB0011D34800EB011030300C
:10F460009DF89C1000EB0110801C0990007820F0A2
:10F470000202099802709DF8AC00C0EBC00101EBDC
:10F480008011C74800EB411060309DF89C1001EBE3
:10F49000011100EBC100C07831282ED19DF8AC00DD
:10F4A00000EB400101EB0011BF4800EB01103030D0
:10F4B0009DF89C1000EB0110801C0990007820F052
:10F4C00020020998027000229DF8AC00C0EBC00138
:10F4D00001EB8011B24800EB411060309DF89C10A8
:10F4E00001EB011100E02FE000EBC10080F83D20AE
:10F4F0009DF8AC100220FAF72BFD9DF8AC00C0EB94
:10F50000C00101EB8011A64800EB411060309DF86E
:10F510009C1001EB011100EBC10090F83E000128A6
:10F5200011D1A9229DF8AC00C0EBC00101EB801104
:10F530009B4800EB411060309DF89C1001EB0111DD
:10F5400000EBC100827072E29DF8AC0000EB40015C
:10F55000C1EBC011934800EBC100407931287DD147
:10F560009DF8AC00C0EBC00101EB80118C4800EBB2
:10F57000411160319DF89C0000EB001011F8301033
:10F580009DF8AC00C0EBC00202EB8012844800EB97
:10F5900042100079814261D19DF8AC00C0EBC001FE
:10F5A00001EB80117E4800EB411060309DF89C100B
:10F5B00001EB011100EBC10090F83E0040BB0122BD
:10F5C0009DF8AC00C0EBC00101EB8011744800EB6A
:10F5D000411160319DF89C0000EB001001EBC00070
:10F5E00080F83D209DF8AC0000EB400101EB0011DC
:10F5F0006D4800EB011130319DF89C0001EB0010CB
:10F60000801C0990007820F00100401C09990870C6
:10F610009DF8AC0000EB400101EB0011624800EBEB
:10F62000011030309DF89C1000EB0110801C0990F7
:10F63000007820F00202099802705C4890F8C80730
:10F64000F0BB5B48407F01283AD15948C06D58490A
:10F65000C98B884234D29DF8AC0000E0B0E0C0EB2A
:10F66000C00101EB80114E4800EB411060309DF865
:10F670009C1001EB011100EBC10090F83D00012846
:10F680001ED19DF8AC00C0EBC00101EB80114448D5
:10F6900000EB411060309DF89C1001EB011100EB74
:10F6A000C10090F8770058B94FF010429DF8AC00B7
:10F6B000C0EBC00101EB8011394800EB411100E0C3
:10F6C0007DE060319DF89C0000EB001001EBC00074
:10F6D00082609DF8AC0000EB400101EB0011324864
:10F6E00000EB011130319DF89C0001EB0010017816
:10F6F0009DF8AC00C0EBC00202EB8012284800EB82
:10F70000421041709DF8AC00C0EBC00101EB8011CC
:10F71000234800EB411160319DF89C0000EB001084
:10F7200011F830109DF8AC00C0EBC00202EB801263
:10F730001B4800EB42100079814240D100229DF825
:10F74000AC00C0EBC00101EB8011154800EB41118A
:10F7500060319DF89C0000EB001001EBC000C2710D
:10F76000A4229DF8AC00C0EBC00101EB80110C4855
:10F7700000EB411160319DF89C0000EB001001EBA3
:10F78000C0008270A3229DF8AC00C0EBC00101EB69
:10F790008011034800EB411060309DF89C1009E097
:10F7A000FC340020246600203C300020BC220020D5
:10F7B000BC12002001EB011100EBC100427136E1E7
:10F7C0009DF8AC0000EB4001C1EBC010FE4901EB1D
:10F7D000C0004079332879D19DF8AC0000EB40019E
:10F7E00001EB0011F94800EB011030309DF89C103E
:10F7F00000EB0110801C0990007820F00100401CF3
:10F80000099908709DF8AC1001EB410000EB011163
:10F81000EE4800EB011030309DF89C1000EB011019
:10F82000801C0990007820F02002099802709DF851
:10F83000AC1001EB410000EB0111E44800EB0110BA
:10F8400030309DF89C1000EB0110801C099000786E
:10F8500020F00200801C099908709DF8AC10C1EBE3
:10F86000C10000EB8111DA4800EB411002799DF8EC
:10F87000AC00C0EBC00101EB8011D54800EB41109A
:10F8800060309DF89C1001EB011100F831209DF8CB
:10F89000AC1001EB410000EB0111CC4800EB011072
:10F8A00030309DF89C1000EB0110801C099000780E
:10F8B00020F080008030099908709DF8AC1001EBB1
:10F8C000410000EB0111C14801E055E322E000EBEB
:10F8D000011030309DF89C1000EB01108078C0F3CF
:10F8E000400020B99DF8AC100220FAF731FBA222AB
:10F8F0009DF8AC00C0EBC00101EB8011B44800EBF7
:10F90000411060309DF89C1001EB011100EBC1002B
:10F9100082708CE09DF8AC1001EB4100C0EBC1108F
:10F92000A94901EBC000407934287DD19DF8AC1085
:10F9300001EB410000EB0111A44800EB0110303055
:10F940009DF89C1000EB0110801C0990007820F0BD
:10F950002002099802709DF8AC1001EB410000EB09
:10F9600001119A4800EB011030309DF89C1000EB1B
:10F970000110801C0990007820F0020209980270A2
:10F9800001229DF8AC00C0EBC00101EB8011904852
:10F9900000EB411060309DF89C1001EB011100EB71
:10F9A000C10080F83E20A9229DF8AC00C0EBC00148
:10F9B00001EB8011864800EB411060309DF89C10EF
:10F9C00001EB011100EBC10082709DF8AC10C1EB9E
:10F9D000C10000EB81117E4800EB411002799DF8D7
:10F9E000AC00C0EBC00101EB8011794800EB411085
:10F9F00060309DF89C1001EB011100F831209DF85A
:10FA0000AC1001EB410000EB0111704800EB01105C
:10FA100030309DF89C1000EB0110801C099000789C
:10FA200020F08000803000E001E00999087000209B
:10FA30002C902D900021369122E0DDE92C10000160
:10FA400040EA11720901CDE92C129DF8AC1001EBCE
:10FA50004100C0EBC1105C4901EBC001BDF8D8000A
:10FA6000801D085C3038C117DDE92C34184341EAA9
:10FA70000402CDE92C02BDF8D800401C80B23690BB
:10FA8000BDF8D8000628D8DB9DF8AC002C99C0EB57
:10FA9000C00202EB80124E4800EB421260329DF829
:10FAA0009C0000EB001002EBC000C0F81A1000220E
:10FAB0002C922D920021369122E0DDE92C100001DC
:10FAC00040EA11720901CDE92C129DF8AC1001EB4E
:10FAD0004100C0EBC1103C4901EBC001BDF8D800AA
:10FAE0000D30085C3038C117DDE92C34184341EA89
:10FAF0000402CDE92C02BDF8D800401C80B236903B
:10FB0000BDF8D8000428D8DB9DF8AC002C99C0EBD8
:10FB1000C00202EB80122E4800EB421260329DF8C8
:10FB20009C0000EB001002EBC000416300222C920D
:10FB30002D920021369122E0DDE92C10000140EAEF
:10FB400011720901CDE92C129DF8AC1001EB4100B6
:10FB5000C0EBC1101C4901EBC001BDF8D800113049
:10FB6000085C3038C117DDE92C34184341EA04023F
:10FB7000CDE92C02BDF8D800401C80B23690BDF80B
:10FB8000D8000628D8DB9DF8AC002C99C0EBC00249
:10FB900002EB80120E4800EB421260329DF89C008E
:10FBA00000EB001002EBC000C0F81E109DF8AC1076
:10FBB00001EB4100C0EBC110034901EBC0004279E9
:10FBC0009DF8AC0006E00000246600203C300020D8
:10FBD000FC340020C0EBC00101EB8011FE4800EBBB
:10FBE000411160319DF89C0000EB001001EBC0005A
:10FBF000C2709DF8AC1001EB410000EB0111F74819
:10FC000000EB011130319DF89C0001EB001082786F
:10FC10009DF8AC00C0EBC00101EB8011EE4800EB99
:10FC2000411160319DF89C0000EB001001EBC00019
:10FC300002769DF8AC10C1EBC10000EB8111E648E3
:10FC400000EB411160319DF89C0000EB001011F8B1
:10FC500030109DF8AC00C0EBC00202EB8012DE4811
:10FC600000EB4210007981427EDA00219DF8AC0061
:10FC7000C0EBC00202EB8012D74800EB4210C1700B
:10FC8000A7229DF8AC00C0EBC00101EB8011D24867
:10FC900000EB411160319DF89C0000EB001001EB7E
:10FCA000C000427101219DF8AC00C0EBC00202EB24
:10FCB0008012C94800EB4210C1709DF8AC10C1EB36
:10FCC000C10000EB8111C44800EB411002799DF89E
:10FCD000AC00C0EBC00101EB8011BF4800EB41114B
:10FCE00060319DF89C0000EB001001F83020A1224B
:10FCF0009DF8AC00C0EBC00101EB8011B64800EBF1
:10FD0000411160319DF89C0000EB001001EBC00038
:10FD100042719DF8AC1001EB410000EB0111AF48BE
:10FD200000EB011130319DF89C0001EB0010801CAC
:10FD30000990007820F080008030099908709DF8C3
:10FD4000AC1001EB410000EB0111A44800EB0110E5
:10FD500030309DF89C1000EB0110801C0990007859
:10FD600020F00400001D00E051E0099908709DF8A2
:10FD7000AC1001EB410000EB0111984800EB0110C1
:10FD800030309DF89C1000EB01108078C0F34010DB
:10FD9000E8B39DF8AC1001EB410000EB01118F4876
:10FDA00000EB011030309DF89C1000EB0110801C1E
:10FDB0000990007820F02002099802709DF8AC109C
:10FDC00001EB410000EB0111844800EB01103030E1
:10FDD0009DF89C1000EB01108078C0F34000E8BB58
:10FDE0009DF8AC1001EB410000EB01117B4800EBEA
:10FDF000011030309DF89C1000EB0110801C099020
:10FE0000007820F0080008300999087000E0B2E09E
:10FE10009DF8AC009DF89C1001EB0010C217CDE9D5
:10FE20002C0200222C9800EB8001C1EB80116C4861
:10FE30000844C0F81D209DF8AC10C1EBC10000EBD8
:10FE40008111654800EB411060309DF89C1001EB7A
:10FE5000011100EBC1002230099000E086E02C98EF
:10FE600000EB8001C1EB80115D4801440D3110228F
:10FE70000891DDE90801F8F7E8F99DF8AC10C1EB4D
:10FE8000C10000EB8111544800EB411160319DF835
:10FE90009C0000EB001001EBC0012C9800EB8002ED
:10FEA000C2EB80124E48104451F81A2F40F8012F2F
:10FEB000496841609DF8AC1001EB410000EB011175
:10FEC000464800EB011130319DF89C0001EB001019
:10FED00001782C9800EB8002C2EB801240488154DC
:10FEE0002C9800EB8001C1EB80113D4801443D4856
:10FEF000026F41F8212FB0F8740088809DF8AC1093
:10FF0000C1EBC10000EB8111334800EB41116031BE
:10FF10009DF89C0000EB001001EBC000416B2C9899
:10FF200000EB8002C2EB80122D481044C0F809108B
:10FF30009DF8AC1001EB410000EB0111274800EBEC
:10FF4000011130319DF89C0001EB001041682C98A4
:10FF500000EB8002C2EB801221481044C0F8271049
:10FF60002C9881B208200991F9F7F2FF9DF8AC10A6
:10FF70000220F9F7EDFF82E200219DF8AC00C0EB12
:10FF8000C00202EB8012144800EB4210C1709DF8D1
:10FF9000AC10C1EBC10000EB81110F4800EB411028
:10FFA00060309DF89C1001EB011110F831000A2817
:10FFB0001ADC0B229DF8AC00C0EBC00101EB8011F4
:10FFC000054800EB411060309DF89C1001EB0111D9
:10FFD00000F831209EE10000FC3400203C3000207D
:10FFE000201300203C2600209DF8AC10C1EBC1007E
:10FFF00000EB8111FD4800EB411160319DF89C0040
:020000040801F1
:1000000000EB001011F830109DF8AC00C0EBC002FE
:1000100002EB8012F54800EB4210007981427DD15D
:10002000F34890F8C807E8BB0021F248C0F83D103B
:100030009DF8AC10C1EBC10000EB8111EB4800EB67
:10004000411060309DF89C1001EB011100EBC100E4
:100050002230102201460990E6482D30F8F7F5F8D5
:100060009DF8AC10C1EBC10000EB8111DF4800EB43
:10007000411060309DF89C1001EB011100EBC101B3
:10008000DC48401C51F81A2F0262496841629DF811
:10009000AC1001EB410000EB0111D74800EB01105F
:1000A000303000E055E09DF89C1000EB0110007826
:1000B000D04981F820009DF8AC10C1EBC10000EBE5
:1000C0008111CA4800EB411060309DF89C1001EB93
:1000D000011100EBC100416BC648C0F82910213066
:1000E000C6490A6F0262B1F8741081842138C06D6C
:1000F00080B2014609900220F8F7EAFF00210620AD
:10010000F9F726FFBB48C06DBA49C98B884204D2B3
:10011000B848C06D401CB749C86500E0FAE000214E
:100120000520F9F715FF9DF8AC1001EB410000EB3D
:100130000111B14800EB011030309DF89C1000EB2C
:100140000110801C0990007820F0080209980270C4
:1001500015E09DF8AC1001EB410000EB0111A64841
:1001600000EB011030309DF89C1000EB0110801C5A
:100170000990007820F008000830099908700022E2
:100180009DF8AC00C0EBC00101EB8011974800EB7B
:10019000411160319DF89C0000EB001001EBC000A4
:1001A00080F83E209DF8AC100220F9F7D1FE9DF8B2
:1001B000AC109DF89C0000EB0110C217CDE92C0299
:1001C00000222C9800EB8001C1EB8011894864303B
:1001D0000844C0F81D209DF8AC10C1EBC10000EB35
:1001E0008111824800EB411060309DF89C1001EBBA
:1001F000011100EBC100223009902C9800EB800126
:10020000C1EB80117B48643001440D31102208910C
:10021000DDE90801F8F719F89DF8AC10C1EBC10051
:1002200000EB8111714800EB411160319DF89C0099
:1002300000EB001001EBC0012C9800EB8002C2EB38
:1002400080126C486430104451F81A2F40F8012F86
:10025000496841609DF8AC1001EB410000EB0111D1
:10026000654800EB011130319DF89C0001EB001056
:1002700001782C9800EB8002C2EB80125D4864305C
:1002800081542C9800EB8001C1EB801159486430F7
:1002900001445A48026F41F8212FB0F87400888059
:1002A0009DF8AC10C1EBC10000EB81114F4800EB91
:1002B000411160319DF89C0000EB001001EBC00083
:1002C000416B2C9800EB8002C2EB801249486430ED
:1002D0001044C0F809109DF8AC1001EB410000EB90
:1002E0000111454800EB011130319DF89C0001EBF4
:1002F000001041682C9800EB8002C2EB80123D4850
:1003000064301044C0F827102C9881B2082009915D
:10031000F9F71EFEA7229DF8AC00C0EBC00101EB6F
:100320008011324800EB411160319DF89C0000EBD8
:10033000001001EBC0004271A2229DF8AC00C0EB9E
:10034000C00101EB8011294800EB411160319DF89B
:100350009C0000EB001001EBC000827000222C9288
:100360002D920021369122E0DDE92C10000140EAB7
:1003700011720901CDE92C129DF8AC1001EB41007E
:10038000C0EBC1101E4901EBC001BDF8D8000B3015
:10039000085C3038C117DDE92C34184341EA040207
:1003A000CDE92C02BDF8D800401C80B23690BDF8D3
:1003B000D8000A28D8DB9DF8AC00DDE92C12C0EB90
:1003C000C00303EB8013094800EB431360339DF82F
:1003D0009C0000EB001003EBC00040F8221F4260BD
:1003E00000222C922D92002136912EE0FC34002028
:1003F000BC220020BC1200203C3000203C26002003
:1004000024660020DDE92C10000140EA1172090188
:10041000CDE92C129DF8AC1001EB4100C0EBC110EE
:10042000FE4901EBC001BDF8D8001530085C30383A
:10043000C117DDE92C34184341EA0402CDE92C024E
:10044000BDF8D800401C80B23690BDF8D8000A280C
:10045000D8DB9DF8AC00DDE92C21C0EBC00303EB39
:100460008013EF4800EB431060309DF89C3003EBA5
:10047000031300EBC30022308260C16000BF00BFE5
:1004800005F01CBE9DF8AC1001EB4100C0EBC110A3
:10049000E24911F83000042801D125900BE09DF8C5
:1004A000AC1001EB4100C0EBC110DC4911F8300089
:1004B000152800D125909DF8AC1001EB4100C0EB50
:1004C000C110D64901EBC00041789DF8AC0000EBAB
:1004D0004002C2EBC010D14A12F8300041EA0020BD
:1004E00041F23001884202D1A62025903DE09DF8DE
:1004F000AC1001EB4100C0EBC110C84901EBC000DA
:1005000041789DF8AC0000EB4002C2EBC010C34A3A
:1005100012F8300041EA002041F23101884202D154
:10052000A720259021E09DF8AC1001EB4100C0EB25
:10053000C110BA4911F83000022816D19DF8AC104C
:1005400001EB4100C0EBC110B44901EBC0000179DF
:100550009DF8AC0000EB4002C2EBC010AF4A02EBCA
:10056000C000C07841EA002125919DF8AC10C1EB94
:10057000C10000EB8111AA4800EB4110817827915E
:100580000021A84A9DF8AC0002EB00129DF89C00E7
:100590001154A548007F012815D19DF8AC1001EB3E
:1005A000410000EB0111A14800EB011030309DF833
:1005B0009C1000EB0110801C0990007820F0800056
:1005C0008030099908709DF8AC1001EB410000EBF8
:1005D0000111964800EB011030309DF89C1000EBA3
:1005E0000110801C0990007820F0400040300999EB
:1005F0000870BDF89400A7287DD006DC04287BD0C5
:1006000015287AD0A62848D148E0A0F558503038AF
:1006100020B1112872D01228F5D1FDE39DF8AC105D
:10062000C1EBC10000EB81117D4800EB411060304F
:100630009DF89C1001EB011110F8310068BB0021FE
:100640009DF8AC00C0EBC00202EB8012744800EBD6
:100650004210C17001229DF8AC00C0EBC00101EB5B
:1006600080116F4800EB411160319DF89C0000EB58
:10067000001001F83020A7229DF8AC00C0EBC001AB
:1006800001EB8011664800EB411160319DF89C0040
:1006900000EB001001EBC0004271FDE300219DF86A
:1006A000AC00C0EBC00202EB80125D4800EB4210D0
:1006B000C1709DF8AC10C1EBC10000EB811158482E
:1006C00000EB411060309DF89C1001EB011110F817
:1006D0003100022828DC03229DF8AC00C0EBC001E9
:1006E00001EB80114E4800EB411160319DF89C00F8
:1006F00000EB001003E0C9E027E14BE279E201F8EA
:100700003020A9229DF8AC00C0EBC00101EB8011A4
:10071000434800EB411060309DF89C1001EB011143
:1007200000EBC1004271B0E09DF8AC10C1EBC1001C
:1007300000EB81113A4800EB411060309DF89C10AD
:1007400001EB011110F83100052823DC06229DF889
:10075000AC00C0EBC00101EB8011314800EB41114E
:1007600060319DF89C0000EB001001F83020A222BF
:100770009DF8AC00C0EBC00101EB8011284800EBF4
:10078000411060309DF89C1001EB011100EBC1009D
:1007900042717AE09DF8AC10C1EBC10000EB811111
:1007A0001F4800EB411060309DF89C1001EB0111D7
:1007B00000EBC1004079A52815D19DF8AC1001EBE4
:1007C000410000EB0111194800EB011030309DF899
:1007D0009C1000EB0110801C0990007820F00400B0
:1007E000001D099908709DF8AC10C1EBC10000EB29
:1007F00081110B4800EB411060309DF89C1001EB1B
:10080000011100EBC1008078A1283ED09DF8AC100A
:10081000C1EBC10000EB8111014809E02466002012
:10082000FC340020702E0020BC1200203C30002040
:1008300000EB411160319DF89C0000EB001001EBD2
:10084000C00082789DF8AC00C0EBC00101EB8011C4
:10085000FE4800EB411160319DF89C0000EB001058
:1008600001EBC0004271A1229DF8AC00C0EBC001B9
:1008700001EB8011F54800EB411060309DF89C10B1
:1008800001EB011100EBC100827006E79DF8AC108E
:10089000C1EBC10000EB8111EC4800EB411060306E
:1008A0009DF89C1001EB011100EBC1004079A428D8
:1008B0002DD19DF8AC1001EB410000EB0111E44893
:1008C00000EB011030309DF89C1000EB0110801CF3
:1008D0000990007820F0200020300999087000224B
:1008E0009DF8AC00C0EBC00101EB8011D74800EBD4
:1008F000411060309DF89C1001EB011100EBC1002C
:1009000080F83D209DF8AC100220F9F721FB002172
:100910009DF8AC00C0EBC00202EB8012CB4800EBAC
:100920004210C170A1229DF8AC00C0EBC00101EBE8
:100930008011C64800EB411060309DF89C1001EB1F
:10094000011100EBC1004271A7E69DF8AC10C1EBAC
:10095000C10000EB8111BD4800EB411060309DF8F3
:100960009C1001EB011110F8310001282EDC002150
:100970009DF8AC00C0EBC00202EB8012B34800EB64
:100980004210C17002229DF8AC00C0EBC00101EB27
:100990008011AE4800EB411160319DF89C0000EBE6
:1009A000001001F83020A3229DF8AC00C0EBC0017C
:1009B00001EB8011A54800EB411060309DF89C10C0
:1009C00001EB011100EBC1004271E2E09DF8AC10B7
:1009D000C1EBC10000EB81119C4800EB411060307D
:1009E0009DF89C1001EB011110F8310004282EDC59
:1009F00000219DF8AC00C0EBC00202EB80129348CE
:100A000000EB4210C17005229DF8AC00C0EBC001A4
:100A100001EB80118D4800EB411160319DF89C0085
:100A200000EB001001F83020A3229DF8AC00C0EBD1
:100A3000C00101EB8011854800EB411060309DF84A
:100A40009C1001EB011100EBC1004271A1E09DF887
:100A5000AC10C1EBC10000EB81117C4800EB4110F0
:100A600060309DF89C1001EB011110F83100062850
:100A700012DCA1229DF8AC00C0EBC00101EB80119B
:100A8000724800EB411060309DF89C1001EB0111A1
:100A900000EBC10042717CE09DF8AC10C1EBC100DD
:100AA00000EB8111694800EB411160319DF89C0019
:100AB00000EB001011F830109DF8AC00C0EBC00244
:100AC00002EB8012614800EB42100079814260D154
:100AD0009DF8AC10C1EBC10000EB81115B4800EB4D
:100AE000411060309DF89C1001EB011100EBC1003A
:100AF0008078A12830D0A3229DF8AC00C0EBC001C3
:100B000001EB8011514800EB411160319DF89C00D0
:100B100000EB001001EBC00042719DF8AC10C1EB7E
:100B2000C10000EB8111494800EB411060309DF895
:100B30009C1001EB011100EBC1008078A22828D0A5
:100B400000219DF8AC00C0EBC00202EB80123F48D0
:100B500000EB4210C1701CE0A1229DF8AC00C0EB7C
:100B6000C00101EB8011394800EB411160319DF863
:100B70009C0000EB001001EBC000427101219DF8C8
:100B8000AC00C0EBC00202EB8012304800EB421018
:100B9000C17082E5A1229DF8AC00C0EBC00101EB61
:100BA00080112A4800EB411160319DF89C0000EB58
:100BB000001001EBC00042719DF8AC00C0EBC00119
:100BC00001EB8011214800EB411160319DF89C0040
:100BD00000EB001001EBC000827000219DF8AC001A
:100BE000C0EBC00202EB8012184800EB4210C1704B
:100BF00053E500219DF8AC00C0EBC00202EB80126F
:100C0000124800EB4210C170A7229DF8AC00C0EB67
:100C1000C00101EB80110D4800EB411160319DF8DE
:100C20009C0000EB001001EBC00042719DF8AC107D
:100C300001EB4100C0EBC110064901EBC000407957
:100C400030287DD19DF8AC1006E00000FC34002077
:100C50003C30002024660020C1EBC10000EB811174
:100C6000FE4800EB411160319DF89C0000EB001044
:100C700011F830109DF8AC00C0EBC00202EB8012FE
:100C8000F64800EB42100079814259D19DF8AC1032
:100C900001EB410000EB0111F14800EB0110303095
:100CA0009DF89C1000EB0110801C0990007820F04A
:100CB0000102099802709DF8AC1001EB410000EBB5
:100CC0000111E74800EB011030309DF89C1000EB5B
:100CD0000110801C0990007820F00202099802702F
:100CE0009DF8AC10C1EBC10000EB8111DB4800EBBB
:100CF000411060309DF89C1001EB011100EBC10028
:100D0000C07831282ED19DF8AC1001EB410000EBEA
:100D10000111D34800EB011030309DF89C1000EB1E
:100D20000110801C0990007820F0200209980270C0
:100D300000229DF8AC00C0EBC00101EB801100E087
:100D400037E0C64800EB411160319DF89C0000EB94
:100D5000001001EBC00080F83D209DF8AC1002208F
:100D6000F9F7F6F89DF8AC10C1EBC10000EB81116A
:100D7000BA4800EB411060309DF89C1001EB011166
:100D800000EBC10090F83E00012811D1A9229DF886
:100D9000AC00C0EBC00101EB8011B04800EB41108A
:100DA00060309DF89C1001EB011100EBC1008270D6
:100DB00074E29DF8AC1001EB4100C0EBC110A949F1
:100DC00001EBC0004079312867D19DF8AC10C1EB30
:100DD000C10000EB8111A14800EB411160319DF889
:100DE0009C0000EB001011F830109DF8AC00C0EB37
:100DF000C00202EB8012994800EB42100079814258
:100E00004BD19DF8AC10C1EBC10000EB81119348B0
:100E100000EB4110603000E0FEE39DF89C1001EB18
:100E2000011100EBC10090F83E0040BB01229DF88B
:100E3000AC00C0EBC00101EB8011884800EB411110
:100E400060319DF89C0000EB001001EBC00080F8C1
:100E50003D209DF8AC1001EB410000EB01118048F2
:100E600000EB011130319DF89C0001EB0010801C5B
:100E70000990007820F00100401C099908709DF845
:100E8000AC1001EB410000EB0111754800EB0110C3
:100E900030309DF89C1001E0F1E3BEE000EB011062
:100EA000801C0990007820F00202099802706E48B8
:100EB00090F8C807E8BB6D48407F012839D16B48DE
:100EC000C06D6A49C98B884233D29DF8AC10C1EB22
:100ED000C10000EB8111614800EB411060309DF8CA
:100EE0009C1001EB011100EBC10090F83D000128BE
:100EF0001FD19DF8AC10C1EBC10000EB8111574828
:100F000000EB411060309DF89C1001EB011100EBEB
:100F1000C10090F8770060B94FF010429DF8AC0026
:100F2000C0EBC00101EB80114C4800EB4111603176
:100F300000E071E09DF89C0000EB001001EBC000A8
:100F400082609DF8AC1001EB410000EB01114448B8
:100F500000EB011130319DF89C0001EB001001788D
:100F60009DF8AC00C0EBC00202EB80123B4800EBE6
:100F7000421041709DF8AC10C1EBC10000EB811133
:100F8000364800EB411160319DF89C0000EB0010E9
:100F900011F830109DF8AC00C0EBC00202EB8012DB
:100FA0002E4800EB42100079814235D100229DF895
:100FB000AC00C0EBC00101EB8011284800EB4111EF
:100FC00060319DF89C0000EB001001EBC000C27185
:100FD000A4229DF8AC00C0EBC00101EB80111F48BA
:100FE00000EB411160319DF89C0000EB001001EB1B
:100FF000C0008270A3229DF8AC00C0EBC00101EBE1
:101000008011164800EB411060309DF89C1001EBF8
:10101000011100EBC100427140E19DF8AC1001EB01
:101020004100C0EBC1100F4901EBC00040793328EB
:101030007ED19DF8AC1001EB410000EB0111084896
:1010400000EB011030309DF89C1000EB0110801C6B
:101050000990007820F00100401C09E0FC340020D9
:101060003C30002024660020BC220020BC1200205E
:10107000099908709DF8AC1001EB410000EB0111DB
:10108000FE4800EB011030309DF89C1000EB011081
:10109000801C0990007820F02002099802709DF8C9
:1010A000AC1001EB410000EB0111F44800EB011022
:1010B00030309DF89C1000EB0110801C09900078E6
:1010C00020F00200801C099908709DF8AC10C1EB5B
:1010D000C10000EB8111EA4800EB411002799DF854
:1010E000AC00C0EBC00101EB8011E54800EB411002
:1010F00060309DF89C1001EB011100F831209DF843
:10110000AC1001EB410000EB0111DC4800EB0110D9
:1011100030309DF89C1000EB0110801C0990007885
:1011200020F080008030099908709DF8AC1000E034
:1011300027E001EB410000EB0111D04800EB01106A
:1011400030309DF89C1000EB01108078C0F3400017
:1011500020B99DF8AC100220F8F7FAFEA2229DF803
:10116000AC00C0EBC00101EB8011C54800EB4110A1
:1011700060309DF89C1001EB011100EBC100827002
:101180008CE09DF8AC1001EB4100C0EBC110BD49F3
:1011900001EBC000407934287ED19DF8AC1001EB02
:1011A000410000EB0111B54800EB011030309DF813
:1011B0009C1000EB0110801C0990007820F02002A8
:1011C000099802709DF8AC1001EB410000EB011191
:1011D000AA4800EB011030309DF89C1000EB011084
:1011E000801C0990007820F0020209980270012208
:1011F0009DF8AC00C0EBC00101EB8011A04800EBF2
:10120000411160319DF89C0000EB001001EBC00023
:1012100080F83E20A9229DF8AC00C0EBC00101EB94
:101220008011974800EB411160319DF89C0000EB64
:10123000001001EBC00082709DF8AC10C1EBC10042
:1012400000EB81118E4800EB411002799DF8AC0053
:10125000C0EBC00101EB8011894800EB4111603106
:101260009DF89C0000EB001001F830209DF8AC10B8
:1012700001EB410000EB0111804800EB0110303020
:101280009DF89C1000EB0110801C0990007820F064
:1012900080008030099900E000E0087000202C9068
:1012A0002D900021369122E0DDE92C10000140EA6A
:1012B00011720901CDE92C129DF8AC1001EB41002F
:1012C000C0EBC1116F4800EBC101BDF8D800801D13
:1012D000085C3038C117DDE92C34184341EA0402B8
:1012E000CDE92C02BDF8D800401C80B23690BDF884
:1012F000D8000828D8DB9DF8AC002C99C0EBC002C0
:1013000002EB80125E4800EB421260329DF89C00B6
:1013100000EB001002EBC000C0F81A1000222C9263
:101320002D920021369122E0DDE92C10000140EAE7
:1013300011720901CDE92C129DF8AC1001EB4100AE
:10134000C0EBC1104F4901EBC001BDF8D8000F3010
:10135000085C3038C117DDE92C34184341EA040237
:10136000CDE92C02BDF8D800401C80B23690BDF803
:10137000D8000628D8DB9DF8AC002C99C0EBC00241
:1013800002EB80123E4800EB421260329DF89C0056
:1013900000EB001002EBC000416300222C922D9262
:1013A0000021369122E0DDE92C10000140EA1172A3
:1013B0000901CDE92C129DF8AC1001EB4100C0EB06
:1013C000C110304901EBC001BDF8D8001530085CF0
:1013D0003038C117DDE92C34184341EA0402CDE965
:1013E0002C02BDF8D800401C80B23690BDF8D80061
:1013F0000828D8DB9DF8AC002C99C0EBC00202EBAA
:1014000080121F4800EB421260329DF89C0000EBF6
:10141000001002EBC000C0F81E109DF8AC1001EBEC
:101420004100C0EBC110174901EBC00042799DF8A3
:10143000AC00C0EBC00101EB8011114800EB411181
:1014400060319DF89C0000EB001001EBC000C27001
:101450009DF8AC1001EB410000EB0111074800EBD7
:10146000011130319DF89C0001EB001082789DF84D
:10147000AC00C0EBC00101EB801105E03C30002066
:10148000FC34002024660020FE4800EB411160314E
:101490009DF89C0000EB001001EBC00002769DF867
:1014A000AC10C1EBC10000EB8111F64800EB41111B
:1014B00060319DF89C0000EB001011F830109DF891
:1014C000AC00C0EBC00202EB8012EE4800EB421011
:1014D000007981427EDA00219DF8AC00C0EBC002A9
:1014E00002EB8012E74800EB4210C170A7229DF882
:1014F000AC00C0EBC00101EB8011E24800EB4111F0
:1015000060319DF89C0000EB001001EBC0004271BF
:1015100001219DF8AC00C0EBC00202EB8012D9485B
:1015200000EB4210C1709DF8AC00C0EBC00101EBB4
:101530008011D44800EB411002799DF8AC00C0EB5B
:10154000C00101EB8011CF4800EB411160319DF8E3
:101550009C0000EB001001F83020A1229DF8AC00A7
:10156000C0EBC00101EB8011C64800EB41116031B6
:101570009DF89C0000EB001001EBC00042719DF84B
:10158000AC0000EB400101EB0011BF4800EB011182
:1015900030319DF89C0001EB0010801C0990007810
:1015A00020F080008030099908709DF8AC0000EBB5
:1015B000400101EB0011B44800EB011030309DF800
:1015C0009C1000EB0110801C0990007820F00400B2
:1015D000001D00E052E0099908709DF8AC0000EB96
:1015E000400101EB0011A84800EB011030309DF8DC
:1015F0009C1000EB01108078C0F34010F0B39DF810
:10160000AC0000EB400101EB00119F4800EB011022
:1016100030309DF89C1000E0E7E000EB0110801CEA
:101620000990007820F02002099802709DF8AC0023
:1016300000EB400101EB0011934800EB011030304A
:101640009DF89C1000EB01108078C0F34000E8BBCF
:101650009DF8AC0000EB400101EB00118A4800EB63
:10166000011030309DF89C1000EB0110801C099097
:10167000007820F008000830099901E0B4E04AE35E
:1016800008709DF8AC009DF89C1001EB0010C2178B
:10169000CDE92C0200222C9800EB8001C1EB8011D7
:1016A0007A480844C0F81D209DF8AC00C0EBC0018A
:1016B00001EB8011734800EB411060309DF89C10E5
:1016C00001EB011100EBC100223000E087E009903E
:1016D0002C9800EB8001C1EB80116C4801440D3166
:1016E00010220891DDE90801F6F7AFFD9DF8AC0086
:1016F000C0EBC00101EB8011624800EB4111603189
:101700009DF89C0000EB001001EBC0012C9800EB51
:101710008002C2EB80125D48104451F81A2F40F845
:10172000012F496841609DF8AC0000EB400101EBDE
:101730000011554800EB011130319DF89C0001EB80
:10174000001001782C9800EB8002C2EB80124F4809
:1017500081542C9800EB8001C1EB80114B4801446F
:101760004B48026F41F8212FB0F8740088809DF833
:10177000AC00C0EBC00101EB8011424800EB41110D
:1017800060319DF89C0000EB001001EBC000416B44
:101790002C9800EB8002C2EB80123C481044C0F849
:1017A00009109DF8AC0000EB400101EB0011364838
:1017B00000EB011130319DF89C0001EB00104168F5
:1017C0002C9800EB8002C2EB801230481044C0F825
:1017D00027102C9881B208200991F8F7B9FB9DF8E1
:1017E000AC100220F8F7B4FB95E200219DF8AC00A4
:1017F000C0EBC00202EB8012224800EB4210C17025
:101800009DF8AC00C0EBC00101EB80111D4800EB5E
:10181000411060309DF89C1001EB011110F831006F
:10182000032811DC04229DF8AC00C0EBC00101EBE1
:101830008011144800EB411060309DF89C1001EBC2
:10184000011100F83120A0E19DF8AC10C1EBC100FE
:1018500000EB81110B4800EB411160319DF89C00B9
:1018600000EB001011F830109DF8AC00C0EBC00286
:1018700002EB8012034800EB4210007981427DD1D7
:10188000044809E0FC3400203C30002020130020F4
:101890003C260020BC22002090F8C807E8BB0021AD
:1018A000F948C0F83D109DF8AC10C1EBC10000EB49
:1018B0008111F64800EB411060309DF89C1001EB5F
:1018C000011100EBC1002230102201460990EE48C0
:1018D0002D30F6F7BAFC9DF8AC10C1EBC10000EB5F
:1018E0008111EA4800EB411060309DF89C1001EB3B
:1018F000011100EBC101E448401C51F81A2F0262AB
:10190000496841629DF8AC1001EB410000EB011108
:10191000DF4800EB0110303000E055E09DF89C10EE
:1019200000EB01100078D84981F820009DF8AC1038
:10193000C1EBC10000EB8111D44800EB41106030D5
:101940009DF89C1001EB011100EBC100416BCE48EA
:10195000C0F829102130CF490A6F0262B1F8741023
:1019600081842138C06D80B2014609900220F7F7CA
:10197000AFFB00210620F8F7EBFA00E005E1C248D2
:10198000C06DC149C98B884204D2BF48C06D401C9C
:10199000BD49C86500210520F8F7DAFA9DF8AC10BA
:1019A00001EB410000EB0111B94800EB01103030B0
:1019B0009DF89C1000EB0110801C0990007820F02D
:1019C00008020998027015E09DF8AC1001EB410087
:1019D00000EB0111AE4800EB011030309DF89C1077
:1019E00000EB0110801C0990007820F008000830FE
:1019F0000999087000229DF8AC00C0EBC00101EB12
:101A00008011A24800EB411160319DF89C0000EB71
:101A1000001001EBC00080F83E209DF8AC100220C1
:101A2000F8F796FA9DF8AC109DF89C0000EB0110B9
:101A3000C217CDE92C0200222C9800EB8001C1EBEB
:101A40008011914864300844C0F81D209DF8AC0016
:101A5000C0EBC00101EB80118C4800EB41106030FD
:101A60009DF89C1001EB011100EBC10022300990A0
:101A70002C9800EB8001C1EB801183486430014455
:101A80000D3110220891DDE90801F6F7DEFB9DF823
:101A9000AC00C0EBC00101EB80117C4800EB4111B0
:101AA00060319DF89C0000EB001001EBC0012C9808
:101AB00000EB8002C2EB801273486430104451F88E
:101AC0001A2F40F8012F496841609DF8AC0000EBE7
:101AD000400101EB00116E4800EB011130319DF81F
:101AE0009C0001EB001001782C9800EB8002C2EB07
:101AF00080126548643081542C9800EB8001C1EB62
:101B000080116148643001446248026F41F8212F1E
:101B1000B0F8740088809DF8AC00C0EBC00101EB08
:101B200080115A4800EB411160319DF89C0000EB98
:101B3000001001EBC000416B2C9800EB8002C2EB5F
:101B40008012514864301044C0F809109DF8AC0070
:101B500000EB400101EB00114D4800EB0111303169
:101B60009DF89C0001EB001041682C9800EB80026E
:101B7000C2EB8012444864301044C0F827102C98FF
:101B800081B208200991F8F7E3F900229DF8AC0032
:101B9000C0EBC00101EB80113C4800EB411160310A
:101BA0009DF89C0000EB001001EBC00080F83E2087
:101BB000A7229DF8AC00C0EBC00101EB80113348B7
:101BC00000EB411160319DF89C0000EB001001EB2F
:101BD000C0004271A2229DF8AC00C0EBC00101EB35
:101BE00080112A4800EB411160319DF89C0000EB08
:101BF000001001EBC000827000222C922D92002177
:101C0000369122E0DDE92C10000140EA1172090151
:101C1000CDE92C129DF8AC0000EB4001C1EBC010E7
:101C20001D4901EBC001BDF8D8000B30085C30380D
:101C3000C117DDE92C34184341EA0402CDE92C0236
:101C4000BDF8D800401C80B23690BDF8D8000C28F2
:101C5000D8DB9DF8AC00DDE92C12C0EBC00303EB30
:101C600080130A4800EB431360339DF89C0000EB9F
:101C7000001003EBC00040F8221F426000222C92AB
:101C80002D92002136912CE0BC120020FC34002063
:101C90003C3000203C26002024660020DDE92C108A
:101CA000000140EA11720901CDE92C129DF8AC0047
:101CB00000EB4001C1EBC010FE4901EBC001BDF8D3
:101CC000D8001730085C3038C117DDE92C341843D0
:101CD00041EA0402CDE92C02BDF8D800401C80B2D4
:101CE0003690BDF8D8000C28D8DB9DF8AC00DDE9B3
:101CF0002C21C0EBC00303EB8013EF4800EB431033
:101D000060309DF89C3003EB031300EBC3002230DE
:101D10008260C16000BF00BF04F0D0B90021E74A73
:101D20009DF8AC0002EB00129DF89C0011549DF848
:101D3000AC0000EB4001C1EBC010DE4901EBC0007C
:101D4000407870280ED19DF8AC0000EB4001C1EB4B
:101D5000C010D84901EBC0008078FA2802D1B12028
:101D6000259042E09DF8AC0000EB4001C1EBC010B3
:101D7000D04901EBC000407800F0F000C0280ED13F
:101D80009DF8AC0000EB4001C1EBC010C94901EB6C
:101D9000C0008078FA2802D1B620259025E09DF871
:101DA000AC0000EB4001C1EBC010C24911F830009B
:101DB00000F0F000502818D19DF8AC0000EB400175
:101DC000C1EBC010BB4901EBC000407800F0F0004F
:101DD00030280AD19DF8AC0000EB4001C1EBC010E7
:101DE000B44901EBC000817825919DF8AC00C0EBAF
:101DF000C00101EB8011B04800EB411081782791C0
:101E00000021AE4A9DF8AC0002EB00129DF89C0048
:101E100011549DF8AC0000EB400101EB0011A84803
:101E200000EB011130319DF89C0001EB0010801C8B
:101E30000990007820F04000403009990870A148CE
:101E4000007F012815D19DF8AC0000EB400101EBAB
:101E500000119B4800EB011030309DF89C1000EB06
:101E60000110801C0990007820F0800080300999D2
:101E70000870BDF89400652872D004DC012809D0F0
:101E8000032805D173E0B12802D0B62800D100E0C4
:101E90007EE17DE19DF8AC0000EB4001C1EBC0109C
:101EA000844901EBC0000079012806D0022805D042
:101EB000032804D0052858D102E056E055E054E04C
:101EC0009DF8AC00C0EBC00101EB80117A4800EB3B
:101ED000411060309DF89C1001EB011110F83100A9
:101EE000E8BB00219DF8AC00C0EBC00202EB801201
:101EF000714800EB4210C17001229DF8AC00C0EBAC
:101F0000C00101EB80116C4800EB411160319DF87C
:101F10009C0000EB001001F83020B6229DF8AC00C8
:101F2000C0EBC00101EB8011634800EB411160314F
:101F30009DF89C0000EB001001EBC0004271B22242
:101F40009DF8AC00C0EBC00101EB80115A4800EBDA
:101F5000411060309DF89C1001EB011101E003E09D
:101F60002DE000EBC100827000BF00BF10E19DF8C2
:101F7000AC0000EB4001C1EBC0104E4901EBC000CA
:101F8000C179514880F8E8119DF8AC0000EB4001A0
:101F900001EB00114A4800EB011130319DF89C0023
:101FA00001EB0010801C0990474890F8E801C20836
:101FB0000998007862F3000009990870E8E09DF83C
:101FC000AC0000EB4001C1EBC0103A4901EBC0008E
:101FD000007900F0F00010B9B820259001E0B92098
:101FE00025909DF8AC0000EB4001C1EBC0103149D9
:101FF00001EBC000007900F00F012691002136911D
:1020000020E09DF8AC0000EB400101EB00112C48F2
:1020100000EB01113031BDF8D80001EB0010417820
:102020009DF8AC0000EB4002C2EBC010214A12F850
:1020300030005038814200D112E0BDF8D800401C79
:1020400081B236919DF8AC0000EB400101EB00112C
:102050001B4800EB0110C179BDF8D8008142D0DCEB
:1020600000BFBDF8D8109DF898000844C1B2279170
:102070009DF8AC00C0EBC00101EB80110E4800EBF5
:10208000411060309DF89C1001EB011110F83100F7
:1020900001283CD100219DF8AC00C0EBC00202EB4E
:1020A0008012054800EB4210C17002229DF8AC007E
:1020B0000CE0000024660020FC340020702E00207C
:1020C0003C300020BC120020BC220020C0EBC0012C
:1020D00001EB8011FE4800EB411160319DF89C003E
:1020E00000EB001001F83020B9229DF8AC00C0EBE5
:1020F000C00101EB8011F64800EB411060309DF803
:102100009C1001EB011100EBC10042713FE09DF812
:10211000AC10C1EBC10000EB8111ED4800EB4110A8
:1021200060309DF89C1001EB011110F8310001287E
:102130002DD100219DF8AC00C0EBC00202EB801253
:10214000E34800EB4210C17002229DF8AC00C0EBE6
:10215000C00101EB8011DE4800EB411160319DF8B8
:102160009C0000EB001001F83020B9229DF8AC0073
:10217000C0EBC00101EB8011D54800EB411060308D
:102180009DF89C1001EB011100EBC100427100BFF2
:1021900000BFC1E59DF8AC1001EB410000EB01115F
:1021A000CC4800EB0110007B20B101287DD0022833
:1021B0007CD1E4E2C8499DF8AC0031F81000801FE2
:1021C00081B209919DF8AC1001EB4100C0EBC11048
:1021D000C24901EBC000401C08900999F7F77AFB4F
:1021E0000022CDE92E029DF8AC1001EB4100C0EBBE
:1021F000C110BA4901EBC002B7489DF8AC1030F8E5
:102200001100401F111809910421099815F0C2FE10
:10221000C217CDE92C022DA819C82C99594060404D
:1022200001437DD1AE4A9DF8AC0002EB0010017075
:102230009DF8AC1001EB4100C0EBC110A74901EBC8
:10224000C00001792591BDF89400312802D04528BD
:1022500067D1EAE0A0489DF8AC1030F811001838BA
:10226000412190FBF1F0C217C1B2CDE92C029D488B
:1022700080F8901500203690CDE09DF8AC1001EB71
:102280004100C0EBC110954901EBC001BDF8D80079
:1022900000EB80101430095C934ABDF8D80011544B
:1022A0009DF8AC1001EB410001E0C1E066E2C0EB3B
:1022B000C1108A4901EBC001BDF8D80000EB8010C5
:1022C0001A30014409910821099815F021FE8DED7D
:1022D0000E0A854A0C32BDF8D8000E9902EB0010A8
:1022E00041609DF8AC1001EB4100C0EBC1107B498F
:1022F00001EBC001BDF8D80000EB80103230014482
:1023000009910821099815F003FE8DED0E0A764A11
:102310000C32BDF8D8000E9902EB0010016001E00C
:1023200085E083E09DF8AC1001EB4100C0EBC110EB
:102330006A4901EBC001BDF8D80000EB80103A30CB
:10234000014409910821099815F0E2FD8DED0E0A6E
:10235000654A0C32BDF8D8000E9902EB001081607E
:102360009DF8AC1001EB4100C0EBC1105B4901EBE3
:10237000C001BDF8D80000EB801042300144099143
:102380000821099815F0C4FD8DED0E0A564A0C324D
:10239000BDF8D8000E9902EB0010C1609DF8AC109A
:1023A00001EB410000EB01114A4800EB0111303113
:1023B000BDF8D80001EB0010801C0990007820F0D7
:1023C00080008030099908709DF8AC1001EB410045
:1023D000C0EBC110414901EBC0023F489DF8AC1071
:1023E00030F81100401E125C9DF8AC00C0EBC0013B
:1023F00001EB8011364800EB411060309DF89C10D5
:1024000001EB011100EBC10080F83C20BDF8D800C1
:10241000401C80B23690BDF8D8000021DDE92C3494
:10242000C01AA141FFF629AF00E000BF00BFB9E22A
:102430009DF8AC1001EB4100C0EBC110274901EB46
:10244000C000407D9DF8AC1001EB4102C2EBC11110
:10245000224A02EBC101897D40EA0120C217CDE981
:102460002C029DF8AC1001EB4100C0EBC1101B49E0
:1024700001EBC001099115210998F7F70FFA002225
:10248000CDE92E02DDE92E42DDE92C1061405040FD
:1024900001437DD19DF8AC1001EB4100C0EBC110B0
:1024A0000E4911F83000401EC1B2279100210C4A9C
:1024B0009DF8AC0002EB00129DF89C0011540A4AF2
:1024C0009DF89C0011549FED090A10EE101A0FE0C0
:1024D000FC3400203C3000207C5800202466002082
:1024E000702E0020BC2200204D280020000000009B
:1024F0000C329DF89C0002EB001041609DF8AC008E
:1025000000EB4001C1EBC010FE4901EBC000817936
:102510009DF8AC0000EB4002C2EBC010F94A02EBA0
:10252000C000407941EA002000EE100AB8EEC00A6F
:102530009FEDF51AC0EE010A9DF8AC0000EB4001DA
:10254000C1EBC010114601EBC00001799DF8AC0051
:1025500000EB4002C2EBC010EA4A02EBC000C078B8
:1025600041EA002000EE100AB8EEC00A30EE800A00
:1025700010EE101AE54A9DF89C0002EB0010016075
:102580009DF8AC0000EB4001C1EBC010DD4900E05C
:10259000F4E001EBC000817A9DF8AC0000EB400252
:1025A000C2EBC010D74A02EBC000407A41EA0020DB
:1025B00000EE100AB8EEC00A9FEDD31AC0EE010A71
:1025C0009DF8AC0000EB4001C1EBC010114601EBDF
:1025D000C000017A9DF8AC0000EB4002C2EBC010D5
:1025E000C84A02EBC000C07941EA002000EE100AA0
:1025F000B8EEC00A30EE800A10EE101AC34A9DF8F9
:102600009C0002EB001081609DF8AC1001EB4100D2
:10261000C0EBC110BB4901EBC000C07A00F08000E4
:1026200030BB9DF8AC1001EB4100C0EBC110B549C7
:1026300001EBC000017B9DF8AC0000EB4002C2EB57
:10264000C010B04A02EBC000C07A41EA002000EEA0
:10265000100AF8EEC00AB3EE001A80EE810A10EEFE
:10266000100AAA4A9DF89C1002EB0111C86046E0CE
:102670009DF8AC0000EB4001C1EBC010A14901EB9B
:10268000C000017B9DF8AC0000EB4002C2EBC01023
:102690009C4A02EBC000C07A41EA0020404280B26E
:1026A00000EE100AB8EEC00A8DED030A0398F6F7A3
:1026B00035F89FED970B53EC102BCDE904019DED00
:1026C000040B51EC100BF5F70DFF9FED930B53EC42
:1026D000102BCDE906019DED060B51EC100BF5F723
:1026E0008CFECDE908019DED080B51EC100BF6F7BF
:1026F00028F8864A9DF89C1002EB0111C8609DF8ED
:10270000AC1001EB410000EB0111854800EB01101A
:1027100030309DF89C1000EB0110801C099000786F
:1027200020F080018031099801709DF8AC1001EB18
:102730004100C0EBC110734901EBC000C27D9DF8A0
:10274000AC00C0EBC00101EB8011764800EB4111F9
:1027500060319DF89C0000EB001001EBC00080F898
:102760003C209DF8AC1001EB410000EB01116C48DE
:1027700000EB0110C1796C4880F8901512E19DF8CA
:10278000AC1001EB4100C0EBC1105E4901EBC00091
:10279000C0799DF8AC1001EB4102C2EBC111594A5E
:1027A00002EBC101097A40EA0120C217CDE92C02EF
:1027B0009DF8AC1001EB4100C0EBC110514901EB99
:1027C000C001099107210998F7F768F80022CDE9BF
:1027D0002E022DA819C82C995940604001437DD183
:1027E0009DF8AC1001EB4100C0EBC110454911F858
:1027F0003000401EC1B2279100214C4A9DF8AC0028
:1028000002EB00100170A2F223629DF89C001154AB
:102810009DF8AC1001EB4100C0EBC110394901EB50
:10282000C000817908460191F5F7F2FECDE9020179
:102830009DED021B9FED3E0B19F0B2FD8DED060BD9
:102840009DF8AC1001EB4100C0EBC1102D4901EB2C
:10285000C00001799DF8AC0000EB4002C2EBC01053
:10286000284A02EBC000C07841EA002000EE100ABE
:10287000B8EEC00A8DED030A0398F5F74FFFCDE9D6
:1028800004019DED060B53EC102B9DED040B51EC58
:10289000100BF5F727FECDE908019DED080B51EC73
:1028A000100BF5F74EFF194A9DF89C1002EB011131
:1028B00048601FEDF20A10EE100A9DF89C1002EB22
:1028C000011108601FEDF70A10EE100A9DF89C1028
:1028D00002EB011188601FEDFB0A00E061E010EEE1
:1028E000100A9DF89C1002EB0111C8609DF8AC1015
:1028F00001EB410000EB0111094800EB0110303001
:102900001AE000002466002000FF7F4759280020BD
:102910000000000000003040000000000000000047
:102920003C300020FC340020BC220020702E00200F
:1029300000000000000024409DF89C1000EB0110F6
:10294000801C0990007820F0800180310998017086
:102950009DF8AC1001EB4100C0EBC110FE4901EB4A
:10296000C000427A9DF8AC00C0EBC00101EB8011C1
:10297000FA4800EB411160319DF89C0000EB00101B
:1029800001EBC00080F83C209DF8AC1001EB410049
:1029900000EB0111F24800EB0110C179F14880F819
:1029A000901500BF00BF03F089BB9DF8AC1001EB90
:1029B0004100C0EBC110E84901EBC000C1789DF8AF
:1029C000AC0000EB4002C2EBC010E34A02EBC000D7
:1029D000807841EA002128919DF8AC1001EB41007C
:1029E000C0EBC110114601EBC001BDF8A000401CB6
:1029F000095C9DF8AC0000EB4002C2EBC010D64A67
:102A000002EBC002BDF8A000105C41EA0020C21732
:102A1000CDE92C029DF8AC1001EB4100C0EBC110D8
:102A2000CD4901EBC0000990BDF8A010F6F736FFC4
:102A30000022CDE92E022DA819C82C9959406040DA
:102A400001437DD19DF8AC1001EB4100C0EBC110FA
:102A5000C14901EBC00041782791002136911CE06B
:102A60009DF8AC1001EB410000EB0111BC4800EBFC
:102A700001113031BDF8D80001EB001041789DF80C
:102A80009C00814204D1BDF8D800C1B2279112E068
:102A9000BDF8D800401C81B236919DF8AC1001EB16
:102AA000410000EB0111AE4800EB0110C179BDF807
:102AB000D8008142D4DC00BF9DF8AC1001EB41008E
:102AC00000EB0111A64800EB011030309DF89C107E
:102AD00000EB0110801C0990007820F0800180310B
:102AE000099801709DF8AC1001EB4100C0EBC110DA
:102AF000994901EBC0000179259100219A4A9DF87E
:102B0000AC0002EB00129DF89C0011549DF8AC1033
:102B100001EB410000EB0111914800EB0111303154
:102B20009DF89C0001EB0010801C0990007820F0BB
:102B30004001403109980170BDF89400F32800E08D
:102B4000AFE37DD006DC05287BD0F12807D0F22842
:102B500078D180E2F42876D0F62873D1A1E29DF8EE
:102B6000AC10C1EBC10000EB81117C4800EB4110BF
:102B700060309DF89C1001EB011110F8310018BB7A
:102B800001229DF8AC00C0EBC00101EB801173483D
:102B900000EB411160319DF89C0000EB001001F842
:102BA0003020F4229DF8AC00C0EBC00101EB801195
:102BB0006A4800EB411060309DF89C1001EB011158
:102BC00000EBC1004271C2E09DF8AC1001EB410086
:102BD00000EB0111624800EB011030309DF89C10B1
:102BE00000EB0110407A00F0010068B39DF8AC10D2
:102BF000C1EBC10000EB8111584800EB411060307F
:102C00009DF89C1001EB011100EBC10090F88600CB
:102C100000F00100C0B99DF8AC10C1EBC10000EBA1
:102C200081114E4800EB411060309DF89C1001EB83
:102C3000011100EBC10090F8780028B1002004E0F9
:102C40001CE2BDE206E250E281E0369029E09DF808
:102C5000AC10C1EBC10000EB8111404800EB411109
:102C600060319DF89C0000EB001001EBC00000F10A
:102C70007901BDF8D8000A5C9DF8AC0000EB40017A
:102C800001EB0011364800EB01100E30BDF8D810F2
:102C9000405C824200D008E0BDF8D800401C81B200
:102CA0003691BDF8D8000428D1DB00BFBDF8D800AC
:102CB00004284CD1369029E09DF8AC10C1EBC1003E
:102CC00000EB8111254800EB411160319DF89C001B
:102CD00000EB001001EBC00000F17901BDF8D80055
:102CE0000A5C9DF8AC0000EB400101EB00111C48B0
:102CF00000EB01100E30BDF8D810405C824200D0CD
:102D000008E0BDF8D800401C81B23691BDF8D8006B
:102D10000A28D1DB00BFBDF8D8000A2817D09DF8DB
:102D2000AC10C1EBC10000EB81110C4800EB41106D
:102D300060309DF89C1001EB011100EBC100863062
:102D40000990007820F00100401C09990870BDF836
:102D5000A00011287CD109E024660020FC3400206A
:102D60003C300020BC220020702E00209DF8AC10CA
:102D700001EB410000EB0111F84800EB011030308D
:102D80009DF89C1000EB0110801C0990007820F049
:102D90000400001D099908700020369025E09DF878
:102DA000AC1001EB4100C0EBC110ED4901EBC001DB
:102DB000BDF8D800401D0A5C9DF8AC00C0EBC00116
:102DC00001EB8011E74800EB411160319DF89C0058
:102DD00000EB001001EBC0013F31BDF8D8000A54F0
:102DE000BDF8D800401C81B23691BDF8D8000A2841
:102DF000D5DB0021369125E09DF8AC1001EB4100B8
:102E0000C0EBC110D64901EBC001BDF8D8000F30AE
:102E10000A5C9DF8AC00C0EBC00101EB8011D14809
:102E200000EB411160319DF89C0000EB001001EBBC
:102E3000C0015831BDF8D8000A54BDF8D800401C74
:102E400081B23691BDF8D8000228D5DB02E1FFE758
:102E5000BDF8A00014287DD19DF8AC1001EB410015
:102E600000EB0111BD4800EB011030309DF89C10C3
:102E700000EB0110801C0990007820F00401091D6E
:102E8000099801700021369125E09DF8AC1001EB06
:102E90004100C0EBC110B24901EBC001BDF8D80040
:102EA000401D0A5C9DF8AC00C0EBC00101EB801135
:102EB000AC4800EB411160319DF89C0000EB001024
:102EC00001EBC0013F31BDF8D8000A54BDF8D8006D
:102ED000401C81B23691BDF8D8000A28D5DB00210C
:102EE000369125E09DF8AC1001EB4100C0EBC1101C
:102EF0009B4901EBC001BDF8D8000F300A5C9DF87A
:102F0000AC00C0EBC00101EB8011964800EB411111
:102F100060319DF89C0000EB001001EBC0015831BE
:102F2000BDF8D8000A54BDF8D800401C81B23691D3
:102F3000BDF8D8000228D5DB9DF8AC1001EB4100AC
:102F4000C0EBC110864901EBC001BDF8D8001130BB
:102F5000085C00E02FE001049DF8AC0000EB4002AB
:102F6000C2EBC0107E4A02EBC002BDF8D80012309E
:102F7000105C41EA00219DF8AC0000EB4002C2EB7E
:102F8000C010774A02EBC002BDF8D8001330105CC5
:102F900001439DF8AC00C0EBC00202EB8012714807
:102FA00000EB421060309DF89C2002EB021200EB17
:102FB000C200C1664EE09DF8AC1001EB410000EB91
:102FC0000111664800EB011030309DF89C1000EBB9
:102FD0000110801C0990007820F00402099802700A
:102FE0009DF8AC10C1EBC10000EB81115D4800EB16
:102FF000411060309DF89C1001EB011100EBC10005
:1030000090F8860000F0010020B300229DF8AC008B
:10301000C0EBC00101EB8011524800EB411160315F
:103020009DF89C0000EB001001EBC000A0F884208C
:1030300005229DF8AC00C0EBC00101EB80114948AE
:1030400000EB411060309DF89C1001EB011100EB8A
:10305000C100427124E1F1229DF8AC00C0EBC00137
:1030600001EB80113F4800EB411060309DF89C104F
:1030700001EB011100EBC100427111E1F1229DF859
:10308000AC00C0EBC00101EB8011364800EB4110F1
:1030900060309DF89C1001EB011100EBC100427102
:1030A000FEE003229DF8AC00C0EBC00101EB8011F3
:1030B0002C4800EB411160319DF89C0000EB0010A2
:1030C00001F83020F1229DF8AC00C0EBC00101EB0B
:1030D0008011244800EB411060309DF89C1001EBFA
:1030E000011100EBC1004271DAE002229DF8AC0050
:1030F000C0EBC00101EB80111A4800EB41116031B7
:103100009DF89C0000EB001001F83020F6229DF89D
:10311000AC00C0EBC00101EB8011124800EB411183
:1031200060319DF89C0000EB001001EBC000427183
:1031300001229DF8AC00C0EBC00101EB80110948F1
:1031400000EB411160319DF89C0000EB001001EB99
:10315000C00080F87820002136912CE03C3000201F
:1031600024660020FC3400209DF8AC0000EB4001F8
:10317000C1EBC010FE4901EBC001BDF8D800401DF5
:103180000A5C9DF8AC00C0EBC00101EB8011F9486E
:1031900000EB411160319DF89C0000EB001001EB49
:1031A000C00000F17901BDF8D8000A54BDF8D8007C
:1031B000401C81B23691BDF8D8000A28D4DB6FE0FC
:1031C0009DF8AC0000EB4001C1EBC010E84901EBF9
:1031D000C00081799DF8AC0000EB4002C2EBC0104A
:1031E000E34A02EBC000407941EA00229DF8AC00BE
:1031F000C0EBC00101EB8011DE4800EB41116031F2
:103200009DF89C0000EB001001EBC000A0F88420AA
:103210009DF8AC00C0EBC00101EB8011D54800EB7C
:10322000411160319DF89C0000EB001001EBC000E3
:10323000B0F884109DF8AC0000EB400202EB0012E5
:10324000CD4800EB0210408B814228DBF1229DF833
:10325000AC00C0EBC00101EB8011C64800EB41118E
:1032600060319DF89C0000EB001001EBC000427142
:103270009DF8AC00C0EBC00101EB8011BD4800EB34
:10328000411060309DF89C1001EB011100EBC10072
:1032900086300990007820F001020998027000BF82
:1032A00000BF02F00BBF9DF8AC0000EB4001C1EB8A
:1032B000C010AF4901EBC000017927910021349182
:1032C0001CE09DF8AC0000EB400101EB0011AA48A6
:1032D00000EB01113031BDF8D00001EB0010417856
:1032E0009DF89C00814204D1BDF8D000C1B2279165
:1032F00012E0BDF8D000401C81B234919DF8AC00C2
:1033000000EB400101EB00119B4800EB0110C1797B
:10331000BDF8D0008142D4DC00BF9DF8AC0000EBCA
:10332000400101EB0011944800EB011030309DF892
:103330009C1000EB0110801C0990007820F04001E7
:103340004031099801709DF8AC0000EB4001C1EBE1
:10335000C010874901EBC000C1782591BDF89400E9
:10336000172834D2DFE800F0330C0F331215181B86
:103370001E33333333333321242733332A2D3000A4
:103380000720289023E00720289020E0062028909E
:103390001DE0062028901AE00620289017E0122150
:1033A000289114E00720289011E0092028900EE0D1
:1033B000062028900BE00620289008E00B2028909B
:1033C00005E00B20289002E02A21289100BF00BFD1
:1033D000BDF8A000001FC1B209919DF8AC0000EB40
:1033E0004001C1EBC010624901EBC000C01C089055
:1033F0000999F6F76FF835909DF8AC0000EB4001A5
:10340000C1EBC0105A4901EBC001BDF8A000401E3D
:10341000095CBDF8D40081427DD19DF8AC0000EB81
:103420004001C1EBC010524901EBC00040780028B8
:1034300071DD9DF8AC0000EB4001C1EBC0104C49C0
:1034400001EBC001BDF8A0000A5C9DF8AC00C0EB28
:10345000C00101EB8011474800EB411160319DF83C
:103460009C0000EB001001EBC00080F83C20002124
:10347000424A9DF8AC0002EB00129DF89C001154EA
:103480003F48007F012815D19DF8AC0000EB4001BA
:1034900001EB0011384800EB011030309DF89C1012
:1034A00000EB0110801C0990007820F08000803033
:1034B00009990870BDF89400072858D007DC072840
:1034C0007ED2DFE800F07DFDFC7DFBFAF9001038CC
:1034D0000728F5D2DFE810F07B0968097400740052
:1034E000070008005E0500BFBDF89400142868D1ED
:1034F0009DF8AC0000EB4001C1EBC0101C4901EB92
:10350000C000407901069DF8AC0000EB4002C2EB20
:10351000C010174A00E0FCE302EBC000807941EAEA
:1035200000419DF8AC0000EB4002C2EBC010104A15
:1035300002EBC000C07941EA00219DF8AC0000EB2D
:103540004002C2EBC0100A4A02EBC000007A0143FD
:103550009DF8AC00C0EBC00202EB8012054800EB06
:10356000421260329DF89C0000EB00100AE0FBE381
:1035700024660020FC3400203C300020702E002007
:10358000BC12002002EBC000C0F81A109DF8AC007D
:10359000C0EBC00101EB8011FE4800EB411160312E
:1035A0009DF89C0000EB001001EBC000D0F81A1051
:1035B00008460991002109F0F1FBCDE92C0101E059
:1035C000FEE387E09DF8AC0000EB400101EB001149
:1035D000F14800EB0110007F00F003019DF8AC0002
:1035E00000EB400202EB0012EB4800EB0210007F00
:1035F000C0F3011001449DF8AC0000EB400202EB67
:103600000012E54800EB0210007FC0F38100091AA8
:1036100008460591F4F7EBFFCDE906019DED061B89
:103620009FEDDE0B18F0BCFE8DED080B9DED080B39
:1036300051EC100BF5F74DF8CDE92E019DF8AC00DB
:10364000C0EBC00101EB8011D24800EB41116031A9
:103650009DF89C0000EB001001EBC000416B084698
:103660000791002109F09AFBDDE92C32A0FB03450C
:1036700001FB035100FB021502220023DDE92E01AC
:10368000F4F7A0FD20186941CDE90801DDE92E23FA
:10369000F4F798FDCDE92C01DDE92C010AF032F9AF
:1036A00001469DF8AC00C0EBC00202EB8012B948A5
:1036B00000EB4210603004E0FEE397E3CAE3FCE372
:1036C000DBE39DF89C2002EB021200EBC200C0F885
:1036D0001E1043E0BDF8940015283FD19DF8AC00C2
:1036E00000EB4001C1EBC010AE4901EBC0004079D6
:1036F00001069DF8AC0000EB4002C2EBC010A94AE5
:1037000002EBC000807941EA00419DF8AC0000EB7B
:103710004002C2EBC010A34A02EBC000C07941EAEC
:1037200000219DF8AC0000EB4002C2EBC0109D4AA6
:1037300002EBC000007A01439DF8AC00C0EBC00270
:1037400002EB8012934800EB421060309DF89C2001
:1037500002EB021200EBC200C0F81E109DF8AC0094
:1037600000EB4001C1EBC0108E4901EBC000417A73
:103770008D4880F8E7119DF8AC0000EB400101EBAB
:103780000011854800EB011030309DF89C1000EBD3
:103790000110801C0990844890F8E701C20909983B
:1037A000007862F30000099908707F4890F8E701FB
:1037B00000F00300012806D07B4890F8E70100F0F4
:1037C000030003282BD19DF8AC0000EB400101EB76
:1037D0000011714800EB011030309DF89C1000EB97
:1037E0000110801C0990007820F00200801C0999CB
:1037F00008709DF8AC0000EB400101EB0011664839
:1038000000EB011030309DF89C1000EB0110801C83
:103810000990007820F020020998027014E09DF8C9
:10382000AC0000EB400101EB00115B4800EB011024
:1038300030309DF89C1000EB0110801C099000783E
:1038400020F00202099802709DF8AC0000EB4001E4
:1038500001EB0011504800EB011130319DF89C0044
:1038600001EB00108078C0F340029DF8AC10C1EB72
:10387000C10000EB8111474800EB411160319DF818
:103880009C0000EB001001EBC000007EC0F3400084
:10389000824265D09DF8AC00C0EBC00101EB801105
:1038A0003C4800EB411060309DF89C1001EB011189
:1038B00000EBC100183009909DF8AC0000EB40010E
:1038C00001EB0011344800EB011130319DF89C00F0
:1038D00001EB0010807842080998017862F34101F9
:1038E00001709DF8AC0000EB400101EB00112A488B
:1038F00000EB011030309DF89C1000EB0110807837
:10390000C0F3400038BB9DF8AC0000EB400101EB78
:103910000011214800EB011030309DF89C1000EBA5
:103920000110801C0990007820F020020998027094
:1039300001229DF8AC00C0EBC00101EB80111548DD
:1039400000EB411060309DF89C1001EB011100EB81
:10395000C10080F83E209DF8AC100220F6F7F8FA7E
:103960009DF8AC0000EB400101EB00110A4800EBB0
:10397000011130319DF89C0001EB0010807800F0BF
:1039800001029DF8AC00C0EBC00101EB80110148C1
:103990000CE00000FC3400203C300020000000005F
:1039A0000000244024660020BC22002000EB4110CF
:1039B00060309DF89C1001EB011100EBC100007E0E
:1039C00000F0010082425FD09DF8AC00C0EBC00166
:1039D00001EB8011FE4800EB411060309DF89C1017
:1039E00001EB011100EBC100183009909DF8AC000B
:1039F00000EB400101EB0011F64800EB0111303102
:103A00009DF89C0001EB001082780998017862F320
:103A1000000101709DF8AC0000EB400101EB0011CA
:103A2000EC4800EB011030309DF89C1000EB0110C9
:103A3000807800F0010040BB9DF8AC0000EB400135
:103A400001EB0011E34800EB011030309DF89C10B1
:103A500000EB0110801C0990007820F020020998EA
:103A6000027000229DF8AC00C0EBC00101EB801198
:103A7000D74800EB411060309DF89C1001EB01111C
:103A800000EBC10080F83D2007E19DF8AC00C0EBE1
:103A9000C00101EB8011CE4800EB411060309DF871
:103AA0009C1001EB011100EBC10090F83E0098B9A9
:103AB00001229DF8AC00C0EBC00101EB8011C448AD
:103AC00000EB411060309DF89C1001EB011100EB00
:103AD000C10080F83D2027E000229DF8AC00C0EB3B
:103AE000C00101EB8011BA4800EB411160319DF833
:103AF0009C0000EB001001EBC00080F83D209DF819
:103B0000AC0000EB400101EB0011B24800EB0110EA
:103B100030309DF89C1000EB0110801C099000785B
:103B200020F0010209980270AB4890F8C807E8BB82
:103B3000AA48407F012839D1A848C06DA749C98B40
:103B4000884233D29DF8AC00C0EBC00101EB80117C
:103B50009F4800EB411060309DF89C1001EB011173
:103B600000EBC10090F83D0001281FD19DF8AC008A
:103B7000C0EBC00101EB8011954800EB41106030B3
:103B80009DF89C1001EB011100EBC10090F877004B
:103B900060B99DF8AC0000EB400101EB00118D48CD
:103BA00000EB011130319DF89C0000E075E001EB65
:103BB000001001789DF8AC00C0EBC00202EB80124F
:103BC000834800EB4210417005229DF8AC00C0EB29
:103BD000C00101EB80117E4800EB411160319DF87E
:103BE0009C0000EB001001EBC000427100229DF828
:103BF000AC0000EB400101EB0011764800EB011135
:103C000030319DF89C0001EB001042609DF8AC1033
:103C10000220F6F79DF90021369119E000229DF867
:103C2000AC00C0EBC00101EB8011694800EB411111
:103C300060319DF89C0000EB001001EBC0013F31AA
:103C4000BDF8D8000A54BDF8D800401C81B23691A6
:103C5000BDF8D8001428E1DB0020369019E00022DE
:103C60009DF8AC00C0EBC00101EB8011584800EB9F
:103C7000411160319DF89C0000EB001001EBC00188
:103C80005B31BDF8D8000A54BDF8D800401C81B2A1
:103C90003691BDF8D8000A28E1DB9DF8AC00C0EBF6
:103CA000C00101EB80114A4800EB411060309DF8E3
:103CB0009C1001EB011110F83100012811DC0222E7
:103CC0009DF8AC00C0EBC00101EB8011404800EB57
:103CD000411060309DF89C1001EB011100F831207B
:103CE00083E09DF8AC00C0EBC00101EB80113848C7
:103CF00000EB411060309DF89C1001EB011110F8B1
:103D00003100022831DC00219DF8AC00C0EBC0027C
:103D100000E0FCE302EB80122D4800EB4210C17082
:103D200003229DF8AC00C0EBC00101EB80112848D4
:103D300000EB411160319DF89C0000EB001001F890
:103D4000302007229DF8AC00C0EBC00101EB8011D0
:103D50001F4800EB411060309DF89C1001EB0111F1
:103D600000EBC100427140E0E4E19DF8AC00C0EB23
:103D7000C00101EB8011164800EB411160319DF844
:103D80009C0000EB001011F830109DF8AC00C0EB67
:103D9000C00202EB80120E4800EB42100079814213
:103DA00023D10D4890F8E701C0F34010E8B1162286
:103DB0009DF8AC00C0EBC00101EB8011044800E0AD
:103DC000FEE300EB411060309DF89C1008E000001D
:103DD000FC3400203C300020BC220020BC1200201B
:103DE00001EB011100EBC1004271E9E314229DF8DF
:103DF000AC00C0EBC00101EB8011FE4800EB4111AB
:103E000060319DF89C0000EB001001EBC000427196
:103E100001219DF8AC00C0EBC00202EB8012F54816
:103E200000EB4210C1709DF8AC0000EB400101EBCB
:103E30000011F14800EB011130319DF89C0001EBBD
:103E40000010801C0990007820F020002030099993
:103E50000870B5E314229DF8AC00C0EBC00101EB83
:103E60008011E44800EB411160319DF89C0000EBAB
:103E7000001001EBC0004271A2E39DF8AC00C0EB62
:103E8000C00101EB8011DB4800EB41106030BDF850
:103E9000D01001EB011100EBC1008079012827D17E
:103EA00000229DF8AC00C0EBC00101EB8011D148AD
:103EB00000EB4111603101E0FDE337E0BDF8D000D7
:103EC00000EB001001EBC000827114229DF8AC00E1
:103ED000C0EBC00101EB8011C64800EB411060301F
:103EE0009DF89C1001EB011100EBC10042711CE038
:103EF00000219DF8AC00C0EBC00202EB8012BD486F
:103F000000EB4210C17005229DF8AC00C0EBC0016F
:103F100001EB8011B74800EB411060309DF89C1018
:103F200001EB011100EBC100427149E301219DF851
:103F3000AC00C0EBC00202EB8012AE4800EB4210B6
:103F4000C17014229DF8AC00C0EBC00101EB8011E0
:103F5000A84800EB411160319DF89C0000EB001077
:103F600001EBC00042719DF8AC0000EB400101EB99
:103F70000011A14800EB011130319DF89C0001EBCC
:103F80000010801C0990007820F00400001D0999A1
:103F9000087015E300202C902D90002136911FE031
:103FA000DDE92C10000240EA11620902CDE92C1271
:103FB0009DF8AC0000EB4001C1EBC0108F4901EB54
:103FC000C001BDF8D800401D085CDDE92C3440EA92
:103FD0000302CDE92C24BDF8D800401C81B23691F3
:103FE000BDF8D8000328DBDBDDE92C0109F08AFCF1
:103FF00001469DF8AC00C0EBC00202EB80127D4888
:1040000000EB421260329DF89C0000EB001002EBC6
:10401000C000C0F81E1000222C922D920021369173
:104020001EE0DDE92C10000240EA11620902CDE930
:104030002C129DF8AC0000EB4001C1EBC0106F49A1
:1040400001EBC001BDF8D8000830085CDDE92C3474
:104050001843CDE92C04BDF8D800401C80B236903E
:10406000BDF8D8000328DCDBDDE92C0109F04AFCAF
:1040700001469DF8AC00C0EBC00202EB80125D4827
:1040800000EB421260329DF89C0000EB001002EB46
:10409000C000C0F81A1000222C922D9200213691F7
:1040A0001FE0DDE92C10000240EA11620902CDE9AF
:1040B0002C129DF8AC0000EB4001C1EBC0104F4941
:1040C00001EBC001BDF8D8001330085CDDE92C34E9
:1040D00040EA0302CDE92C24BDF8D800401C81B28F
:1040E0003691BDF8D8000328DBDB9DF8AC002C9995
:1040F000C0EBC00202EB80123E4800EB421260327D
:104100009DF89C0000EB001002EBC0004163072209
:104110009DF8AC00C0EBC00101EB8011354800EB0D
:10412000411160319DF89C0000EB001001EBC000D4
:1041300042715FE300202C902D90002136911EE00B
:10414000DDE92C10000240EA11620902CDE92C12CF
:104150009DF8AC0000EB4001C1EBC010274901EB1A
:10416000C001BDF8D800401D085CDDE92C341843BF
:10417000CDE92C04BDF8D800401C80B23690BDF8C3
:10418000D8000428DCDBDDE92C0109F0BBFB9DF83D
:10419000AC20C2EBC20303EB8213164A02EB4313BB
:1041A00060339DF89C2002EB021203EBC202223224
:1041B0009060D16000212C912D910020369026E056
:1041C000DDE92C10000240EA11620902CDE92C124F
:1041D0009DF8AC0000EB4001C1EBC010074901EBBA
:1041E000C001BDF8D8000930085CDDE92C34184363
:1041F00006E00000FC3400203C3000202466002053
:10420000CDE92C04BDF8D800401C80B23690BDF832
:10421000D8000428D4DBDDE92C0109F073FB9DF8FC
:10422000AC20C2EBC20303EB8213FE4A02EB431342
:1042300060339DF89C2002EB021203EBC20242F8AD
:10424000220F51609DF8AC00C0EBC00101EB801162
:10425000F44800EB411160319DF89C0000EB001028
:1042600011F830109DF8AC00C0EBC00202EB8012D8
:10427000EC4800EB4210007981426DD1EA4890F899
:10428000E701C0F3401090B117229DF8AC00C0EBDD
:10429000C00101EB8011E34800EB411060309DF854
:1042A0009C1001EB011100EBC100427111E01422DE
:1042B0009DF8AC00C0EBC00101EB8011D94800EBC8
:1042C000411060309DF89C1001EB011100EBC10022
:1042D0004271D54890F8C807E8BB00229DF8AC00B1
:1042E000C0EBC00101EB8011CE4800EB4111603101
:1042F0009DF89C0000EB001001EBC00080F83E2010
:104300000021CA48C0F83D109DF8AC00C0EBC001C8
:1043100001EB8011C34800EB411160319DF89C0016
:1043200000EB001001EBC000223010220146099082
:10433000BE482D30F3F789FF9DF8AC00C0EBC001FB
:1043400001EB8011B74800EB411060309DF89C10E4
:1043500001EB011101E066E04AE100EBC101B34865
:10436000401C51F81A2F0262496841629DF8AC0066
:1043700000EB400101EB0011AD4800EB01103030C3
:104380009DF89C1000EB01100078A84981F82000EE
:104390009DF8AC00C0EBC00101EB8011A14800EB1F
:1043A000411160319DF89C0000EB001001EBC00052
:1043B000416B9E48C0F8291021309E490A6F026265
:1043C000B1F8741081842138C06D81B20220099146
:1043D000F4F77EFE00210620F5F7BAFD9348C06D84
:1043E0009249C98B884204D29048C06D401C8F49C5
:1043F000C86500210520F5F7ABFD9DF8AC0000EB8A
:10440000400101EB00118A4800EB011030309DF8AB
:104410009C1000EB0110801C0990007820F008022D
:104420000998027028E09DF8AC0000EB400101EB18
:1044300000117F4800EB011030309DF89C1000EB1C
:104440000110801C0990007820F0080108310998BB
:10445000017000229DF8AC00C0EBC00101EB80119F
:10446000704800EB411060309DF89C1001EB011189
:1044700000EBC10080F83E209DF8AC100220F5F75B
:1044800067FD9DF8AC109DF89C0000EB0110C21771
:10449000CDE92C0200222C9800EB8001C1EB8011A9
:1044A000624864300844C0F81D209DF8AC00C0EBA1
:1044B000C00101EB80115B4800EB411060309DF8BA
:1044C0009C1001EB011100EBC100223009902C98E7
:1044D00000EB8001C1EB80115448643008440D307A
:1044E000102208900999F3F7B0FE9DF8AC00C0EBDC
:1044F000C00101EB80114B4800EB411160319DF888
:104500009C0000EB001001EBC0012C9800E072E170
:1045100000EB8002C2EB801244486430104451F832
:104520001A2F40F8012F496841609DF8AC0000EB5C
:10453000400101EB00113E4800EB011130319DF8C4
:104540009C0001EB001001782C9800EB8002C2EB7C
:1045500080123648643081542C9800EB8001C1EB06
:1045600080113248643001443248026F41F8212FF3
:10457000B0F8740088809DF8AC00C0EBC00101EB7E
:104580008011284800EB411160319DF89C0000EB40
:10459000001001EBC000416B2C9800EB8002C2EBD5
:1045A0008012224864301044C0F809109DF8AC0015
:1045B00000EB400101EB00111D4800EB011100E090
:1045C00018E130319DF89C0001EB001041682C98F7
:1045D00000EB8002C2EB8012144864301044C0F833
:1045E00027102C9881B208200991F5F7B1FC8BE0D7
:1045F0009DF8AC00C0EBC00101EB8011094800EB55
:10460000411160319DF89C0000EB001011F8301052
:104610009DF8AC00C0EBC00202EB8012014800EB39
:10462000421009E0FC340020BC220020BC12002013
:104630003C3000203C2600200079814264DA9DF85D
:10464000AC0000EB400101EB0011FE4800EB011053
:1046500030309DF89C1000EB0110801C0990007810
:1046600020F00401091D099801709DF8AC0000EBD1
:10467000400101EB0011F34800EB011130319DF8CE
:104680009C0001EB0010801C0990007820F0800154
:1046900080310998017001219DF8AC00C0EBC00287
:1046A00002EB8012E84800EB4210C1709DF8AC00AC
:1046B000C0EBC00100E028E001EB8011E24800EB14
:1046C000411002799DF8AC00C0EBC00101EB8011F4
:1046D000DD4800EB411160319DF89C0000EB0010BB
:1046E00001F8302014229DF8AC00C0EBC00101EBB2
:1046F0008011D54800EB411160319DF89C0000EB22
:10470000001001EBC000427174E00121CF4880F835
:10471000EC169DF8AC00C0EBC00101EB8011CA485B
:1047200000EB411160319DF89C0000EB001011F886
:1047300030109DF8AC00C0EBC00202EB8012C24802
:1047400000EB4210007981422DDA00219DF8AC0087
:10475000C0EBC00202EB8012BB4800EB4210C170FC
:1047600001229DF8AC00C0EBC00101EB8011B648FE
:1047700000EB411160319DF89C0000EB001001F846
:10478000302014229DF8AC00C0EBC00101EB801179
:10479000AD4800EB411060309DF89C1001EB011119
:1047A00000EBC100427125E014229DF8AC00C0EB83
:1047B000C00101EB8011A44800EB411060309DF86E
:1047C0009C1001EB011100EBC100427112E01422B8
:1047D0009DF8AC00C0EBC00101EB80119A4800EBE2
:1047E000411060309DF89C1001EB011100EBC100FD
:1047F000427100BF00BFFCE39DF8AC00C0EBC001FC
:1048000001EB8011904800EB4110817827919DF8D1
:10481000AC0000EB4001C1EBC0108D4911F8301025
:1048200028919DF8AC00C0EBC00101EB80118648D7
:1048300000EB411160319DF89C0000EB001001EB92
:10484000C000417925919DF8AC0000EB4001C1EB1F
:10485000C0107F4901EBC0010991BDF8A010099873
:10486000F6F7F6F835909DF8AC0000EB4001C1EB8F
:10487000C010774901EBC001BDF8A000095CBDF88C
:10488000D40081427ED19DF8AC0000EB4001C1EB29
:10489000C0106F4901EBC0004078002872DD002194
:1048A0006C4A9DF8AC0002EB00129DF89C0011547C
:1048B000BDF89400892866D00CDC14287DD004DC77
:1048C00008287BD010287AD1FDE3152878D08028DD
:1048D000F9D1F9E38B2874D08C2873D08E2872D04C
:1048E0008F28F0D1BDF8A0000D286DD19DF8AC0047
:1048F00000EB4001C1EBC010554901EBC00041780D
:10490000524880F8E9119DF8AC0000EB4001C1EB82
:10491000C0104F4901EBC000C17A4C4880F8EA1141
:104920009DF8AC00C0EBC00101EB8011464800EBE4
:10493000411060309DF89C1001EB011110F831001E
:1049400003287DDC414890F8EA01002879DD9DF8D4
:10495000AC00C0EBC00101EB80113B4800EB411102
:1049600060319DF89C0000EB001001EBC001099143
:104970000878401CC1B2099801709DF8AC00C0EBEA
:10498000C00101E0FEE3FEE301EB80112E4800EBE5
:10499000411060309DF89C1001EB011110F83100BE
:1049A00004284EDB9DF8AC0000EB400101EB001148
:1049B000244800EB0110303007E0FCE3FCE3FCE3AB
:1049C000FCE3FCE3FCE3FCE3FCE39DF89C1000EB60
:1049D0000110801C09901D4890F8EA01C0F30010F6
:1049E000C0F101000999097860F30001099801708C
:1049F000164890F8E901C0F3C00068BB9DF8AC0010
:104A000000EB400101EB00110E4800EB01103030CB
:104A10009DF89C1000EB01108078C0F34010D8B1D5
:104A20009DF8AC0000EB400101EB0011054800EBE4
:104A3000011030309DF89C1000EB0110801C0CE040
:104A40005EE0F7E03C300020FC340020BC22002077
:104A500024660020702E002023E00990007820F0CA
:104A60000200801C099908709DF8AC00C0EBC001E1
:104A700001EB8011FE4800EB411060309DF89C1066
:104A800001EB011100EBC10018300990007820F013
:104A90000200801C099908709DF8AC100220F5F7FF
:104AA00057FA00219DF8AC00C0EBC00202EB801267
:104AB000EF4800EB4210C17004229DF8AC00C0EB3F
:104AC000C00101EB8011EA4800EB411160319DF813
:104AD0009C0000EB001001F830208C229DF8AC0007
:104AE000C0EBC00101EB8011E14800EB41106030E8
:104AF0009DF89C1001EB011100EBC1004271A4E391
:104B00009DF8AC00C0EBC00101EB8011D84800EB70
:104B1000411160319DF89C0000EB001011F830103D
:104B20009DF8AC00C0EBC00202EB8012D04800EB55
:104B30004210007981427DD19DF8AC0000EB40012C
:104B400001EB0011CB4800EB011030309DF89C10B8
:104B500000EB0110801C0990C74890F8EA01C0F3EF
:104B60000010C0F1010009990A7860F300020A7090
:104B70009DF8AC0000EB400101EB0011BD4800EBDB
:104B8000011030309DF89C1000EB0110801C099042
:104B9000B94890F8E901C2080998007862F3410029
:104BA000099908709DF8AC0000EB400101EB001181
:104BB000B04800EB011030309DF89C1000EB011064
:104BC0008078C0F340029DF8AC00C0EBC00101EB5F
:104BD0008011A74800EB411060309DF89C1001EB5C
:104BE000011100EBC100007EC0F34000824264D09E
:104BF0009DF8AC00C0EBC00101EB80119C4800EBBC
:104C0000411060309DF89C1001EB011100EBC100D8
:104C1000183009909DF8AC0000EB400101EB001149
:104C2000944800EB011030309DF89C1000EB01100F
:104C3000807800E0BEE242080998007862F3410003
:104C4000099908709DF8AC0000EB400101EB0011E0
:104C5000884800EB011030309DF89C1000EB0110EB
:104C60008078C0F3400018BB01229DF8AC00C0EB77
:104C7000C00101EB80117E4800EB411160319DF8CD
:104C80009C0000EB001001EBC00042739DF8AC00EB
:104C9000C0EBC00101EB8011754800EB41106030A2
:104CA0009DF89C1001EB011100EBC10080F83E2043
:104CB0009DF8AC100220F5F74BF99DF8AC0000EB25
:104CC000400101EB00116B4800EB011130319DF800
:104CD0009C0001EB0010807800F001029DF8AC0010
:104CE000C0EBC00101EB8011614800EB4111603164
:104CF0009DF89C0000EB001001EBC000007E00F06E
:104D00000100824277D09DF8AC00C0EBC00101EBFE
:104D10008011574800EB411060309DF89C1001EB6A
:104D2000011100EBC100183009909DF8AC0000EBB8
:104D3000400101EB00114F4800EB011130319DF8AB
:104D40009C0001EB001081780998027861F3000261
:104D500002709DF8AC0000EB400101EB00114548EA
:104D600000EB011030309DF89C1000EB01108078B2
:104D700000F00100F0BB9DF8AC0000EB400101EB3E
:104D800000113C4800EB011030309DF89C1000EB06
:104D900001108078C0F3401070B39DF8AC00C0EBF8
:104DA000C00101EB8011324800EB411060309DF8EA
:104DB0009C1001EB011100EBC10090F83E00D8B946
:104DC0009DF8AC00C0EBC00101EB8011284800EB5E
:104DD000411060309DF89C1001EB011100EBC10007
:104DE000407B48B99DF8AC0000EB400101EB00119D
:104DF000204802E04BE06DE12EE000EB0110303086
:104E00009DF89C1000EB01108078C0F3400018BBA7
:104E100001229DF8AC00C0EBC00101EB80111448E9
:104E200000EB411160319DF89C0000EB001001EB9C
:104E3000C00042739DF8AC00C0EBC00101EB8011D3
:104E40000B4800EB411160319DF89C0000EB001015
:104E500001EBC00080F83E2000229DF8AC00C0EBC2
:104E6000C00101EB8011024800EB4110603005E009
:104E7000FC3400203C300020BC2200209DF89C1017
:104E800001EB011100EBC10080F83D201AE19DF813
:104E9000AC00C0EBC00101EB8011FE4800EB4110FB
:104EA00060309DF89C1001EB011100EBC10090F8FF
:104EB0003E0098B901229DF8AC00C0EBC00101EBA7
:104EC0008011F44800EB411060309DF89C1001EB1C
:104ED000011100EBC10080F83D2027E000229DF881
:104EE000AC00C0EBC00101EB8011EA4800EB4111BE
:104EF00060319DF89C0000EB001001EBC00080F8D1
:104F00003D209DF8AC0000EB400101EB0011E248B0
:104F100000EB011130319DF89C0001EB0010801C6A
:104F20000990007820F0010209980270DB4890F89F
:104F3000C80780B19DF8AC0000EB400101EB001107
:104F4000D54800EB011030309DF89C1000EB0110AB
:104F5000807A02286ED1D248407F01286AD1D04899
:104F6000C06DCF49C98B884264D29DF8AC00C0EBBC
:104F7000C00101EB8011C74800EB411060309DF883
:104F80009C1001EB011100EBC10090F83D000128DD
:104F900050D19DF8AC00C0EBC00101EB8011BD48C1
:104FA00000EB411060309DF89C1001EB011100EB0B
:104FB000C10090F87700E8BB9DF8AC0000EB400121
:104FC00001EB0011B44800EB011130319DF89C0059
:104FD00001EB001001789DF8AC00C0EBC00202EBC1
:104FE0008012AC4800EB4210417008229DF8AC00E2
:104FF00000E0FDE3C0EBC00101EB8011A54800EB30
:10500000411160319DF89C0000EB001001EBC000E5
:10501000427100229DF8AC0000EB400101EB001151
:105020009D4800EB011130319DF89C0001EB001010
:10503000426000E046E09DF8AC100220F4F788FFE3
:105040000021369119E000229DF8AC00C0EBC001B0
:1050500001EB80118F4800EB411160319DF89C00FD
:1050600000EB001001EBC0013F31BDF8D8000A543D
:10507000BDF8D800401C81B23691BDF8D800142884
:10508000E1DB0021369119E000229DF8AC00C0EB75
:10509000C00101EB80117F4800EB411160319DF8A8
:1050A0009C0000EB001001EBC0015B31BDF8D800A3
:1050B0000A54BDF8D800401C81B23691BDF8D80022
:1050C0000A28E1DB01E0F9E1C2E39DF8AC1002201F
:1050D000F4F73EFF9DF8AC00C0EBC00101EB80117E
:1050E0006C4800EB411060309DF89C1001EB011101
:1050F00000EBC1008078802835D19DF8AC0000EB32
:10510000400101EB0011644800EB011030309DF8C4
:105110009C1000EB01108078C0F3400018BB9DF894
:10512000AC0000EB400101EB00115B4800EB01100B
:1051300030309DF89C1000EB01108078C0F34010D7
:1051400088B915229DF8AC00C0EBC00101EB8011BD
:10515000504800EB411060309DF89C1001EB0111AC
:1051600000EBC10042719DF8AC0000EB400101EB87
:105170000011494800EB011030309DF89C1000EB05
:10518000011001E0E7E3B0E18078C0F34000D0B166
:105190008F229DF8AC00C0EBC00101EB80113D48AF
:1051A00000EB411060309DF89C1001EB011100EB09
:1051B000C100427149E0FCE35EE149E2FAE3EEE15D
:1051C00047E279E357E19DF8AC00C0EBC00101EB89
:1051D0008011304800EB411060309DF89C1001EBCD
:1051E000011100EBC100807B01282ED100229DF827
:1051F000AC00C0EBC00101EB8011264800EB41116F
:1052000060319DF89C0000EB001001EBC000827340
:105210008C229DF8AC00C0EBC00101EB80111D4851
:1052200000EB411160319DF89C0000EB001001EB98
:10523000C000427100219DF8AC00C0EBC00202EB3F
:105240008012144800EB4210C1709DF8AC0000EBD6
:10525000400101EB0011104800EB0110007BE8BB9E
:105260009DF8AC0000EB4001C1EBC0100D4901EB13
:10527000C000807801049DF8AC0000EB4002C2EB56
:10528000C010084A02EBC000C07841EA00219DF836
:10529000AC0009E0FC3400203C300020BC2200209F
:1052A000BC1200202466002000EB4002C2EBC010BC
:1052B000FE4A02EBC00000790843C117CDE908019E
:1052C00008F020FB01469DF8AC00C0EBC00202EBE9
:1052D0008012F74800EB4212603200E041E09DF896
:1052E0009C0000EB001002EBC000C0F81E109DF8FF
:1052F000AC0000EB4001C1EBC010EC4901EBC00079
:10530000407901049DF8AC0000EB4002C2EBC010F4
:10531000E64A02EBC000807941EA00219DF8AC002A
:1053200000EB4002C2EBC010E04A02EBC000C079C3
:105330000843C117CDE9080108F0E4FA9DF8AC1064
:10534000C1EBC10202EB8112D94901EB421160317C
:105350009DF89C2002EB021201EBC201C1F81A0079
:1053600089E09DF8AC0000EB4001C1EBC010CF49D3
:1053700001EBC000807801069DF8AC0000EB400214
:10538000C2EBC010C94A02EBC000C07841EA00413C
:105390009DF8AC0000EB4002C2EBC010C34A02EB28
:1053A000C000007941EA00219DF8AC0000EB40020A
:1053B000C2EBC010BD4A02EBC00040790843C117E0
:1053C000CDE9080108F09EFA9DF8AC10C1EBC102CE
:1053D00002EB8112B64901EB421260329DF89C103B
:1053E00001EB011102EBC101C1F81E009DF8AC00F8
:1053F00000EB4001C1EBC010AC4901EBC00080796B
:1054000000069DF8AC1001EB4102C2EBC111A74AA6
:1054100002EBC101C97940EA01409DF8AC1001EBF3
:105420004102C2EBC111A14A02EBC101097A40EA73
:1054300001209DF8AC1001EB4102C2EBC1119B4A67
:1054400002EBC101497A0843C117CDE9080108F010
:1054500059FA9DF8AC10C1EBC10202EB81129449DC
:1054600001EB421160319DF89C2002EB021201EB2E
:10547000C201C1F81A00EBE0BDF8A00003281CD15E
:105480008F229DF8AC00C0EBC00101EB8011884871
:1054900000EB411160319DF89C0000EB001001EB26
:1054A000C000427101219DF8AC00C0EBC00202EBCC
:1054B00080127F4800EB4210C170C9E0BDF8A00027
:1054C000032811D18F229DF8AC00C0EBC00101EB85
:1054D0008011774800EB411060309DF89C1001EB83
:1054E000011100EBC1004271B2E0BDF8A000032839
:1054F00054D19DF8AC00C0EBC00101EB80116C48A9
:1055000000EB41106030BDF8D01001EB011100EB51
:10551000C1008079012824D100229DF8AC00C0EBA5
:10552000C00101EB8011624800EB41116031BDF810
:10553000D00000EB001001EBC00082718F229DF8BB
:10554000AC00C0EBC00101EB8011594800EB4110E9
:1055500060309DF89C1001EB011100EBC10042711D
:105560001CE008229DF8AC00C0EBC00101EB8011EB
:105570004F4800EB411160319DF89C0000EB00109A
:1055800001EBC000427100219DF8AC00C0EBC002ED
:1055900002EB8012464800EB4210C17058E0BDF8A3
:1055A000A000032854D19DF8AC00C0EBC00101EB72
:1055B00080113F4800EB41106030BDF8D01001EB86
:1055C000011100EBC1008079012824D100229DF84F
:1055D000AC00C0EBC00101EB8011354800EB41117C
:1055E0006031BDF8D00000EB001001EBC00082710B
:1055F0008F229DF8AC00C0EBC00101EB80112C485C
:1056000000EB411060309DF89C1001EB011100EBA4
:10561000C10042711CE008229DF8AC00C0EBC00143
:1056200001EB8011224800EB411160319DF89C0094
:1056300000EB001001EBC000427100219DF8AC00AE
:10564000C0EBC00202EB8012194800EB4210C1709F
:10565000FDE3BDF8A00008287DD19DF8AC0000EB6B
:105660004001C1EBC010114901EBC0008078010678
:105670009DF8AC0000EB4002C2EBC0100B4A02EBFD
:10568000C000C07841EA00419DF8AC0000EB400248
:10569000C2EBC010054A02EBC000007941EA0021CC
:1056A0009DF8AC0000EB400204E0000024660020FE
:1056B000FC340020C2EBC010FE4A02EBC00040796F
:1056C0000843C117CDE9080108F01CF901469DF80F
:1056D000AC00C0EBC00202EB8012F74800EB4212B4
:1056E00060329DF89C0000EB001002EBC0004163AB
:1056F0009DF8AC00C0EBC00101EB8011EE4800EB5F
:10570000411160319DF89C0000EB001011F8301041
:105710009DF8AC00C0EBC00202EB8012E64800EB43
:1057200042100079814230DA00219DF8AC00C0EBD4
:10573000C00202EB8012E04800EB4210C17005226B
:105740009DF8AC00C0EBC00101EB8011DA4800EB22
:105750004111603100E07AE09DF89C0000EB001000
:1057600001F830208E229DF8AC00C0EBC00101EBA7
:105770008011D14800EB411060309DF89C1001EB86
:10578000011100EBC100427161E09DF8AC00C0EB7B
:10579000C00101EB8011C84800EB41106030BDF83A
:1057A000D01001EB011100EBC1008079012831D14B
:1057B00000229DF8AC00C0EBC00101EB8011BE4897
:1057C00000EB41116031BDF8D00000EB001001EB9F
:1057D000C00082718F229DF8AC00C0EBC00101EBCC
:1057E0008011B54800EB411160319DF89C0000E04C
:1057F000FDE300EB001001EBC000427101219DF8B8
:10580000AC00C0EBC00202EB8012AB4800EB4210D0
:10581000C1701CE08E229DF8AC00C0EBC00101EB12
:105820008011A54800EB411160319DF89C0000EB10
:10583000001001EBC000427100219DF8AC00C0EBEC
:10584000C00202EB80129C4800EB4210C170FEE2E5
:10585000BDF8A00003282ED100219DF8AC00C0EBBC
:10586000C00202EB8012944800EB4210C17001228A
:105870009DF8AC00C0EBC00101EB80118E4800EB3D
:1058800041116031BDF8D00000EB001001EBC00009
:1058900082718C229DF8AC00C0EBC00101EB80113D
:1058A000854800EB411060309DF89C1001EB011120
:1058B00000EBC1004271FFE3BDF8A0000F287AD1D0
:1058C0009DF8AC0000EB400101EB00117B4800EBC0
:1058D0000110007BF0BB00202C902D900021369110
:1058E0001FE0DDE92C10000240EA11620902CDE957
:1058F0002C129DF8AC0000EB4001C1EBC0106D49CB
:1059000001EBC001BDF8D800C0F10600085CDDE97C
:105910002C341843CDE92C04BDF8D800401C80B2CB
:105920003690BDF8D8000528DBDB9DF8AC00DDE93A
:105930002C12C0EBC00303EB80135F4800EB431352
:1059400060339DF89C0000EB001003EBC00040F8B2
:10595000221F01E046E0B0E3426000222C922D922B
:105960000021369120E0DDE92C10000240EA1162AE
:105970000902CDE92C129DF8AC0000EB4001C1EB0F
:10598000C0104C4901EBC001BDF8D800C0F10B00BC
:10599000085CDDE92C3440EA0302CDE92C24BDF893
:1059A000D800401C81B23691BDF8D8000528DADB5A
:1059B00002E066E3CDE2CBE29DF8AC00DDE92C121B
:1059C000C0EBC00303EB80133B4800EB4310603097
:1059D0009DF89C3003EB031300EBC3002230816081
:1059E000C26086E000202C902D900021369120E0AE
:1059F000DDE92C10000240EA11620902CDE92C1207
:105A00009DF8AC0000EB4001C1EBC010294901EB4F
:105A1000C001BDF8D800C0F10700085CDDE92C34F6
:105A200040EA0302CDE92C24BDF8D800401C81B225
:105A30003691BDF8D8000628DADB9DF8AC00DDE928
:105A40002C12C0EBC00303EB80131B4800EB431385
:105A500060339DF89C0000EB001003EBC00040F8A1
:105A6000221F426000222C922D920021369120E0CC
:105A7000DDE92C10000240EA11620902CDE92C1286
:105A80009DF8AC0000EB4001C1EBC010094901EBEF
:105A9000C001BDF8D800C0F10D00085CDDE92C3470
:105AA00040EA0302CDE92C24BDF8D800401C81B2A5
:105AB000369105E024660020FC3400203C300020B4
:105AC000BDF8D8000628D3DB9DF8AC00DDE92C2119
:105AD000C0EBC00303EB8013FE4800EB43106030C3
:105AE0009DF89C3003EB031300EBC300223082606F
:105AF000C1609DF8AC00C0EBC00101EB8011F5481E
:105B000000EB411160319DF89C0000EB001011F892
:105B100030109DF8AC00C0EBC00202EB8012ED48E3
:105B200000EB4210007981427ED1EB4890F8C80723
:105B3000E8BB0021E948C0F83D109DF8AC00C0EB7F
:105B4000C00101EB8011E34800EB411060309DF88B
:105B50009C1001EB011100EBC10022301022014624
:105B60000990DE482D30F2F770FB9DF8AC00C0EBD9
:105B7000C00101EB8011D74800EB411060309DF867
:105B80009C1001EB011100EBC101D448401C51F8FD
:105B90001A2F0262496841629DF8AC0000EB400197
:105BA00001EB0011CE4800EB0110303000E067E05F
:105BB0009DF89C1000EB01100078C84981F8200086
:105BC00001F1210001F59C510A6F0262B1F87410D5
:105BD00081849DF8AC00C0EBC00101EB8011BD4891
:105BE00000EB411160319DF89C0000EB001001EBCF
:105BF000C000416BB948C0F829109DF8AC0000EB1B
:105C0000400101EB0011B64800EB011130319DF865
:105C10009C0001EB00104168B048C0F84710C06D0F
:105C200081B20220099100E023E1F3F751FA00214B
:105C30000620F4F78DF9A948C06DA849C98B8842A0
:105C400004D2A648C06D401CA449C86500210520A7
:105C5000F4F77EF99DF8AC0000EB400101EB001178
:105C60009F4800EB011030309DF89C1000EB0110B4
:105C7000801C0990007820F008020998027015E055
:105C80009DF8AC0000EB400101EB0011944800EBE3
:105C9000011030309DF89C1000EB0110801C099021
:105CA000007820F008000830099908709DF8AC00D1
:105CB00000EB400101EB0011894800EB011030308E
:105CC0009DF89C1000EB0110801C0990007820F0DA
:105CD0002002099802709DF8AC100220F4F738F900
:105CE0009DF8AC009DF89C1001EB0010C217CDE9A7
:105CF0002C0200222C9800EB8001C1EB8011774828
:105D000064300844C0F81D209DF8AC00C0EBC00111
:105D100001EB80116F4800EB411060309DF89C1042
:105D200001EB011100EBC100223009902C9800EB2F
:105D30008001C1EB80116948643001440D311022AB
:105D40000891DDE90801F2F780FA9DF8AC00C0EB9C
:105D5000C00101EB80115F4800EB411160319DF8FB
:105D60009C0000EB001001EBC0012C9800EB8002BE
:105D7000C2EB801259486430104451F81A2F40F891
:105D8000012F496841609DF8AC0000EB400101EB38
:105D90000011534800EB011130319DF89C0001EBDC
:105DA000001001782C9800EB8002C2EB80124B4867
:105DB000643081542C9800EB8001C1EB801147487E
:105DC000643001444748026F41F8212FB0F8740055
:105DD00088809DF8AC00C0EBC00101EB80113D480C
:105DE00000EB411160319DF89C0000EB001001EBCD
:105DF000C000416B2C9800EB8002C2EB8012374848
:105E000064301044C0F809109DF8AC0000EB40016C
:105E100001EB0011324800EB011130319DF89C007C
:105E200001EB001041682C9800EB8002C2EB80125D
:105E30002A4864301044C0F827102C9881B20820FA
:105E40000991F4F785F800229DF8AC0000E033E1F9
:105E5000C0EBC00101EB80111E4800EB4111603125
:105E60009DF89C0000EB001001EBC00080F83E2084
:105E70005CE09DF8AC0000EB400101EB001118481C
:105E800000EB011030309DF89C1000EB0110801CDD
:105E90000990007820F00400001D099908709DF811
:105EA000AC0000EB400101EB00110D4800EB0110CC
:105EB00030309DF89C1000EB0110801C0990007898
:105EC00020F0800180310998017001219DF8AC001B
:105ED0000AE00000FC340020BC220020BC1200209C
:105EE0003C3000203C260020C0EBC00202EB8012B8
:105EF000FE4800EB4210C1709DF8AC00C0EBC00141
:105F000001EB8011F94800EB411002799DF8AC00DB
:105F1000C0EBC00101EB8011F44800EB4110603090
:105F20009DF89C1001EB011100F831208F229DF8A3
:105F3000AC00C0EBC00101EB8011EC4800EB41105C
:105F400060309DF89C1001EB011100EBC100427123
:105F5000B2E0BDF8A00003284FD10121E44880F849
:105F6000EC169DF8AC00C0EBC00101EB8011DF48DE
:105F700000EB411160319DF89C0000EB001011F81E
:105F800030109DF8AC00C0EBC00202EB8012D74885
:105F900000EB42100079814230DA00219DF8AC001C
:105FA000C0EBC00202EB8012D04800EB4210C1707F
:105FB00001229DF8AC00C0EBC00101EB8011CB4881
:105FC00000EB411160319DF89C0000EB001001F8DE
:105FD00030208F229DF8AC00C0EBC00101EB801196
:105FE000C24800EB411060309DF89C1000E065E075
:105FF00001EB011100EBC100427141E09DF8AC00E2
:10600000C0EBC00101EB8011B84800EB41106030DB
:106010009DF89C1001EB011100EBC10080788028F5
:106020002ED100219DF8AC00C0EBC00202EB801223
:10603000AE4800EB4210C17080229DF8AC00C0EB6E
:10604000C00101EB8011A94800EB411160319DF8BE
:106050009C0000EB001001EBC000427100229DF893
:10606000AC00C0EBC00101EB8011A04800EB411077
:1060700060309DF89C1001EB011100EBC1008270B3
:106080001AE0BDF8A000032815D10021984880F837
:10609000EC168F229DF8AC00C0EBC00101EB801123
:1060A000924800EB411060309DF89C1001EB01110B
:1060B00000EBC100427100BF00BF00BF00BF8C48B1
:1060C00090F8EF03B0B18B499DF8AC0031F8101097
:1060D00009919DF8AC0000EB4001C1EBC01086496E
:1060E00001EBC001012308919DF8AC20DDE9080116
:1060F000F4F7C6FC0021369111E000219DF8AC00B8
:1061000000EB4002C2EBC0107B4A02EBC002BDF8BC
:10611000D8001154BDF8D800401C81B23691BDF8AA
:10612000D800142843DAE8E774499DF8AC0011F868
:106130001000C009D8BB9DF8AC0011F81000C0F3E6
:10614000C300062832D2DFE800F0036291FDFC3381
:106150009DF8AC0000EB4001C1EBC010664901EBBB
:10616000C001099166A1099817F02CFC11901198B3
:10617000E0B100219DF8AC0000EB40005F4A3C32EA
:1061800002EB8000416001219DF8AC0000EB400073
:1061900002EB8000817059499DF8AC0001EB400191
:1061A0000991087820F07800283008705DE15DE101
:1061B0009DF8AC0000EB4001C1EBC0104E4901EB73
:1061C000C00109914EA1099817F0FCFB119011989C
:1061D000E0B100219DF8AC0000EB4000474A3C32A2
:1061E00002EB8000416001219DF8AC0000EB400013
:1061F00002EB8000817041499DF8AC0001EB400149
:106200000991087820F07800203008702DE19DF881
:10621000AC0000EB4001C1EBC010374901EBC001FD
:10622000099137A1099817F0CDFB11901198E0B1B1
:1062300000219DF8AC0000EB4000304A3C3202EBFC
:106240008000416001219DF8AC0000EB400002EBB2
:106250008000817029499DF8AC0001EB4001099153
:10626000087820F0780018300870FEE000219DF8D2
:10627000AC0000EB4000214A3C3202EB8000416060
:1062800001219DF8AC0000EB400002EB8000817022
:106290009DF8AC0000EB4001C1EBC010164901EBCA
:1062A000C0011198801D095C30399DF8AC0000EBED
:1062B0004002C2EBC010104A02EBC0021198401D10
:1062C000105C303841EA0010C117CDE9080106F032
:1062D00065FD0C4988719DF8AC1001EB4100C0EBE5
:1062E000C110054901EBC00109910DE0FC3400200B
:1062F000BC2200207C58002024660020042E0020B0
:106300004F4B0000842A002060A1099817F05AFB27
:106310001190119890B39DF8AC1001EB4100C0EBC7
:10632000C1105B4901EBC0011198401C085C30288A
:1063300025DB9DF8AC1001EB4100C0EBC1105449C6
:1063400001E068E03AE001EBC0011198401C095CF3
:1063500030399DF8AC0000EB4002C2EBC0104C4A53
:1063600002EBC0031198185C303841EA0010C117E5
:10637000CDE9080106F012FD4649C87112E09DF80A
:10638000AC1001EB4100C0EBC110414901EBC00171
:106390001198085C3038C117CDE9080106F0FEFC01
:1063A0003C49C8713C499DF8AC0001EB40010991A2
:1063B000087820F078001830087056E09DF8AC108E
:1063C00001EB4100C0EBC110314901EBC001099163
:1063D000AFF2D401099817F0F5FA11901198C8B1ED
:1063E00000202E4908602C499DF8AC0001EB4001CB
:1063F0000991087820F080018031099801704FF4EC
:106400007A719DF8AC0000EB4000234A3C3202EB6D
:106410008000816029E09DF8AC1001EB4100C0EBE9
:10642000C1101B4901EBC0010991AFF22C11099871
:1064300017F0C8FA11901198B0B1194890F8EE060B
:1064400020F08001164880F8EE1613499DF8AC0044
:1064500001EB40010991087820F0780008300870BD
:10646000002110488170416000BF00BF0E480078D5
:106470000E49097808440E49097808440D490978FD
:106480000844002874F411AD38B070BD2C00000031
:1064900024660020842A0020042E00208802424224
:1064A000BC220020BC580020120000201300002055
:1064B000140000201500002007B5D2B000211A9169
:1064C0001991189117911691159114910022129219
:1064D0001392109211920F910E910D910C910B91BC
:1064E0000A91FEA006C8CDE90812FEA006C8CDE9B3
:1064F0000612002105910020FC490870529800EB1B
:10650000400101EB0011FA4800EB0110817916916E
:10651000F849529801EB00115398085C05287CDD7E
:106520000621F44A529802EB0012539811540022AB
:106530005298C0EBC00101EB8011EF4800EB411114
:106540006031539800EB001001F83020529800EBB6
:10655000400101EB0011E64800EB01113031539886
:1065600001EB0010807820F08002529800EB40018F
:1065700001EB0011DE4800EB01113031539801EBC3
:10658000001082705298C0EBC00101EB8011DA4814
:1065900000EB41116031539800EB001001EBC0009B
:1065A00090F8860020F008025298C0EBC00101EB81
:1065B0008011D14800EB41116031539800EB00107D
:1065C00001EBC00080F886205298C0EBC00101EBBF
:1065D0008011C94800EB41116031539800EB001065
:1065E00001EBC00090F8860020F001025298C0EB49
:1065F000C00101EB8011C04800EB4111603153989C
:1066000000EB001001EBC00080F88620529800EBF0
:10661000400101EB0011B64800E094E000EB0110EE
:106620008079092816D2DFE800F08D051627384951
:106630005A6B7C00E5225298C0EBC00101EB80113F
:10664000AD4800EB41106030539901EB011100EBB4
:10665000C100427176E0A1225298C0EBC00101EB6B
:106660008011A54800EB41106030539901EB0111F6
:1066700000EBC100427165E0A1225298C0EBC0015D
:1066800001EB80119C4800EB41106030539901EB05
:10669000011100EBC100427154E0B1225298C0EBED
:1066A000C00101EB8011944800EB41106030539918
:1066B00001EB011100EBC100427143E0312252981D
:1066C000C0EBC00101EB80118B4800EB4110603042
:1066D000539901EB011100EBC100427132E0F1224C
:1066E0005298C0EBC00101EB8011834800EB4110D0
:1066F0006030539901EB011100EBC100427121E0C0
:1067000006225298C0EBC00101EB80117A4800EBE1
:1067100041106030539901EB011100EBC10042714F
:1067200010E015225298C0EBC00101EB80117248B5
:1067300000EB41106030539901EB011100EBC100F7
:10674000427100BF00BF6B496C39529811F81000BC
:106750000121B1EBD01F46F03681529800EB400189
:1067600001EB0011624800EB0110407B02287DD153
:1067700010E011F079F96149C1F8FC030846D0F83E
:10678000FC03C0F300410E915C48D0F8FC03C0F359
:1067900042010D910D980028EBD055215298C0EB85
:1067A000001000EB8000564A02F83010FD2152988C
:1067B000C0EB001000EB800002EBC0004170AA218A
:1067C0005298C0EB001000EB800002EBC00081701B
:1067D00000215298C0EB001000EB800002EBC000DB
:1067E000C1705298C0EB001000EB800002EBC000BB
:1067F000017161215298C0EB001000EB800002EBA8
:10680000C000417100215298C0EB001000EB8000E5
:1068100002EBC0008171FA215298C0EB001000EB2E
:10682000800002EBC000C171364841795298C0EB3C
:10683000001000EB800002EBC000017231480179CA
:106840005298C0EB001000EB800002EBC0004172D8
:106850002C48C1785298C0EB001000EB800002EB8E
:10686000C000817227488178529800E0FEE3C0EBB7
:10687000001000EB800002EBC000C172214841789B
:106880005298C0EB001000EB800002EBC0000173D7
:106890001A4890F8F0135298C0EB001000EB8000FB
:1068A00002EBC000417300211A9132E01348D0F886
:1068B000FC03BDF86810C1F10301C900C840C1B2B2
:1068C0005298C0EB001000EB80000D4A02EBC002B2
:1068D000BDF868001030115416E000000169323034
:1068E0003130300001693230453030001600002070
:1068F0003C300020702E0020FC340020BC22002000
:10690000C45C0020AC260020BDF86800401C81B2A9
:106910001A91BDF868000428C8DB5298C0EB00103B
:1069200000EB8000FE4A02EBC0005499017515216E
:106930000F9100215298C0EBC00202EB8012F9487F
:1069400000EB42104171549808B95120549054986A
:10695000002806F014825498152876D00ADCA0F19D
:106960000B000A2872D2DFE800F0FEFD77FC71719F
:10697000787971FBA1286CD006DC502868D05128AA
:1069800007D0522862D1FDE3A22863D0A428F9D110
:1069900061E0E54890F8C807012825D100201A9049
:1069A00015E0BDF868000E30E049095C5298C0EB74
:1069B000001000EB8000DA4A02EBC002BDF868006C
:1069C00015301154BDF86800401C81B21A91D848A6
:1069D00080880838BDF868108842E2DCD448808896
:1069E000C01D80B20F902FE05298C0EB001000EB5A
:1069F0008000CB4A02EBC0005499017500211A9126
:106A000015E000215298C0EB001000EB8000C44A52
:106A100002EBC002BDF83C001154BDF83C00401C24
:106A200081B20F91BDF86800401C81B21A91529852
:106A300000EB400101EB0011BE4800EB0110C179F1
:106A4000BDF868008142DCDC86E3FCE3FCE300E0A7
:106A50002AE000BF00BF00BF00BF00BF00201A90A7
:106A600015E0BDF868000E30B049095C5298C0EBE3
:106A7000001000EB8000AA4A02EBC002BDF86800DB
:106A800015301154BDF86800401C81B21A91A84815
:106A900080880838BDF868108842E2DCA448808805
:106AA000C01D80B20F9057E35298C0EBC00101EBBC
:106AB00080119C4800EB411081795298C0EB001086
:106AC00000EB8000964A02EBC002BDF83C00115476
:106AD000BDF83C00401C81B20F915298C0EBC00140
:106AE00001EB80118F4800EB4110807900EB4001F1
:106AF00001EB00118F4800EB01100168084604917A
:106B0000002106F0FFFECDE9120100211A911EE0DE
:106B1000BDF86800C0F10200C200DDE91201CDE954
:106B20001B10F1F780FBC2B25298C0EB001000EBD3
:106B300080007B4901EBC000BDF83C30BDF8681017
:106B400019444254BDF86800401C80B21A90BDF848
:106B500068000328DCDBBDF83C00C01C81B203E008
:106B6000B1E34BE349E3F8E20F915298C0EBC00167
:106B700001EB80116B4800EB4110807900EB400184
:106B800001EB00116B4800EB0110017908460491FC
:106B9000002106F0B7FEC1B25298C0EB001000EB26
:106BA00080005F4A02EBC002BDF83C001154BDF802
:106BB0003C00401C81B20F915298C0EBC00101EB28
:106BC0008011584800EB4110807900EB400101EB47
:106BD0000011584800EB011041790846049100214A
:106BE00006F090FEC1B25298C0EB001000EB80009E
:106BF0004B4A02EBC002BDF83C001154BDF83C000A
:106C0000401C81B20F915298C0EBC00101EB801182
:106C1000444800EB4110807900EB400101EB00118A
:106C2000444800EB0110817908460491002106F0E8
:106C300069FEC1B25298C0EB001000EB8000384AE8
:106C400002EBC002BDF83C001154BDF83C00401CF2
:106C500081B20F915298C0EBC00101EB8011314815
:106C600000EB4110807900EB400101EB001131484D
:106C700000EB0110C17908460491002106F042FEA4
:106C8000C1B25298C0EB001000EB8000244A02EB26
:106C9000C002BDF83C001154BDF83C00401C81B25C
:106CA0000F915298C0EBC00101EB80111D4800EB21
:106CB0004110807900EB400101EB00111D4800EB11
:106CC0000110816808460491002106F01BFEC1B244
:106CD0005298C0EB001000EB8000114A02EBC0029A
:106CE000BDF83C001154BDF83C00401C81B20F912E
:106CF0005298C0EBC00101EB80110A4800EB411033
:106D0000807900EB400101EB00110A4800EB011013
:106D1000017B08460491002106F0F4FDC1B20BE0AE
:106D2000C45C0020FC340020BC220020EC7D00204C
:106D3000BC1200203C3000205298C0EB001000EB49
:106D40008000FE4A02EBC002BDF83C001154BDF8C1
:106D50003C00401C81B20F915298C0EBC00101EB86
:106D60008011F74800EB4110807900EB400101EB06
:106D70000011F44800EB0110807906287ED1002034
:106D80001A908CE05298C0EBC00101EB8011EC48E6
:106D900000EB4110807900EB400101EB0011E94864
:106DA00000EB01113031BDF8680001EB00100178F3
:106DB00008460491002106F0A5FDC1B25298C0EB2F
:106DC000001000EB8000DD4A02EBC002BDF8680055
:106DD00000EB4003BDF83C00184411545298C0EB3E
:106DE000C00101EB8011D64800EB4110807900EB27
:106DF000400101EB0011D34800EB01113031BDF827
:106E0000680001EB0010417808460491002106F06B
:106E100079FDC1B25298C0EB001000EB8000C74A68
:106E200002EBC002BDF8680000EB4003BDF83C0077
:106E30001844401C11545298C0EBC00101EB801162
:106E4000BF4800EB4110807900EB400101EB0011DD
:106E5000BC4800EB01113031BDF8680001EB0010B7
:106E6000017A08460491002106F04CFDC1B2529807
:106E7000C0EB001000EB8000B04A00E036E002EB0F
:106E8000C002BDF8680000EB4003BDF83C001844A8
:106E9000801C1154BDF86800401C81B21A915298B0
:106EA00000EB400101EB0011A64800EB0110C17995
:106EB000BDF8680081423FF765AF5298C0EBC00152
:106EC00001EB80119E4800EB4110807900EB4001FE
:106ED00001EB00119B4800EB0110C07900EB400171
:106EE000BDF83C00084481B20F9135E100201A90B2
:106EF0005BE05298C0EBC00101EB8011904800EBC1
:106F00004110807900EB400101EB00118D4800EB4E
:106F100001113031BDF8680001EB0010017808461E
:106F20000491002106F0EEFCC2B25298C0EB0010B2
:106F300000EB8000814901EBC003BDF86810BDF88B
:106F40003C0000EB41001A545298C0EBC00101EB29
:106F500080117B4800EB4110807900EB400101EB90
:106F60000011784800EB01113031BDF8680001EBE9
:106F70000010417808460491002106F0C3FCC2B21B
:106F80005298C0EB001000EB80006C4901EBC0038D
:106F9000BDF86810BDF83C0000EB4100401C1A54DD
:106FA000BDF86800401C81B21A91529800EB400174
:106FB00001EB0011634800EB0110C179BDF86800D6
:106FC000814296DC5298C0EBC00101EB80115C4815
:106FD00000EB4110807900EB400101EB00115948B2
:106FE00000EB0110C179BDF83C0000EB410081B21B
:106FF0000F915298C0EBC00101EB8011504800EB9B
:107000004110807900EB400101EB00114D4800EB8D
:107010000110007F00F003015298C0EB001000EB5C
:107020008000464A02EBC002BDF83C001154BDF896
:107030003C00401C81B20F915298C0EBC00101EBA3
:1070400080113F4800EB4110807900EB400101EBDB
:1070500000113C4800EB0110007FC0F30111529871
:10706000C0EBC00202EB8012354800E096E200EB74
:107070004210807900EB400202EB0012314800EB35
:107080000210007FC0F3810041EA00115298C0EB6A
:10709000001000EB8000294A02EBC002BDF83C0062
:1070A0001154BDF83C00401C81B20F9100211A918F
:1070B00028E05298C0EBC00101EB8011204800EBA2
:1070C0004110807900EB400101EB00111D4800EBFD
:1070D00001113031BDF8680001EB0010817A52983F
:1070E000C0EB001000EB8000144A02EBC002BDF8B8
:1070F0003C30BDF8680018441154BDF86800401CCD
:1071000081B21A91529800EB400101EB00110D4839
:1071100000EB0110C179BDF868008142C9DC5298CA
:10712000C0EBC00101EB8011054800EB41108079F4
:1071300000EB400101EB0011024805E0C45C0020B7
:10714000FC3400203C30002000EB0110C179BDF878
:107150003C00084481B20F91D2E0FE484179529838
:10716000C0EB001000EB8000FB4A02EBC000417551
:10717000F84801795298C0EB001000EB800002EB58
:10718000C00000E03BE08175F248C1785298C0EB46
:10719000001000EB800002EBC000C175ED48817863
:1071A0005298C0EB001000EB800002EBC0000176AB
:1071B000E84841785298C0EB001000EB800002EBE9
:1071C000C0004176E54890F8F0135298C0EB0010EB
:1071D00000EB800002EBC0008176BDF83C00801D12
:1071E00081B20F9100215298C0EBC00202EB8012D5
:1071F000DB4800EB4210417182E081E080E000203A
:107200001A905BE05298C0EBC00101EB8011D448AA
:1072100000EB4110C01DBDF8681001EB410202EB0C
:10722000C10110F8110090B300225298C0EBC001C8
:1072300001EB8011CA4800EB4111C91DBDF868007F
:1072400000EB400301E03FE03FE003EBC00001F84A
:1072500010205298C0EBC00101EB8011C04800EB38
:107260004111C91DBDF8680000EB400202EBC000EF
:1072700001EB400041785298C0EB001000EB800019
:10728000B54A02EBC002BDF83C0011540CE0FFE728
:10729000FF215298C0EB001000EB8000AE4A02EBD9
:1072A000C002BDF83C001154BDF83C00401C81B246
:1072B0000F91BDF86800401C81B21A91BDF86800BA
:1072C00004289FDB1CE01BE01AE000210F911A91BB
:1072D00011E00021529800EB4002C2EBC010A14A1D
:1072E00002EBC002BDF868000D301154BDF8680013
:1072F000401C81B21A91BDF868000528E9DB00BF87
:1073000000BFBDF83C00C01F010A5298C0EB00103E
:1073100000EB8000904A02EBC0008173BDF83C0096
:10732000C01FC1B25298C0EB001000EB800002EB0E
:10733000C000C17300211A9123E05298C0EB0010E5
:1073400000EB8000844901EBC001BDF868001430F7
:10735000095C0491DDE90D210498F2F728FD01464E
:107360005298C0EB001000EB80007B4A02EBC00299
:10737000BDF8680014301154BDF86800401C81B29B
:107380001A91BDF83C00C01FBDF868108842D4DCDB
:10739000724890F8EF0398B1BDF83C00C01F81B26D
:1073A00004915298C0EB001000EB80006A4901EB99
:1073B000C000C01D00230390529A0499F3F760FBAC
:1073C000BDF83C00C01F81B204915298C0EB001080
:1073D00000EB8000604901EBC000C01D03900499E0
:1073E000F2F75CFA05900598020A5298C0EB00107B
:1073F00000EB8000584901EBC000BDF83C1042543E
:10740000BDF83C00401C80B20F900598C2B2529863
:10741000C0EB001000EB80004F4901EBC000BDF84D
:107420003C104254BDF83C00401C80B20F90BDF8A7
:107430003C00401F020A5298C0EB001000EB800095
:10744000454901EBC000C270BDF83C00401FC2B20C
:107450005298C0EB001000EB800001EBC0000271FD
:10746000BDF83C00401F80B204905298C0EB001061
:1074700000EB800001EBC000401D0390049910F068
:1074800053FC01465298C0EB001000EB8000324ADA
:1074900002EBC002BDF83C001154BDF83C00401C9A
:1074A00081B20F91529830B1012815D0022825D011
:1074B000032849D135E0BDF83C0060B180212A485D
:1074C000F3F7A8FABDF83C002849086001212748D5
:1074D000001FF2F763FA37E0BDF83C0068B10821FD
:1074E0002148F3F797FABDF83C002049A4394867D2
:1074F00001211E483438F2F751FA25E0BDF83C006E
:1075000070B14FF480711A48F3F784FABDF83C006B
:10751000164918310860012114481430F2F73EFA78
:1075200012E0BDF83C0070B14FF480610E48F3F7F3
:1075300071FABDF83C000D49A439C86501210B481A
:107540004C38F2F72BFA00BF00BF044890F8EF0365
:1075500000280FE0AC260020C45C0020BC220020E4
:10756000FC34002024660020000C0240A46002408D
:107570000000024005F003845298C0EB001000EBBD
:107580008000FB4901EBC00100230491BDF83C10D1
:10759000529A0498F3F774FA05F0F1BBF548007FAE
:1075A000012805F001829DF858000028F9D09DF8C7
:1075B0005800092885F08F81DFE810F01A270900AC
:1075C0004B095D0ED81258168E174C1C1B2352986F
:1075D00000EB400101EB0011E74800EB01113031F5
:1075E000539801EB0010417808460491002106F001
:1075F00089F9C1B215915298C0EBC00101EB80111D
:10760000DE4800EB41116031539800EB001011F897
:1076100030105298C0EBC00202EB8012D74800EB4A
:1076200042100079814209D101215298C0EBC00279
:1076300002EB8012D14800EB4210C170D049529841
:1076400001EB00115398085C401CC1B2CC4A52981F
:1076500002EB0012539811545298C0EBC00101EB99
:107660008011C64800EB41106030539901EB0111C5
:1076700000EBC10090F88600C0F3C00090B15398B1
:1076800000EB400101EB0011BB4800EB0110417918
:107690000B464FF4805204914FF4E131529806F0BA
:1076A0001FF819E0529800EB400101EB0011B248BD
:1076B00000EB011041790491529800EB400101EB7D
:1076C0000011AD4800EB0110016803914FF48052A6
:1076D000049B529806F004F85498C5287DD012DC1B
:1076E000B5287BD008DC112879D0122878D013284F
:1076F00077D0B22856D1A0E3B62873D0B92872D07B
:10770000C328F7D1D4E2D9284DD006DCCA286BD0E3
:10771000CE286AD0D528EDD106E0E12866D0E5284C
:1077200065D0E728E6D1FCE3F5215298C0EB0010C4
:1077300000EB80008E4A02F830109DF854105298E9
:10774000C0EB001000EB800002EBC0004170A221F2
:107750005298C0EB001000EB800002EBC00081707B
:10776000D5215298C0EB001000EB800002EBC00066
:10777000C1705298C0EB001000EB8000114601EB85
:10778000C00104910321049805F098FF0146529826
:10779000C0EB001000EB8000754A02EBC0000171E5
:1077A00005210F9109E3F5215298C0EB001000EB81
:1077B00080006F4A02F830109DF854105298C0EBC8
:1077C000001000EB800002EBC0004170A221529833
:1077D000C0EB001000EB80000AE0FCE32EE0FBE3CE
:1077E000FBE3FBE3EAE249E1A1E2F8E3F8E3F8E3D3
:1077F00002EBC0008170D9215298C0EB001000EB61
:10780000800002EBC000C1705298C0EB001000EB8A
:107810008000114601EBC00104910321049805F09A
:107820004DFF01465298C0EB001000EB8000504A1B
:1078300002EBC000017105210F91B3E7F5215298C9
:10784000C0EB001000EB8000494A02F830109DF8B0
:1078500054105298C0EB001000EB800002EBC00007
:107860004170529800EB400101EB0011424800EBDF
:107870000110007BB0BB5298C0EBC00101EB80113E
:107880003E4800EB41106030539901EB011100EBD1
:10789000C1008068B0F5100F05D34FF4100100202F
:1078A000CDE9101011E05298C0EBC00101EB80113E
:1078B000324800EB41106030539901EB011100EBAD
:1078C000C10080680022CDE91002A5215298C0EBCA
:1078D000001000EB8000264A02EBC00081700021FE
:1078E0001A911DE04EE0BDF86800C0F10200C20030
:1078F000DDE91001CDE91D10F0F795FCC2B25298F8
:10790000C0EB001000EB8000194901EBC003BDF88B
:107910006800C01C1A54BDF86800401C80B21A9060
:10792000BDF868000328DEDBB5215298C0EB0010DB
:1079300000EB80000E4A02EBC00081715298C0EB50
:10794000001000EB8000114601EBC00104910621FC
:10795000049805F0B3FE01465298C0EB001000EB0E
:107960008000034A02EBC000C17108210F9184E03E
:10797000C45C0020BC1200203C300020FC340020FD
:10798000702E00205298C0EBC00101EB8011FE4820
:1079900000EB41106030539901EB011100EBC10085
:1079A0008068B0F1104F05D34FF010410020CDE9B1
:1079B000101011E05298C0EBC00101EB8011F248A9
:1079C00000EB41106030539901EB011100EBC10055
:1079D00080680022CDE91002A6215298C0EB001069
:1079E00000EB8000E94A02EBC000817000211A918F
:1079F0001CE0BDF86800C0F10300C200DDE9100121
:107A0000CDE91F10F0F70FFCC2B25298C0EB001086
:107A100000EB8000DD4901EBC003BDF86800C01C2D
:107A20001A54BDF86800401C80B21A90BDF8680076
:107A30000428DEDBB5215298C0EB001000EB80007B
:107A4000D24A02EBC000C1715298C0EB001000EBAB
:107A50008000114601EBC00104910721049805F054
:107A60002DFE01465298C0EB001000EB8000C74A83
:107A700002EBC000017209210F9193E6F5215298A3
:107A8000C0EB001000EB8000C04A02F830109DF8F7
:107A900054105298C0EB001000EB800002EBC000C5
:107AA0004170529800EB400101EB0011B84800EB27
:107AB0000110007BB0BB5298C0EBC00101EB8011FC
:107AC000B14800EB41106030539901EB011100EB1C
:107AD000C1008068B0F5100F05D14FF410010020EF
:107AE000CDE9101011E05298C0EBC00101EB8011FC
:107AF000A54800EB41106030539901EB011100EBF8
:107B0000C10080680022CDE91002A5215298C0EB87
:107B1000001000EB80009D4A02EBC0008170002144
:107B20001A911FE046E0BDF86800C0F10200C200F3
:107B3000DDE91010CDE9210108462199F0F773FB2A
:107B4000C2B25298C0EB001000EB80008F4901EBED
:107B5000C003BDF86800C01C1A54BDF86800401C82
:107B600080B21A90BDF868000328DCDBB921529876
:107B7000C0EB001000EB8000844A02EBC000817172
:107B80005298C0EB001000EB8000114601EBC001E1
:107B900004910621049805F091FD01465298C0EB2E
:107BA000001000EB8000794A02EBC000C17108218F
:107BB0000F917CE05298C0EBC00101EB801172483C
:107BC00000EB41106030539901EB011100EBC10053
:107BD0008068B0F1104F05D14FF010400021CDE981
:107BE000100111E05298C0EBC00101EB8011664812
:107BF00000EB41106030539901EB011100EBC10023
:107C000080680022CDE91002A6215298C0EB001036
:107C100000EB80005D4A02EBC000817000211A91E8
:107C20001EE0BDF86800C0F10300C200DDE91010DD
:107C3000CDE9230108462399F0F7F5FAC2B252982C
:107C4000C0EB001000EB8000504901EBC003BDF811
:107C50006800C01C1A54BDF86800401C80B21A901D
:107C6000BDF868000428DCDBB9215298C0EB001095
:107C700000EB8000454A02EBC000C1715298C0EB96
:107C8000001000EB8000114601EBC00104910721B8
:107C9000049805F013FD01465298C0EB001000EB6C
:107CA00080003A4A02EBC000017209210F9179E588
:107CB000F5215298C0EB001000EB8000334A02F827
:107CC00030109DF854105298C0EB001000EB80006B
:107CD00002EBC0004170A2215298C0EB001000EBF3
:107CE000800002EBC0008170C3215298C0EB0010ED
:107CF00000EB800002EBC000C1705298C0EB001096
:107D000000EB8000114601EBC001049103210498AF
:107D100005F0D4FC01465298C0EB001000EB800047
:107D20001A4A02EBC000017105210F913AE5F521D5
:107D30005298C0EB001000EB8000144A02F830109B
:107D40009DF854105298C0EB001000EB800002EB3D
:107D5000C0004170A2215298C0EB001000EB8000DF
:107D600002EBC0008170CA215298C0EB001000EBFA
:107D7000800002EBC000C1705298C0EB001000EB15
:107D80008000114606E00000FC340020C45C0020A6
:107D90003C30002001EBC00104910321049805F060
:107DA0008DFC01465298C0EB001000EB8000FC4AAD
:107DB00002EBC000017105210F9117E3F5215298E4
:107DC000C0EB001000EB8000F54A02F830109DF87F
:107DD00054105298C0EB001000EB800002EBC00082
:107DE0004170A2215298C0EB001000EB800002EB22
:107DF000C0008170B6215298C0EB001000EB8000EB
:107E000002EBC000C1705298C0EB001000EB800084
:107E1000114601EBC00104910321049805F04EFCCA
:107E200001465298C0EB001000EB8000DC4A02EBE8
:107E3000C000017105210F91D8E2F5215298C0EBE5
:107E4000001000EB8000D64A02F830109DF8541064
:107E50005298C0EB001000EB800002EBC0004170B4
:107E6000529800EB400101EB0011CE4800EB0110ED
:107E7000007BE8BBA4215298C0EB001000EB80000F
:107E800002EBC000817000211A9125E05298C0EBEE
:107E9000C00101EB8011C44800EB411160315398DF
:107EA00000EB001001EBC000416BBDF86800C0F1B1
:107EB0000100C000C1405298C0EB001000EB8000F0
:107EC000B74A02EBC002BDF86800C01C1154BDF8EF
:107ED0006800401C81B21A91BDF868000228D5DB09
:107EE000B2215298C0EB001000EB8000AC4A00E0D9
:107EF0001EE002EBC00041715298C0EB001000EB95
:107F00008000114601EBC00104910521049805F0A1
:107F1000D5FB01465298C0EB001000EB8000A04A50
:107F200000E0A3E202EBC000817107210F9161E044
:107F3000A5215298C0EB001000EB8000984A02EB9C
:107F4000C000817000211A9125E05298C0EBC00159
:107F500001EB8011944800EB41116031539800EB24
:107F6000001001EBC000416BBDF86800C0F10200D9
:107F7000C000C1405298C0EB001000EB8000884A5E
:107F800002EBC002BDF86800C01C1154BDF86800C7
:107F9000401C81B21A91BDF868000328D5DBB221DC
:107FA0005298C0EB001000EB80007D4A02EBC0004D
:107FB00081715298C0EB001000EB8000114601EB7C
:107FC000C00104910621049805F078FB01465298FF
:107FD000C0EB001006E07BE087E2E9E242E3B6E0B6
:107FE00009E004E200EB80006D4A02EBC000C171C1
:107FF00008210F91FAE1F5215298C0EB001000EB37
:108000008000674A02F830109DF854105298C0EB77
:10801000001000EB800002EBC0004170A6215298D6
:10802000C0EB001000EB800002EBC000817000216B
:108030001A9125E05298C0EBC00101EB80115A481B
:1080400000EB41116031539800EB001001EBC000D0
:10805000816BBDF86800C0F10300C000C1405298B8
:10806000C0EB001000EB80004D4A02EBC002BDF8EF
:108070006800C01C1154BDF86800401C81B21A9100
:10808000BDF868000428D5DBE1215298C0EB001050
:1080900000EB8000424A02EBC000C1715298C0EB75
:1080A000001000EB8000114601EBC0010491072194
:1080B000049805F003FB01465298C0EB001000EB5A
:1080C0008000374A02EBC000017209210F91BDE325
:1080D000F5215298C0EB001000EB8000304A02F806
:1080E00030109DF854105298C0EB001000EB800047
:1080F00002EBC0004170A2215298C0EB001000EBCF
:10810000800002EBC0008170C5215298C0EB0010C6
:1081100000EB800002EBC000C1705298C0EB001071
:1081200000EB8000114601EBC0010491032104988B
:1081300005F0C4FA01465298C0EB001000EB800035
:10814000174A02EBC000017105210F917EE3F52172
:108150005298C0EB001000EB8000114A02F830107A
:108160009DF854105298C0EB001000EB800002EB19
:10817000C0004170529800EB400101EB001109482A
:1081800000EB0110007BE8BBAC215298C0EB001063
:1081900000EB800002EBC000817000211A9135E0F5
:1081A000C45C00203C300020FC3400205298C0EB1E
:1081B000C00101EB8011FC4800EB41106030539985
:1081C00001EB011100EBC10050F8221F4068BDF81F
:1081D0006820C2F10402D200CDE9250108462599A4
:1081E000F0F721F8C2B25298C0EB001000EB80000B
:1081F000EE4901EBC003BDF86800C01C1A54BDF87D
:10820000680000E05DE0401C80B21A90BDF8680094
:108210000528CBDB00201A902BE05298C0EBC00160
:1082200001EB8011E04800EB41106030539901EB05
:10823000011100EBC10122318868C968BDF86820CE
:10824000C2F10402D200CDE92710EFF7ECFFC2B271
:108250005298C0EB001000EB8000D44901EBC00342
:10826000BDF8680008301A54BDF86800401C80B2A0
:108270001A90BDF868000528CFDBCE215298C0EBDC
:10828000001000EB8000C94A02EBC0004173529815
:10829000C0EB001000EB8000114601EBC00104911F
:1082A0000D21049805F00AFA01465298C0EB00101F
:1082B00000EB8000BD4A02EBC00081730F210F91DB
:1082C00094E0AE215298C0EB001000EB8000B74A5A
:1082D00002EBC000817000211A912DE05298C0EB92
:1082E000C00101EB8011B04800EB411060305399A0
:1082F00001EB011100EBC10050F8221F4068BDF8EE
:108300006820C2F10502D200CDE929010846299969
:10831000EFF789FFC2B25298C0EB001000EB80006B
:10832000A24901EBC003BDF86800C01C1A54BDF897
:108330006800401C80B21A90BDF868000628CDDBAA
:1083400000201A902BE05298C0EBC00101EB801185
:10835000954800EB41106030539901EB011100EB9F
:10836000C10122318868C968BDF86820C2F10502E0
:10837000D200CDE92B10EFF756FFC2B25298C0EBF6
:10838000001000EB8000894901EBC003BDF86800D4
:1083900009301A54BDF86800401C80B21A90BDF82C
:1083A00068000628CFDBCE215298C0EB001000EB0E
:1083B00080007E4A02EBC000C1735298C0EB0010EF
:1083C00000EB8000114601EBC00104910F210498DD
:1083D00005F074F901465298C0EB001000EB8000E4
:1083E000724A02EBC000017411210F912EE2F521B7
:1083F0005298C0EB001000EB80006C4A02F830107D
:108400009DF854105298C0EB001000EB800002EB76
:10841000C0004170A2215298C0EB001000EB800018
:1084200002EBC0008170E5215298C0EB001000EB18
:10843000800002EBC000C1705298C0EB001000EB4E
:108440008000114601EBC00104910321049805F05E
:1084500035F901465298C0EB001000EB8000534AFA
:1084600002EBC000017105210F91EFE1F521529857
:10847000C0EB001000EB80004C4A02F830109DF871
:1084800054105298C0EB001000EB800002EBC000CB
:108490004170A2215298C0EB001000EB800002EB6B
:1084A000C0008170E7215298C0EB001000EB800003
:1084B00002EBC000C1705298C0EB001000EB8000CE
:1084C000114601EBC00104910321049805F0F6F870
:1084D00001465298C0EB001000EB8000334A02EBDB
:1084E000C000017105210F91B0E1F5215298C0EB58
:1084F000001000EB80002D4A02F830109DF8541057
:108500005298C0EB001000EB800002EBC0004170FD
:10851000A2215298C0EB001000EB800002EBC000DB
:10852000817011215298C0EB001000EB800002EB2B
:10853000C000C1705298C0EB001000EB80001146E3
:1085400001EBC00104910321049805F0B7F801463E
:108550005298C0EB001000EB8000144A02EBC00000
:10856000017105210F9101225298C0EBC00101EB6E
:1085700080110D4800EB41116031539800EB001061
:1085800001F83020D5225298C0EBC00101EB8011D8
:10859000054800EB41106030539901EB011100EBED
:1085A000C100427152E10000FC340020C45C002094
:1085B000F5215298C0EB001000EB8000FE4A02F853
:1085C00030109DF854105298C0EB001000EB800062
:1085D00002EBC0004170A5215298C0EB001000EBE7
:1085E000800002EBC000817001215298C0EB0010A6
:1085F00000EB800002EBC000C170C2215298C0EBBA
:10860000001000EB800002EBC000017100215298C5
:10861000C0EB001000EB800002EBC00041711221A2
:108620005298C0EB001000EB800002EBC00081719B
:108630005298C0EB001000EB8000114601EBC00126
:1086400004910621049805F039F801465298C0EBD0
:10865000001000EB8000D84A02EBC000C171082175
:108660000F91F3E0F5215298C0EB001000EB800071
:10867000D14A02F830109DF854105298C0EB001007
:1086800000EB800002EBC0004170FF215298C0EB6C
:10869000001000EB800002EBC000817000211A91F5
:1086A0001CE0529800EB400101EB0011C34800EBC5
:1086B00001110E31BDF86800095C5298C0EB001042
:1086C00000EB8000BC4A02EBC002BDF86800C01C91
:1086D0001154BDF86800401C81B21A91BDF86800C1
:1086E0000A28DEDB529800EB400101EB0011B34891
:1086F00000EB0110408B01125298C0EB001000EB10
:108700008000AD4A02EBC0004173529800EB40017B
:1087100001EB0011A94800EB0110408BC1B2529847
:10872000C0EB001000EB800002EBC0008173529898
:10873000C0EBC00101EB8011A14800EB4111603199
:10874000539800EB001001EBC000B0F88400011258
:108750005298C0EB001000EB800002EBC000C17328
:108760005298C0EBC00101EB8011954800EB41111C
:108770006031539800EB001001EBC000B0F88400AA
:10878000C1B25298C0EB001000EB800002EBC000B9
:1087900001745298C0EBC00101EB8011884800EBD6
:1087A00041116031539800EB001001EBC000B0F8AC
:1087B0008410529801EB802081B203200491F0F7DD
:1087C000EBFB00211A9114E07E49BDF86800095CBA
:1087D0005298C0EB001000EB8000774A02EBC00219
:1087E000BDF8680011301154BDF86800401C81B21A
:1087F0001A91BDF86800B0F5007FE5DB13215298AF
:10880000C0EB001000EB80006B4A02EBC00080F868
:1088100011125298C0EB001000EB8000114601EBE2
:10882000C001049140F21121049804F047FF014671
:108830005298C0EB001000EB80005F4A02EBC000D2
:1088400080F8121240F213210F9100BF00BF04F014
:1088500042B8529800EB400101EB0011574800EB81
:1088600001113031539801EB001041781591529865
:10887000C0EBC00101EB8011514800EB41116031A8
:10888000539800EB001011F830105298C0EBC00262
:1088900002EB80124A4800EB42100079814209D174
:1088A00001215298C0EBC00202EB8012444800EB59
:1088B0004210C1704449529801EB00115398085C72
:1088C000401CC1B2404A529802EB00125398115416
:1088D0009DF85400002804DD9DF85400401EC1B2EC
:1088E00015915498A1380A2870D2DFE800F0FCFBFB
:1088F000FAF9F8F7F605F5F402215298C0EB0010EA
:1089000000EB80002C4A02F830109DF854004030F3
:10891000C1B25298C0EB001000EB800002EBC00027
:10892000417041215298C0EB001000EB800002EB37
:10893000C000817030215298C0EB001000EB800025
:1089400002EBC000C1705298C0EB001000EB800039
:1089500002EBC00001715298C0EBC00101EB801125
:10896000174800EB41116031539800EB001001EB08
:10897000C000007901095298C0EB001000EB8000A4
:1089800002EBC00041715298C0EB001000EB800078
:10899000114601EBC00040790A281EDA5298C0EB5C
:1089A000001000EB800001EBC00040793030C1B214
:1089B0005298C0EB00100AE0C45C00203C3000205C
:1089C000FC340020AA240020702E002056E200EB88
:1089D000800002EBC000417113E05298C0EB001020
:1089E00000EB8000FE4901EBC00040793730C1B296
:1089F0005298C0EB001000EB8000F94A02EBC00077
:108A000041715298C0EBC00101EB8011F54800EBB9
:108A100041116031539800EB001001EBC000007968
:108A200000F00F015298C0EB001000EB8000EC4A00
:108A300002EBC00081715298C0EB001000EB800087
:108A4000114601EBC00080790A2812DA5298C0EB77
:108A5000001000EB800001EBC00080793030C1B223
:108A60005298C0EB001000EB800002EBC000817157
:108A700013E05298C0EB001000EB8000D84901EBE6
:108A8000C00080793730C1B25298C0EB001000EBC3
:108A90008000D34A02EBC000817103225298C0EBE0
:108AA000001000EB8000CE4901EBC000C27152986B
:108AB000C0EB001000EB800001EBC000401C072160
:108AC0000490F0F707FD01465298C0EB001000EB50
:108AD0008000C34A08E05EE1C1E0B4E397E3E7E267
:108AE000CDE10FE168E03DE002EBC0000172092139
:108AF0000F915298C0EBC00101EB8011B94800EB17
:108B000041106030539901EB011110F83100042835
:108B10000ED105225298C0EBC00101EB8011B14883
:108B200000EB41106030539901EB011100F8312046
:108B300000215298C0EBC00202EB8012A94800EB62
:108B40004210C17006225298C0EBC00101EB8011A7
:108B5000A44800EB41106030539901EB011100F87B
:108B6000312085E304215298C0EB001000EB800017
:108B70009B4A02F830109DF854004030C1B2529820
:108B8000C0EB001000EB800002EBC00041705121EF
:108B90005298C0EB001000EB800002EBC000817027
:108BA00005215298C0EB001000EB800002EBC000E2
:108BB000C17004210F915BE302215298C0EB0010B9
:108BC00000EB8000864A02F830109DF854004030D7
:108BD000C1B25298C0EB001000EB800002EBC00065
:108BE000417041215298C0EB001000EB800002EB75
:108BF000C000817031215298C0EB001000EB800062
:108C000002EBC000C17035215298C0EB001000EBA0
:108C1000800002EBC000017103215298C0EB0010EC
:108C200000EB800002EBC00041715298C0EB0010D5
:108C300000EB8000114601EBC000401C05210490B0
:108C4000F0F748FC01465298C0EB001000EB8000A2
:108C5000634A02EBC000817107210F9108E30221F2
:108C60005298C0EB001000EB80005D4A02F8301013
:108C70009DF854004030C1B25298C0EB001000EB98
:108C8000800002EBC000417041215298C0EB0010FF
:108C900000EB800002EBC000817032215298C0EBE3
:108CA000001000EB800002EBC000C1703021529830
:108CB000C0EB001000EB800002EBC000017103214B
:108CC0005298C0EB001000EB800002EBC000417135
:108CD0005298C0EB001000EB8000114601EBC00081
:108CE000401C05210490F0F7F5FB01465298C0EBBB
:108CF000001000EB80003A4A02EBC00081710721AE
:108D00000F91B5E204215298C0EB001000EB8000F7
:108D1000334A02F830109DF854004030C1B25298E6
:108D2000C0EB001000EB800002EBC000417041215D
:108D30005298C0EB001000EB800002EBC000817085
:108D400005215298C0EB001000EB800002EBC00040
:108D5000C17004210F915298C0EBC00101EB80114A
:108D6000204800EB41106030539901EB011110F8DD
:108D7000310002280ED103225298C0EBC00101EB52
:108D80008011184800EB41106030539901EB01113C
:108D900000F831206CE202215298C0EB001000EB89
:108DA00080000F4A02F830109DF854004030C1B2E4
:108DB0005298C0EB001000EB800002EBC000417045
:108DC00041215298C0EB001000EB800002EBC00084
:108DD000817031215298C0EB001000EB800003E05D
:108DE000C45C0020FC34002002EBC000C1703221C2
:108DF0005298C0EB001000EB800002EBC000017144
:108E000003215298C0EB001000EB800002EBC00081
:108E100041715298C0EB001000EB8000114601EB4D
:108E2000C000401C05210490F0F754FB0146529805
:108E3000C0EB001000EB8000FE4A02EBC000817125
:108E400007210F91529800EB400101EB0011FA4805
:108E500000EB01113031539801EB0010807820F0C5
:108E60002002529800EB400101EB0011F24800EBA8
:108E700001103030539900EB01108270F8E10221AB
:108E80005298C0EB001000EB8000EA4A02F8301064
:108E90009DF854004030C1B25298C0EB001000EB76
:108EA000800002EBC000417041215298C0EB0010DD
:108EB00000EB800002EBC000817031215298C0EBC2
:108EC000001000EB800002EBC000C170302152980E
:108ED000C0EB001000EB800002EBC0000171529863
:108EE000C0EBC00101EB8011D44800EB41106030B1
:108EF000539901EB011100EBC1008068B0F5100F30
:108F000009D330215298C0EB001000EB800002EB37
:108F1000C000417109E032215298C0EB001000EB13
:108F20008000C44A02EBC00041715298C0EBC001FE
:108F300001EB8011C14800EB41106030539901EB07
:108F4000011100EBC100C07901280AD131215298EA
:108F5000C0EB001000EB8000B64A02EBC00081714C
:108F600019E05298C0EBC00101EB8011B34800EB4F
:108F700041106030539901EB011100EBC100C07941
:108F800048B932215298C0EB001000EB8000A94A8A
:108F900002EBC000817100201A9028E05298C0EBCB
:108FA000C00101EB8011A54800EB411160315398DD
:108FB00000EB001001EBC0008168BDF86800C0F153
:108FC00005008000C14001F00F0130315298C0EB24
:108FD000001000EB8000974A02EBC002BDF8680069
:108FE000C01D1154BDF86800401C81B21A91BDF833
:108FF00068000628D2DB32215298C0EB001000EB4B
:1090000080008C4A02EBC000417300211A9128E0D5
:109010005298C0EBC00101EB8011884800EB411170
:109020006031539800EB001001EBC000416BBDF8BC
:109030006800C0F103008000C14001F00F01303131
:109040005298C0EB001000EB80007A4A02EBC0029D
:10905000BDF868000E301154BDF86800401C81B2A4
:109060001A91BDF868000428D2DB03225298C0EBA5
:10907000001000EB80006F4901EBC0008274529831
:10908000C0EB001000EB800001EBC000401C12217F
:109090000490F0F71FFA01465298C0EB001000EB65
:1090A0008000644A02EBC000C17414210F91DFE01C
:1090B00002215298C0EB001000EB80005D4A02F8DC
:1090C00030109DF854004030C1B25298C0EB0010EF
:1090D00000EB800002EBC000417041215298C0EBD0
:1090E000001000EB800002EBC0008170322152982A
:1090F000C0EB001000EB800002EBC000C17031211A
:109100005298C0EB001000EB800002EBC000017130
:1091100032215298C0EB001000EB800002EBC0003F
:1091200041715298C0EB001000EB800002EBC000D0
:10913000817100211A9128E05298C0EBC00101EB27
:1091400080113E4800EB41116031539800EB001054
:1091500001EBC000416BBDF86800C0F10300800066
:10916000C14001F00F0130315298C0EB001000EB0C
:109170008000304A02EBC002BDF86800C01D1154E7
:10918000BDF86800401C81B21A91BDF8680004283F
:10919000D2DB00201A9011E030215298C0EB001071
:1091A00000EB8000234A02EBC002BDF868000B30E0
:1091B0001154BDF86800401C81B21A91BDF86800D6
:1091C0001928E9DB03225298C0EB001000EB800065
:1091D000184901EBC00080F824205298C0EB001021
:1091E00000EB800001EBC000401C24210490F0F74C
:1091F00071F901465298C0EB001000EB80000D4A57
:1092000002EBC00080F8251026210F9130E01021DC
:109210005298C0EB001000EB8000064A02F83010B4
:1092200030215298C0EB001000EB800002EBC00030
:10923000417005E0C45C00203C300020FC3400207C
:1092400002210F9114E010215298C0EB001000EBA6
:109250008000FE4A02F8301031215298C0EB001015
:1092600000EB800002EBC000417002210F9100BFB3
:1092700000BF03F030BB529800EB400101EB00113E
:10928000F34800EB01113031539801EB00104178A5
:1092900015915298C0EBC00101EB8011ED4800EB35
:1092A00041116031539800EB001011F830105298C2
:1092B000C0EBC00202EB8012E64800EB42100079DE
:1092C000814209D101215298C0EBC00202EB801209
:1092D000E04800EB4210C170DF49529801EB0011E9
:1092E0005398085C401CC1B2DB4A529802EB001252
:1092F000539811549DF85400002804DD9DF8540043
:10930000401EC1B215915498A1380A282FD2DFE827
:1093100000F0052FD5FCFBFAF92E82F804215298B3
:10932000C0EB001000EB8000C84A02F830109DF836
:1093300054004030C1B25298C0EB001000EB8000E6
:1093400002EBC000417051215298C0EB001000EBBD
:10935000800002EBC000817005215298C0EB001024
:1093600000EB800002EBC000C17004210F91FAE312
:1093700002215298C0EB001000EB8000B34A02F8C3
:1093800030109DF854004030C1B25298C0EB00102C
:1093900000EB800002EBC000417041215298C0EB0D
:1093A000001000EB800002EBC00081703121529868
:1093B000C0EB001000EB800002EBC000C170352153
:1093C0005298C0EB001000EB800002EBC00001716E
:1093D00003215298C0EB001000EB800002EBC000AC
:1093E00041715298C0EB001000EB8000114601EB78
:1093F000C000401C05210490F0F76CF8014652981B
:10940000C0EB001000EB8000904A02EBC0008171BD
:1094100007210F91A7E302215298C0EB001000EB47
:1094200080008A4A02F830109DF854004030C1B2E2
:109430005298C0EB001000EB800002EBC0004170BE
:1094400041215298C0EB001000EB800002EBC000FD
:10945000817032215298C0EB001000EB800002EBCB
:10946000C000C17030215298C0EB001000EB8000AA
:1094700002EBC000017103215298C0EB001000EB19
:10948000800002EBC00041715298C0EB001000EB6D
:109490008000114601EBC000401C05210490F0F74C
:1094A00019F801465298C0EB001000EB8000674AA3
:1094B00002EBC000817107210F9154E304215298FF
:1094C000C0EB001000EB8000604A02F830109DF8FD
:1094D00054004030C1B25298C0EB001000EB800045
:1094E00002EBC000417041215298C0EB001000EB2C
:1094F000800002EBC000817005215298C0EB001083
:1095000004E00BE01AE304E34DE276E000EB8000B8
:1095100002EBC000C17004210F9124E30221529894
:10952000C0EB001000EB8000484A02F830109DF8B4
:1095300054004030C1B25298C0EB001000EB8000E4
:1095400002EBC000417041215298C0EB001000EBCB
:10955000800002EBC000817031215298C0EB0010F6
:1095600000EB800002EBC000C17032215298C0EBCA
:10957000001000EB800002EBC00001710321529843
:10958000C0EB001000EB800002EBC000417152986C
:10959000C0EB001000EB8000114601EBC000401C46
:1095A00005210490EFF796FF01465298C0EB00109A
:1095B00000EB8000254A02EBC0008171529800EB5D
:1095C000400101EB0011224800EB011130315398AA
:1095D00001EB0010807820F02002529800EB40014F
:1095E00001EB00111A4800EB01113031539801EBE7
:1095F0000010827007210F91B5E202215298C0EB52
:10960000001000EB8000114A02F830109DF8540061
:109610004030C1B25298C0EB001000EB800002EB6A
:10962000C000417041215298C0EB001000EB800057
:1096300002EBC000817031215298C0EB001000EBAA
:10964000800002EBC000C170412107E0C45C002033
:109650003C300020FC340020702E00205298C0EBDB
:10966000001000EB800002EBC00001715298C0EBCB
:10967000C00101EB8011FE4800EB411060305399AE
:1096800001EB011100EBC1008068B0F1104F09D16E
:1096900030215298C0EB001000EB800002EBC000BC
:1096A000417109E032215298C0EB001000EB8000BC
:1096B000F04A02EBC00041715298C0EBC00101EBCF
:1096C0008011EB4800EB41106030539901EB011120
:1096D00000EBC100C07901280AD131215298C0EBBA
:1096E000001000EB8000E34A02EBC000817119E03A
:1096F0005298C0EBC00101EB8011DD4800EB411036
:109700006030539901EB011100EBC100C07948B9F9
:1097100032215298C0EB001000EB8000D54A02EBDA
:10972000C000817100201A9028E05298C0EBC0015F
:1097300001EB8011CE4800EB41116031539800EBF2
:10974000001001EBC0008168BDF86800C0F107009F
:109750008000C14001F00F0130315298C0EB001081
:1097600000EB8000C34A02EBC002BDF86800C01DD8
:109770001154BDF86800401C81B21A91BDF8680010
:109780000828D2DB32215298C0EB001000EB800099
:10979000B84A02EBC000C17300211A9128E0529828
:1097A000C0EBC00101EB8011B14800EB4111603109
:1097B000539800EB001001EBC000416BBDF868004E
:1097C000C0F105008000C14001F00F013031529816
:1097D000C0EB001000EB8000A64A02EBC002BDF80F
:1097E000680010301154BDF86800401C81B21A9115
:1097F000BDF868000628D2DB30215298C0EB00107B
:1098000000EB80009B4A02EBC000817500211A9199
:1098100011E030215298C0EB001000EB8000954A17
:1098200002EBC002BDF8680017301154BDF86800A3
:10983000401C81B21A91BDF868000628E9DB30218E
:109840005298C0EB001000EB80008A4A02EBC00087
:10985000417700211A9111E030215298C0EB00109D
:1098600000EB8000834A02EBC002BDF868001E30A6
:109870001154BDF86800401C81B21A91BDF868000F
:109880000628E9DB30215298C0EB001000EB800085
:10989000784A02EBC00080F8241000211A9111E0F0
:1098A00030215298C0EB001000EB8000714A02EBAF
:1098B000C002BDF8680025301154BDF86800401C96
:1098C00081B21A91BDF868000628E9DB3021529870
:1098D000C0EB001000EB8000664A02EBC00080F88D
:1098E0002B1000211A9111E030215298C0EB00108A
:1098F00000EB80005F4A02EBC002BDF868002C302C
:109900001154BDF86800401C81B21A91BDF868007E
:109910000628E9DB30215298C0EB001000EB8000F4
:10992000544A02EBC00080F8321000211A9111E075
:1099300030215298C0EB001000EB80004D4A02EB42
:10994000C002BDF8680033301154BDF86800401CF7
:1099500081B21A91BDF868000628E9DB032252980B
:10996000C0EB001000EB8000424901EBC00080F822
:1099700039205298C0EB001000EB800001EBC000D2
:10998000401C39210490EFF7A5FD01465298C0EB29
:10999000001000EB8000374A02EBC00080F83A105C
:1099A0003B210F91DFE002215298C0EB001000EB49
:1099B0008000304A02F830109DF854004030C1B2A7
:1099C0005298C0EB001000EB800002EBC000417029
:1099D00041215298C0EB001000EB800002EBC00068
:1099E000817032215298C0EB001000EB800002EB36
:1099F000C000C17031215298C0EB001000EB800014
:109A000002EBC000017133215298C0EB001000EB53
:109A1000800002EBC000417132215298C0EB00106F
:109A200000EB800002EBC000817100211A912EE052
:109A30005298C0EBC00101EB80110D4800EB4111C1
:109A40006031539800EB001001EBC000416BBDF892
:109A50006800C0F105008000C14001F00F01303105
:109A60005298C0EB001000EB8000024A04E00000B6
:109A7000FC340020C45C002002EBC002BDF868008A
:109A8000C01D1154BDF86800401C81B21A91BDF888
:109A900068000628CCDB00201A9011E03021529893
:109AA000C0EB001000EB8000FE4A02EBC002BDF8E4
:109AB00068000D301154BDF86800401C81B21A9145
:109AC000BDF868001928E9DB03225298C0EB0010AA
:109AD00000EB8000F34901EBC00080F8262052988B
:109AE000C0EB001000EB800001EBC000401C262101
:109AF0000490EFF7EFFC01465298C0EB001000EB2A
:109B00008000E84A02EBC00080F8271028210F915E
:109B100029E010215298C0EB001000EB8000E14AD0
:109B200002F8301030215298C0EB001000EB80009A
:109B300002EBC000417002210F9114E010215298F5
:109B4000C0EB001000EB8000D64A02F83010312143
:109B50005298C0EB001000EB800002EBC000417097
:109B600002210F9100BF00BF02F0B5BE529800EB7A
:109B7000400101EB0011CC4800EB0111303153984A
:109B800001EB0010417815915298C0EBC00101EB38
:109B90008011C64800EB41116031BDF8680000EB50
:109BA000001011F830105298C0EBC00202EB801286
:109BB000BE4800EB42100079814209D10121529840
:109BC000C0EBC00202EB8012B84800EB4210C1703B
:109BD000B749529801EB00115398085C401CC1B280
:109BE000B34A529802EB00125398115400211A9173
:109BF00017E0529800EB400101EB0011AA4800EB7E
